:100000000C944D160C947E160C947E160C947E1651
:100010000C947E160C947E160C947E160C947E1610
:100020000C947E160C947E160C947E160C947E1600
:100030000C947E160C9435460C947E160C947E1609
:100040000C947E160C94F4490C947E160C947E1637
:100050000C947E160C947E160C9417660C943A63DE
:100060000C947E160C9427970C947E160C947E1696
:100070000C947E160C947E160C947E160C947E16B0
:100080000C947E160C947E160C947E160C947E16A0
:100090000C947E160C947E160C947E160C947E1690
:1000A0000C947E160C947E160C947E160C947E1680
:1000B0000C947E160C947E160C947E160C947E1670
:1000C0000C947E160C947E160C947E160C947E1660
:1000D0000C947E160C947E160C94129B0C94D39A5E
:1000E0000C947E16363853388438A138B638DF3849
:1000F0004E39B439653A663D743D6D3DA83DAC3D21
:10010000BD3D2842D23D223E543E7B3EA43EF83EB9
:10011000093F1A3F2B3F3C3F4D3F2842A440284215
:10012000AF409441A841D44107600A60F95FFD5F88
:10013000036041600E60126018601C6020602660E1
:100140002A602E604160346038603C602161266125
:100150002B6135613F61B8614961516159616361EA
:100160006D61776186619061B8619A61A461AE61E9
:10017000084AD73B3BCE016E84BCBFFDC12F3D6C0E
:1001800074319ABD56833DDA3D00C77F11BED9E474
:10019000BB4C3E916BAAAABE000000803F05A84C54
:1001A000CDB2D44EB93836A9020C50B99186880820
:1001B0003CA6AAAA2ABE000000803F004E414E493C
:1001C0004E495459494E46CDCCCC3D0AD7233C1715
:1001D000B7D13877CC2B329595E6241FB14F0A0062
:1001E0000020410000C84200401C4620BCBE4CCA52
:1001F0001B0E5AAEC59D74434F4D4D554E4943415C
:1002000054494F4E0044525952554E004552524F98
:10021000525300494E464F004543484F0047322F46
:1002200047332062616420706172616D657465722C
:10023000730A004D65736820706F696E7420636186
:100240006E6E6F74206265207265736F6C76656484
:100250000A00456E642066696C65206C6973740AD7
:1002600000426567696E2066696C65206C6973740D
:100270000A00286E6F2066696C652900534420705F
:1002800072696E74696E67206279746520004E6FC2
:1002900074205344207072696E74696E670A00435B
:1002A000757272656E742066696C653A200018027A
:1002B00013020C020502F7016F66660044454255C1
:1002C000473A004B494C4C45442E20004D313133C8
:1002D0002053006F6B005446542053657269616C63
:1002E0002044656275673A204E6F7A7A6C652069A2
:1002F000732068656174696E672E2E2E204A303631
:100300000A004A3036005446542053657269616CC5
:100310002044656275673A20436F6E74696E756933
:100320006E67205344207072696E74206166746534
:10033000722068656174696E672E2E2E204A3034F3
:100340000A004A3034005446542053657269616C87
:100350002044656275673A204E6F7A7A6C65206832
:10036000656174696E6720697320646F6E652E2EF7
:100370002E204A30370A004A30370020573A0054BE
:1003800046542053657269616C2044656275673A12
:10039000204265642069732068656174696E672E08
:1003A0002E2E204A30380A004A3038005446542055
:1003B00053657269616C2044656275673A204265D5
:1003C000642068656174696E6720697320646F6E6C
:1003D000652E2E2E204A30390A004A303900205727
:1003E0003A00544845524D414C5F50524F5445439A
:1003F00054494F4E004155544F5245504F52545F4F
:1004000053445F53544154555300454D455247455D
:100410004E43595F50415253455200434153455F4B
:100420004C494748545F4252494748544E455353FC
:1004300000544F47474C455F4C494748545300537D
:100440004F4654574152455F504F57455200425511
:10045000494C445F50455243454E54004C45564527
:100460004C494E475F44415441005A5F50524F42FD
:1004700045004155544F4C4556454C005052494E4D
:10048000545F4A4F420050524F4752455353004128
:1004900055544F5245504F52545F54454D5000569D
:1004A0004F4C554D455452494300454550524F4DD0
:1004B0000053455249414C5F584F4E5F584F464696
:1004C000004649524D574152455F4E414D453A4DC8
:1004D00061726C696E206275676669782D312E31A4
:1004E0002E7820284769746875622920534F555229
:1004F00043455F434F44455F55524C3A68747470AE
:10050000733A2F2F6769746875622E636F6D2F4D74
:1005100061726C696E4669726D776172652F4D61AB
:10052000726C696E2050524F544F434F4C5F56458A
:100530005253494F4E3A312E30204D414348494E97
:10054000455F545950453A3344205072696E746582
:10055000722045585452554445525F434F554E54AE
:100560003A3120555549443A6365646532613266D3
:100570002D343161322D343734382D396231322DFA
:100580006335356336326633363766660A00205483
:1005900000205200416363656C65726174696F6E1F
:1005A0003A2050005741524E494E4721204C6F7718
:1005B000205A204A65726B206D6179206C656164F8
:1005C00020746F20756E77616E746564207061753C
:1005D0007365732E0A00546F6F2066617220667215
:1005E0006F6D207265666572656E636520706F69F8
:1005F0006E740A00205A00205900580020204D61D6
:10060000783A2000205A00205900580020204D69D7
:100610006E3A20004F6E20004F666600536F66747E
:1006200020656E6473746F70733A200020466C6F9F
:10063000773A20000001363726032BFFFFFF3C3DB1
:10064000382AFFFFFFFF2E303E12FFFFFFFFFF02A1
:10065000FF0809FF2C071A1C18FFFFFF08440A2C8B
:100660004324221E20643A0020693A0020703A0098
:10067000496E76616C696420657874727564657220
:100680000A0043290A0061626C656420286D696E66
:100690002074656D702000436F6C642065787472FF
:1006A0007564657320617265200023646566696EF8
:1006B000652044454641554C545F4B6420002364FB
:1006C0006566696E652044454641554C545F4B69EB
:1006D000200023646566696E652044454641554C9B
:1006E000545F4B702000504944204175746F7475FD
:1006F0006E652066696E6973686564212050757443
:1007000020746865206C617374204B702C204B69D9
:1007100020616E64204B6420636F6E7374616E742D
:10072000732066726F6D2062656C6F7720696E74DE
:100730006F20436F6E66696775726174696F6E2EA4
:10074000680A00504944204175746F74756E6520C5
:100750006661696C6564212074696D656F75740AE2
:1007600000453120544845524D414C2052554E4190
:1007700057415900546865726D616C2052756E6105
:100780007761790045312048656174696E6720663C
:1007900061696C65640048656174696E67206661B3
:1007A000696C656400504944204175746F74756EBE
:1007B00065206661696C6564212054656D706572A1
:1007C000617475726520746F6F20686967680A00CC
:1007D000204B643A2000204B693A2000204B703AAD
:1007E00020000A20436C61737369632050494420E0
:1007F0000A002054753A2000204B753A2000206DE5
:1008000061783A2000206D696E3A200020643A2019
:100810000020626961733A20005049442041757498
:100820006F74756E65206661696C65642120426134
:1008300064206578747275646572206E756D62658A
:10084000720A00504944204175746F74756E6520BA
:1008500073746172740A004E6F2063617365206C5B
:10086000696768740A004F66660A0046616465201D
:100870004865696768742000426564204C65766548
:100880006C696E6720004661696C656420746F2036
:10089000656E61626C6520426564204C6576656CAE
:1008A000696E670A004D65736820706F696E742009
:1008B00063616E6E6F74206265207265736F6C7613
:1008C00065640A004D34323120696E636F7272655F
:1008D000637420706172616D6574657220757361F7
:1008E00067650A00205A004475616C20456E647388
:1008F000746F702041646A7573746D656E7420281E
:100900006D6D293A20003A200050726F6265205ABE
:10091000204F6666736574003F5A206F7574206FB0
:10092000662072616E676520282D323020746F203A
:100930003230290A00416374697665204578747203
:10094000756465723A2000496E76616C6964206551
:10095000787472756465720A0043616E6E6F7420FC
:10096000656E746572207375626469723A20004D19
:10097000353031005370656369616C204D656E756B
:100980003A205265616420454550524F4D0A004D52
:10099000353030005370656369616C204D656E754C
:1009A0003A205361766520454550524F4D0A004725
:1009B00032380A473239005370656369616C204DE3
:1009C000656E753A204175746F20426564204C65F0
:1009D00076656C696E670A004D33303320433820EA
:1009E00053323030005370656369616C204D656E21
:1009F000753A204175746F2054756E6520504944D6
:100A00000A003C5370656369616C5F4D656E753EAD
:100A1000003C5370656369616C5F4D656E753E00A7
:100A20002F002F002F002F2E2E0A002F2E2E002FEA
:100A30002E2E003C5370656369616C5F4D656E7569
:100A40003E0A003C5370656369616C204D656E75AC
:100A50003E003C5370656369616C204D656E753E68
:100A6000003C5265616420454550524F4D3E003C6C
:100A70005265616420454550524F4D3E003C5361E4
:100A8000766520454550524F4D3E003C536176659A
:100A900020454550524F4D3E003C4175746F2042F9
:100AA0006564204C6576656C696E673E003C4175F7
:100AB000746F20426564204C6576656C696E673E94
:100AC000003C4175746F2054756E6520486F7465E5
:100AD0006E64205049443E003C4175746F2054754B
:100AE0006E6520486F74656E64205049443E003C3A
:100AF000457869743E003C457869743E0056313152
:100B000036004A333320004D3530300A4D34323010
:100B10002053310A4731205A313020463234300ACE
:100B2000473120583020593020463630303000547C
:100B30004654204C6576656C20736176696E67203B
:100B4000646174612E2E2E0A004D353030004D3810
:100B50003531205A003E0A0041395620005446548F
:100B60002073656E64696E672063757272656E745A
:100B7000207A2D70726F6265206F666673657420CF
:100B8000646174612E2E2E203C00413956200054A1
:100B900046542053657269616C2044656275673AFA
:100BA000204C6576656C696E67207072696E742082
:100BB0007465737420776974682068656174696E00
:100BC0006720646F6E652E2E2E204A32320A004A4C
:100BD000323200544654204C6576656C206368655B
:100BE000636B2068656174696E672E2E2E0A00544F
:100BF00046542053657269616C2044656275673A9A
:100C0000204C6576656C696E67207072696E742021
:100C10007465737420646F6E652E2E2E204A3232F6
:100C20000A004A323200544654204C6576656C20E6
:100C3000636865636B206E6F2068656174696E67B9
:100C40002E2E2E0A004731205A3520463234300AE3
:100C50004731205831393020593230204636303033
:100C6000300A4731205A302046323430005446543E
:100C7000204C6576656C20636865636B706F696E88
:100C800074206261636B2072696768742E2E2E0A6D
:100C9000004731205A3520463234300A4731205837
:100CA00031393020593139302046363030300A471A
:100CB00031205A30204632343000544654204C659E
:100CC00076656C20636865636B706F696E74206213
:100CD00061636B2072696768742E2E2E0A0047319B
:100CE000205A3520463234300A47312058313930C5
:100CF000205932302046363030300A4731205A30C1
:100D0000204632343000544654204C6576656C20C1
:100D1000636865636B706F696E742066726F6E7462
:100D20002072696768742E2E2E0A004739310A47EF
:100D300031205A313020463234300A4739300A47A0
:100D400032380A4732390A47312058323020593276
:100D5000302046363030300A4731205A3020463273
:100D6000343000544654204C6576656C696E6720BB
:100D70007374617274656420616E64206D6F76694E
:100D80006E7420746F2066726F6E74206C6566746A
:100D90002E2E2E0A0054465420456E746572696EDC
:100DA00067206C6576656C206D656E75652E2E2EE0
:100DB0000A005446542053657269616C2044656290
:100DC00075673A205344206361726420696E6974C8
:100DD00069616C697A65642E2E2E204A30320A00D1
:100DE0004A3032005446542053657269616C204485
:100DF000656275673A20436F6F6C696E6720646F38
:100E0000776E2E2E2E204A31320A004A31320047A8
:100E100031205A3130004F4B004731205A313000D9
:100E20004739300047312045256946353030004785
:100E30003120452D302E314625690047312045307F
:100E40002E31462569004731205A2569462569001B
:100E50004731205A2D302E31462569004731205A1E
:100E6000302E3146256900473120592569462569CC
:100E700000473120592D302E314625690047312059
:100E800059302E31462569004731205825694625BD
:100E90006900473120582D302E31462569004731F1
:100EA0002058302E31462569004739310047323805
:100EB00000473238205A004732382059004732382C
:100EC0002058004132305620004731205A3130003E
:100ED0005446542053657269616C2044656275679D
:100EE0003A205374617274696E67205344205072C3
:100EF000696E742E2E2E204A30340A004A30340097
:100F00005446542053657269616C2044656275676C
:100F10003A2046696C65206F70656E206661696C69
:100F200065642E2E2E204A32310A004A3231005496
:100F300046542053657269616C2044656275673A56
:100F40002046696C65206F70656E207375636365FC
:100F5000737366756C2E2E2E204A32300A004A3288
:100F600030004B494C4C45442E20005446542053ED
:100F7000657269616C2044656275673A205344204C
:100F80007072696E7420737461727465642E2E2E93
:100F9000204A30340A004A303400454E4400464E60
:100FA00020004A3032003939393A393939004D0098
:100FB00048004137562000413656202D2D2D004A3D
:100FC00030320041365620005A3A2000593A20006B
:100FD000583A2000413556004134562000413356DE
:100FE0002000413256200041315620004130562029
:100FF000005446542053657269616C20436F6D6DD7
:10100000616E643A20004D383400544654205365D4
:101010007269616C2044656275673A2053442070A0
:1010200072696E742073746F707065642E2E2E203A
:101030004A31360A004A313600544654205365720C
:1010400069616C2044656275673A20534420707270
:10105000696E742070617573656420646F6E652EAF
:101060002E2E204A31380A004A3138004739310AD9
:101070004731205A313020463234300A4739300067
:101080005446542053657269616C204465627567EB
:101090003A205344207072696E7420646F6E652E1E
:1010A0002E2E204A31340A004A313400544654204E
:1010B00053657269616C2044656275673A205344D8
:1010C000206361726420696E7365727465642E2E8C
:1010D0002E204A30300A004A303000544654205303
:1010E000657269616C2044656275673A20534420DB
:1010F000636172642072656D6F7665642E2E2E209A
:101100004A30310A004A3031005446542053657247
:1011100069616C2044656275673A20486F74656E3A
:10112000642074656D7065726174757265206162AA
:101130006E6F726D616C2E2E2E204A32300A004A7C
:10114000313000025446542053657269616C20446A
:10115000656275673A2046696C616D656E742072D0
:10116000756E6F75742E2E2E204A31350A004A3165
:1011700035004A3132004A3137004B494C4C454426
:101180002E2000202D20496E76616C6964206578E0
:10119000747275646572206E756D62657220210AC5
:1011A000002020506C616E6E6572427566666572D5
:1011B00042797465733A20002046726565204D655A
:1011C0006D6F72793A2000436F6D70696C65643A97
:1011D0002044656320203820323031380A00207CDA
:1011E00020417574686F723A2028646572686F7068
:1011F000702C20416E796375626963206933204DDC
:10120000656761290A00323031382D30372D33318E
:1012100000204C61737420557064617465643A20D9
:10122000006275676669782D312E312E780A004D7F
:1012300061726C696E0020536F667477617265200D
:1012400052657365740A00205761746368646F6740
:101250002052657365740A002042726F776E206FAA
:1012600075742052657365740A0020457874657240
:101270006E616C2052657365740A00506F776572F9
:1012800055700A0073746172740A004D3234004D57
:101290003233202573006175746F25692E670065F0
:1012A00072726F722077726974696E6720746F2032
:1012B00066696C650A0020503A00205A3A002059AD
:1012C0003A0020583A00656E6473746F707320683A
:1012D00069743A2000446F6E6520736176696E67A9
:1012E0002066696C652E0A004D32390024F4D43032
:1012F00050C38E20C2A24017828B7011127A910DBA
:10130000816CD90AA861E108C75866076151430694
:101310001E4B5D05C145A7041A411104093D980300
:10132000713931034036DB0265339102D430540207
:10133000802E1D02632CEE01752AC501B028A00184
:10134000102781018F2564012B244B01E0223401F9
:10135000AC211F018D200D01801FFC00841EED00BB
:10136000971DDF00B81CD200E61BC600201BBC0086
:10137000641AB200B219A8000A19A0006A189900EC
:10138000D117910040178B00B516840031167E00EE
:10139000B31579003A157300C7146F0058146A002A
:1013A000EE1366008813630025135E00C7125B000E
:1013B0006C12570015125400C111510070114F00EA
:1013C00021114B00D61049008D10470046104400F3
:1013D00002104200C00F4000800F3E00420F3C0050
:1013E000060F3B00CB0E3800930E37005C0E350025
:1013F000270E3400F30D3200C10D3100900D300086
:10140000600D2E00320D2D00050D2C00D90C2B0087
:10141000AE0C2900850C29005C0C2700350C270038
:101420000E0C2600E80B2400C40B2400A00B2300A4
:101430007D0B23005A0B2100390B2100180B2000D3
:10144000F80A1F00D90A1E00BB0A1E009D0A1D00D3
:10145000800A1D00630A1C00470A1B002C0A1B009F
:10146000110A1A00F7091A00DD091900C409190048
:10147000AB091900920917007B09180063091700CE
:101480004C09160036091600200916000A09150035
:10149000F5081500E0081400CC081400B808140082
:1014A000A4081400900813007D0812006B081300B4
:1014B00058081200460812003408110023081100D1
:1014C0001208110001081100F0071000E0071000D9
:1014D000D0071000C0071000B0070F00A1071000D0
:1014E00091070E0083070F0074070F0065070E00B9
:1014F00057070E0049070E003B070D002E070E0090
:1015000020070D0013070D0006070D00F9060C005B
:10151000ED060D00E0060C00D4060C00C8060C0019
:10152000BC060C00B0060C00A4060B0099060C00CB
:101530008D060B0082060B0077060B006C060B0075
:1015400061060A0057060B004C060A0042060A0014
:1015500038060A002E060A0024060A001A060A00A7
:101560001006090007060A00FD050900F405090038
:10157000EB050900E2050900D9050900D0050900BD
:10158000C7050900BE050900B5050800AD0508003E
:10159000A50509009C050800940508008C050800B5
:1015A000840508007C050800740508006C05070028
:1015B000650508005D050700560508004E05070093
:1015C00047050700400508003805070031050700FA
:1015D0002A050700230507001C050600160507005D
:1015E0000F0507000805060002050700FB040600BA
:1015F000F5040700EE040600E8040600E204070014
:10160000DB040600D5040600CF040600C90406006A
:10161000C3040600BD040600B7040600B1040500BB
:10162000AC040600A6040600A00405009B04060006
:1016300095040500900406008A0405008504050051
:10164000800406007A040500750405007004050096
:101650006B04050066040500610405005C040500D8
:1016600057040500520405004D0405004804050018
:10167000430405003E0404003A0405003504050057
:10168000300404002C040500270404002304050092
:101690001E0404001A0404001604050011040400CA
:1016A0000D040400090405000404040000040400FF
:1016B000FC030400F8030400F4030400F003040036
:1016C000EC030400E8030400E4030400E003040066
:1016D000DC030400D8030400D4030400D003040096
:1016E000CC030400C8030300C503030024F404D999
:1016F000201BC40C5C0E9804C4095F0265077101CD
:10170000F405F900FB04B30048048700C103690035
:101710005803550003034500BE023A00840231001D
:1017200053022A002902250004022000E4011C00C3
:10173000C8011900AF0117009801140084011300BB
:10174000710110006101100051010E0043010D00F4
:1017500036010B002B010B0020010B0015010900C5
:101760000C01090003010800FB000800F300080059
:10177000EB000700E4000600DE000600D8000600CB
:10178000D2000600CC000500C7000500C20005001D
:10179000BD000400B9000400B5000400B10004005D
:1017A000AD000400A9000400A5000300A20003008E
:1017B0009F0004009B0003009800030095000200B6
:1017C00093000300900003008D0002008B000300D3
:1017D00088000200860002008400030081000200ED
:1017E0007F0002007D0002007B0002007900020001
:1017F0007700010076000200740002007200010010
:10180000710002006F0002006D0001006C00020018
:101810006A00010069000200670001006600010023
:101820006500010064000200620001006100010027
:10183000600001005F0002005D0001005C0001002B
:101840005B0001005A00010059000100580001002E
:10185000570001005600010055000100540001002E
:10186000530000005300010052000100510001002C
:10187000500001004F0001004E0000004E0001002A
:101880004D0001004C0001004B0000004B00010026
:101890004A00010049000100480000004800010022
:1018A000470001004600000046000100450000001E
:1018B0004500010044000100430000004300010016
:1018C0004200000042000100410000004100010010
:1018D000400001003F0000003F0001003E0000000A
:1018E0003E0001003D0000003D0001003C00000002
:1018F0003C0000003C0001003B0000003B000100F8
:101900003A0000003A0001003900000039000100EF
:1019100038000000380000003800010037000000E7
:1019200037000100360000003600000036000100DC
:1019300035000000350000003500010034000000D3
:1019400034000000340001003300000033000000C8
:1019500033000100320000003200000032000100BC
:1019600031000000310000003100010030000000B3
:1019700030000000300001002F0000002F000000A8
:101980002F0000002F0001002E0000002E0000009C
:101990002E0001002D0000002D0000002D00000091
:1019A0002D0001002C0000002C0000002C00000085
:1019B0002C0001002B0000002B0000002B00000079
:1019C0002B0001002A0000002A0000002A0000006D
:1019D0002A00010029000000290000002900000061
:1019E0002900000029000100280000002800000054
:1019F0002800000028000000280001002700000047
:101A00002700000027000000270000002700010039
:101A1000260000002600000026000000260000002E
:101A20002600010025000000250000002500000020
:101A30002500000025000000250001002400000012
:101A40002400000024000000240000002400010005
:101A500023000000230000002300000023000000FA
:101A600023000000230000002300010022000000EA
:101A700022000000220000002200000022000000DE
:101A800022000100210000002100000021000000D0
:101A900021000000210000002100000021000100C1
:101AA00020000000200000002000000020000000B6
:101AB00020000000200000002000000020000100A5
:101AC0001F0000001F0000001F0000001F0000009A
:101AD0001F0000001F0000001F0001001E0000008A
:101AE0001E0000001E0000001E000000C2310000A9
:101AF0001C260000F4190000D80F0000EB080000BD
:101B0000C004000075020000400100002CFFFFFF30
:101B1000FFFF0001010101016265640A002C2073CE
:101B2000797374656D2073746F70706564212048DB
:101B300065617465725F49443A200020746F6F20BC
:101B40006C6F6E6720657874727573696F6E207044
:101B5000726576656E7465640A0020636F6C64203C
:101B6000657874727573696F6E2070726576656ED4
:101B70007465640A00627573793A207061757365E3
:101B80006420666F7220696E7075740A00627573E6
:101B9000793A2070617573656420666F7220757381
:101BA00065720A00627573793A2070726F636573AB
:101BB00073696E670A005446542053657269616CFC
:101BC0002044656275673A2046696C616D656E7484
:101BD0002072756E6F75742E2E2E204A31350A00D4
:101BE0004A3135005446542053657269616C204473
:101BF000656275673A2046696C616D656E74207226
:101C0000756E6F7574207265636F76657265640AB0
:101C1000004B494C4C45442E20004B494C4C206312
:101C20006175736564206279204B494C4C20627564
:101C300074746F6E2F70696E0A004B494C4C4544AA
:101C40002E20004B494C4C20636175736564206203
:101C50007920746F6F206D75636820696E6163749D
:101C60006976652074696D65202D206375727265D3
:101C70006E7420636F6D6D616E643A20005446543B
:101C80002053657269616C2044656275673A204B28
:101C9000696C6C20636F6D6D616E642E2E2E204A10
:101CA00031310A004A3131005072696E7465722018
:101CB00068616C7465642E206B696C6C28292063E4
:101CC000616C6C6564210A000000A0C00000000087
:101CD0000000000000004842000048420000804030
:101CE000000000005761726E696E673A20486F6DA0
:101CF000696E672042756D702044697669736F72F2
:101D0000203C20310A000202040000A0400000A094
:101D10004000000040000057430000524300004DC7
:101D200043FFFFFF1000C90210012C0140012201F6
:101D300070011801B0010E01F00104015002FA0017
:101D4000B002F0003003E600D003DC009004D200C3
:101D50007005C800A006BE000008B400B009AA00C3
:101D6000D00BA000600E960060118C000015820060
:101D700020197800C01D6E00A0226400B0275A0010
:101D8000902C500000314600E0343C001038320006
:101D9000903A2800603C1E00A03D1400803E0A00DE
:101DA000203F00004265642068656174696E6720A9
:101DB0006661696C65640048656174696E67206678
:101DC00061696C65640045312048656174696E67BE
:101DD000206661696C65640048656174696E67209E
:101DE0006661696C65640070012C0190012701B087
:101DF000012201C0011D01F0011801100213013080
:101E0000020E016002090190020401C002FF0000FD
:101E100003FA004003F5008003F000D003EB00203C
:101E200004E6007004E100E004DC004005D700C0D7
:101E300005D2004006CD00D006C8008007C30030A0
:101E400008BE00F008B900C009B400B00AAF00B085
:101E50000BAA00D00CA500000EA000500F9B00C0E4
:101E60001096005012910000148C00C0158700B02D
:101E7000178200B0197D00D01B7800001E7300404F
:101E8000206E0090226900F024640040275F0090DB
:101E9000295A00E02B5500102E500020304B001026
:101EA000324600E033410090353C00103737007077
:101EB000383200A0392D00B03A2800A03B23006042
:101EC0003C1E00103D1900903D1400103E0F0070A4
:101ED0003E0A00C03E0500003F0000403FFBFF807F
:101EE0003FF6FFC03FF1FF453120544845524D4178
:101EF0004C2052554E4157415900424544205448C8
:101F000045524D414C2052554E415741590054685D
:101F100065726D616C2052756E6177617900453133
:101F2000204572723A204D415854454D500045723B
:101F3000723A204D415854454D5020424544004D81
:101F4000415854454D5020747269676765726564E5
:101F5000004531204572723A204D494E54454D504E
:101F6000004572723A204D494E54454D502042452D
:101F700044004D494E54454D502074726967676561
:101F8000726564004D383420582059205A2045008D
:101F9000202800202F002042403A0020403A000034
:101FA000002100240027002A002D0030003300010A
:101FB000010000040107010A010000220025002899
:101FC000002B002E00310034000201000005010842
:101FD000010B01000020002300260029002C002F07
:101FE000003200000100000301060109010505059A
:101FF00005070508080808020202020A0A08080480
:1020000004040401010101010101010303030303AD
:10201000030303040707070C0C0C0C0C0C0C0C023C
:1020200002020206060606060606060B0B0B0B0B43
:102030000B0B0B010210202008081020401020403C
:10204000800201020108040201010204081020407C
:10205000808040201008040201800402018040209A
:1020600010080402010804020101020408102040C3
:1020700080010204081020408000000A0B02090CB5
:102080000D0E08070304010000000000000000001E
:102090000000000000000000000000000000000040
:1020A00000000000001211100000000000000000FD
:1020B00000000000000000000000000000000065BB
:1020C0006E7175657565696E672022004E6F2043DD
:1020D0006865636B73756D2077697468206C696ED1
:1020E00065206E756D6265722C204C617374204C96
:1020F000696E653A20004B494C4C45442E200050F7
:1021000072696E7465722073746F70706564206498
:10211000756520746F206572726F72732E20466928
:102120007820746865206572726F7220616E642019
:10213000757365204D39393920746F207265737459
:102140006172742E202854656D70657261747572A9
:10215000652069732072657365742E205365742041
:10216000697420616674657220726573746172743B
:10217000696E67290A004E6F20436865636B73754B
:102180006D2077697468206C696E65206E756D626C
:1021900065722C204C617374204C696E653A200086
:1021A000636865636B73756D206D69736D617463CE
:1021B000682C204C617374204C696E653A20004C89
:1021C000696E65204E756D626572206973206E6F51
:1021D00074204C617374204C696E65204E756D627D
:1021E00065722B312C204C617374204C696E653AFA
:1021F00020004D313130004D3331005344207265A1
:102200006164206572726F720A00446F6E6520709F
:1022100072696E74696E672066696C650A00204990
:102220006E76616C6964206578747275646572207D
:10223000000000A0C00000000000000000000052EC
:10224000430000524300004D4320746F6F206C6FB9
:102250006E6720657874727573696F6E2070726531
:1022600076656E7465640A0020636F6C642065781F
:1022700074727573696F6E2070726576656E7465C1
:10228000640A00454550524F4D2064617461736982
:102290007A65206572726F722E0A00290A00206228
:1022A000797465733B2063726320005365747469AD
:1022B0006E67732053746F726564202800290A00CA
:1022C0002062797465733B2063726320002073740D
:1022D0006F7265642073657474696E6773207265CC
:1022E00074726965766564202800202863616C63D8
:1022F000756C6174656429210A0020213D20004528
:102300004550524F4D20435243206D69736D6174A7
:102310006368202D202873746F7265642920002063
:1023200053697A653A2000496E6465783A20002046
:102330004D61726C696E3D563535290A0028454558
:1023400050524F4D3D00454550524F4D20766572DD
:1023500073696F6E206D69736D61746368200043EB
:10236000616E6E6F74206F70656E20737562646944
:102370007220004739310A4731205A2D313020462A
:102380003234300A4739300053442063617264208C
:102390006F6B0A006F70656E526F6F7420666169B3
:1023A0006C65640A00766F6C756D652E696E697474
:1023B000206661696C65640A004572726F723A004A
:1023C000534420696E6974206661696C0A00656314
:1023D000686F3A005446542053657269616C20441A
:1023E000656275673A205344207072696E7420707C
:1023F00061757365642E2E2E204A30350A004A30EE
:1024000035005446542053657269616C20446562FE
:1024100075673A2046696C616D656E742072756EE1
:102420006F7574207768696C65207072696E746965
:102430006E672E2E2E204A32330A004A3233003D78
:10244000003F2061646472657373203A200020624B
:1024500079746573206F66206D656D6F7279206980
:102460006E697469616C697A65642E0A0A00556E3A
:1024700061626C6520746F20696E697469616C6952
:102480007A652E0A0A00496E697469616C697A6915
:102490006E672066726565206D656D6F727920626A
:1024A0006C6F636B2E0A0A0A00747275650A00204D
:1024B00072657475726E3D000A4D656D6F7279209C
:1024C000436F7272757074696F6E206465746563B2
:1024D00074656420696E2066726565206D656D6F38
:1024E000727920617265612E0A002020626C6F6330
:1024F0006B5F666F756E643D0020202000292066AA
:102500006F756E643D00202800207370203C2048C9
:1025100065617020002073703D000A5F5F62737315
:102520005F656E643A20003D000A265F5F62726B51
:1025300076616C3A20000A666D632829206E3D00A2
:10254000636865636B5F666F725F667265655F6D1A
:10255000656D6F72795F636F7272757074696F6E9B
:102560002829203D20002062797465732061742041
:10257000000A4C617267657374206672656520623B
:102580006C6F636B20697320000A4D656D6F727903
:1025900020436F7272757074696F6E206465746524
:1025A0006374656420696E2066726565206D656D73
:1025B0006F727920617265612E0A002062797465FC
:1025C0007320667265652061742000466F756E64C5
:1025D00020000A436F7272757074696E67206164BF
:1025E00064726573733A2000436F72727570746918
:1025F0006E672066726565206D656D6F7279206209
:102600006C6F636B2E0A0A000A537461636B20506F
:102610006F696E746572203A20000A737461727477
:10262000206F662066726565207370616365203A6D
:1026300020000A5F5F6273735F656E64203A20005A
:102640000A5F5F62726B76616C203A20007C3C3ED0
:102650005E2B3D3F2F5B5D3B2C2A225C0046696C64
:10266000652064656C657465643A0044656C6574E6
:10267000696F6E206661696C65642C2046696C65C3
:102680003A20002569730025696D202569730025AE
:1026900069682025696D20256973002569642025F6
:1026A00069682025696D20256973002569792025D1
:1026B0006964202569682025696D202569730050AB
:1026C00072696E742074696D653A200050726F747F
:1026D00065637465642050696E0A00205A3A0020D0
:1026E000593A0020436F756E7420583A0020453ADD
:1026F00000205A3A0020593A00583A003A00436103
:10270000703A002F2F2000454550524F4D204F4B1F
:102710000A003F4B2076616C7565206F7574206FE1
:10272000662072616E67652028302D3130292E0AAF
:1027300000416476616E6365204B3D0042696C69BF
:102740006E656172204C6576656C696E67204772B4
:1027500069643A0A00486F6D696E67206661696C4A
:10276000656400202844525952554E290047323999
:10277000204175746F20426564204C6576656C69F4
:102780006E67003F20284C2C522C462C4229206F8B
:102790007574206F6620626F756E64732E0A003F39
:1027A0002856296572626F7365206C6576656C20AA
:1027B000697320696D706C61757369626C6520283E
:1027C000302D34292E0A00426164205A2076616C33
:1027D00075650A004E6F2062696C696E65617220D2
:1027E000677269640A00205A3A200020593A200092
:1027F00042656420583A200048617264636F6465E2
:10280000642044656661756C742053657474696EE8
:102810006773204C6F616465640A00B80B0000B8F0
:102820000B00003C000000102700000000FA4300ED
:1028300000FA430000C040000070420000A04200C7
:1028400000A0420000C8430080CF433A0A0020287D
:102850006D6D290020204D393030204B004C696EC1
:1028600065617220416476616E63653A0A002020DA
:102870004D383531205A005A2D50726F6265204F05
:1028800066667365740020440020490020204D33A3
:1028900030312050005049442073657474696E676C
:1028A000733A0A00205A0020204D36363600456E15
:1028B0006473746F702061646A7573746D656E748F
:1028C0003A0A00205A00204A002020473239205777
:1028D000204900205A0020204D343230205300413E
:1028E00075746F20426564204C6576656C696E670F
:1028F0003A0A00205A0020590020204D323036205C
:102900005800486F6D65206F66667365743A0A00FB
:10291000204500205A002059002058002054002053
:10292000530020204D32303520420020453C6D615F
:10293000785F655F6A65726B3E0020583C6D617818
:102940005F785F6A65726B3E20593C6D61785F7994
:102950005F6A65726B3E205A3C6D61785F7A5F6A90
:1029600065726B3E00416476616E6365643A204235
:102970003C6D696E5F7365676D656E745F74696DDC
:10298000655F75733E20533C6D696E5F6665656477
:10299000726174653E20543C6D696E5F747261763D
:1029A000656C5F66656564726174653E0020540005
:1029B00020520020204D32303420500041636365A6
:1029C0006C65726174696F6E2028756E6974732FFF
:1029D0007332293A20503C7072696E745F61636390
:1029E000656C3E20523C726574726163745F616312
:1029F00063656C3E20543C74726176656C5F616304
:102A000063656C3E0A00204500205A0020590020D2
:102A1000204D3230312058004D6178696D756D2040
:102A2000416363656C65726174696F6E2028756EB1
:102A30006974732F7332293A0A00204500205A0026
:102A400020590020204D3230332058004D617869E4
:102A50006D756D2066656564726174657320287597
:102A60006E6974732F73293A0A00204500205A00BA
:102A700020590020204D393220580053746570735E
:102A80002070657220756E69743A0A0020204D32FC
:102A900030302044300A0020204D323030204400B5
:102AA0002044697361626C65640A0046696C616DFB
:102AB000656E742073657474696E67733A002020C4
:102AC000473231202020203B004572726F72207700
:102AD000726974696E6720746F20454550524F4D7E
:102AE000210A0057726974696E6720746F206669E5
:102AF0006C653A20006F70656E206661696C656474
:102B00002C2046696C653A20006F70656E20666106
:102B1000696C65642C2046696C653A200046696CD6
:102B2000652073656C65637465640A002053697A77
:102B3000653A200046696C65206F70656E65643A81
:102B400020002066696C653A2000646F696E67003A
:102B50006672657368004E6F772000454E442053BF
:102B60005542524F5554494E450A002220706F730A
:102B7000002220706172656E743A220053554252F1
:102B80004F5554494E452043414C4C207461726767
:102B900065743A22004B494C4C45442E2000747217
:102BA00079696E6720746F2063616C6C2073756245
:102BB0002D67636F64652066696C6573207769743F
:102BC0006820746F6F206D616E79206C6576656C1E
:102BD000732E204D4158206C6576656C2069733AE0
:102BE000006F70656E206661696C65642C204669B3
:102BF0006C653A2000556E6B6E6F776E20636F6D5B
:102C00006D616E643A20220050726F62696E6720B7
:102C10006661696C65640A00205A3A200020593ABE
:102C2000200042656420583A20002066697273745F
:102C30000A005A0059005800486F6D6520007A5FFD
:102C400070726F62653A20007A325F6D696E3A2069
:102C5000007A5F6D696E3A2000795F6D696E3A2087
:102C600000785F6D696E3A20005265706F7274690A
:102C70006E6720656E6473746F7020737461747511
:102C8000730A00736C6F743A00526573656E643A30
:102C900020006F6B0000E0D2BFD211241FBECFEF27
:102CA000D1E2DEBFCDBF00E00CBF13E0A0E0B2E098
:102CB000E8EBF3EC01E00BBF02C007900D92AA3FD6
:102CC000B107D9F726E1AAEFB3E001C01D92AC3EEF
:102CD000B207E1F716E1CCE4D6E100E006C02197A7
:102CE0000109802FFE010E9439E1CB34D10780E039
:102CF0000807A9F70E9406CD0C94CBE10C940000C4
:102D00002F923F924F925F926F927F928F929F92FB
:102D1000AF92BF92CF92DF92EF92FF920F931F93E9
:102D2000CF93DF93CDB7DEB7C559D1090FB6F8946D
:102D3000DEBF0FBECDBF21E020938B0680916316CE
:102D40008D3409F4D0C7843511F40C94D12E873416
:102D500011F00C94152F80916116909162168C31B0
:102D6000910509F408C684F48430910534F4823066
:102D700091058CF597FF28C0B2C7049709F0AFC73B
:102D80000E94BFA80C94172F8A32910509F4FBC545
:102D90005CF48D31910509F4F2C54E9709F09FC797
:102DA0000E94C9A70C94172F8B35910509F4C7C64B
:102DB0008C35910509F4C7C68A35910509F08FC78E
:102DC0001092FE030C94172F8091170281110C941E
:102DD0001C2F0C94172F20911702222311F40C940E
:102DE000172F11E0029709F010E00E94FBA882E57E
:102DF0000E941F98882309F44AC10E94D2956B0152
:102E00007C0140900C0450900D0460900E04709072
:102E10000F0420911004309111044091120450913C
:102E2000130428AF39AF4AAF5BAF80914710909140
:102E30004810A0914910B0914A108CAF9DAFAEAF31
:102E4000BFAF20914B1030914C1040914D105091DC
:102E50004E1028962CAF3DAF4EAF5FAF289720E0C5
:102E600030E0A901C701B6010E9417DA882309F4EE
:102E700068C5A30192016CAD7DAD8EAD9FAD0E9482
:102E800017DA81110FC028AD39AD4AAD5BAD289678
:102E90006CAD7DAD8EAD9FAD28970E9417DA88236B
:102EA00009F44FC520E030E0A901C701B6010E9436
:102EB00017DA881F8827881F18130BC080E090E05E
:102EC000A0E8BFE364968CAF9DAFAEAFBFAF649791
:102ED0000AC020E030E040E85FEB64962CAF3DAFE5
:102EE0004EAF5FAF6497A30192016CAD7DAD8EAD27
:102EF0009FAD0E942DDE2C966CAF7DAF8EAF9FAF45
:102F00002C9728AD39AD4AAD5BAD28966CAD7DAD43
:102F10008EAD9FAD28970E942DDE60966CAF7DAF81
:102F20008EAF9FAF60972C962CAD3DAD4EAD5FAD93
:102F30002C97CA01B9010E947CDA4B015C016096B2
:102F40002CAD3DAD4EAD5FAD6097CA01B9010E9499
:102F50007CDA9B01AC01C501B4010E942EDE0E9407
:102F600099E024966CAF7DAF8EAF9FAF249720E0A1
:102F700030E040E05FE30E947CDA4B015C01A70196
:102F80009601C701B6010E947CDA6B017C01A501A4
:102F90009401C501B4010E947CDA9B01AC01C70118
:102FA000B6010E942DDE0E9499E09B01AC0164965F
:102FB0006CAD7DAD8EAD9FAD64970E947CDA4B0108
:102FC0005C012CAD3DAD4EAD5FADC301B2010E94C1
:102FD0002EDE20E030E040E05FE30E947CDA6B010F
:102FE0007C0160966CAD7DAD8EAD9FAD60979058C5
:102FF00024962CAD3DAD4EAD5FAD24970E940ADF07
:103000009B01AC01C501B4010E947CDA9B01AC01BB
:10301000C701B6010E942EDEA30192010E942DDE9F
:103020006B017C0128962CAD3DAD4EAD5FAD289770
:1030300068AD79AD8AAD9BAD0E942EDE20E030E018
:1030400040E05FE30E947CDA2B013C0124962CAD2A
:103050003DAD4EAD5FAD24972C966CAD7DAD8EAD84
:103060009FAD2C970E940ADF9B01AC01C501B40102
:103070000E947CDA9B01AC01C301B2010E942EDEEA
:1030800028AD39AD4AAD5BAD0E942DDE14C089E498
:103090000E941F98882329F00E94D2956B017C0121
:1030A00003C0C12CD12C76018AE40E941F9888238A
:1030B000F9F00E94D29528966CAF7DAF8EAF9FAF8E
:1030C000289720E030E0A901C701B6010E9417DA75
:1030D00081111EC020E030E0A90128966CAD7DADC5
:1030E0008EAD9FAD28970E9417DA811111C029C4B7
:1030F00020E030E0A901C701B6010E9417DA882359
:1031000009F41FC428961CAE1DAE1EAE1FAE289734
:10311000D701C601B05888AF99AFAAAFBBAF289608
:103120002CAD3DAD4EAD5FAD289750582CAF3DAFA7
:103130004EAF5FAF9C01AD01BC01CD010E947CDAB6
:103140004B015C012CAD3DAD4EAD5FADCA01B90187
:103150000E947CDA9B01AC01C501B4010E942EDE05
:103160000E9499E0A0966CAF7DAF8EAF9FAFA09705
:1031700080910C0490910D04A0910E04B0910F0465
:1031800024968CAF9DAFAEAFBFAF2497A701960139
:10319000BC01CD010E942EDE64966CAF7DAF8EAF78
:1031A0009FAF649720911004309111044091120454
:1031B000509113042C962CAF3DAF4EAF5FAF2C97C0
:1031C00028962CAD3DAD4EAD5FAD28972C966CADDD
:1031D0007DAD8EAD9FAD2C970E942EDEA4966CAF78
:1031E0007DAF8EAF9FAFA49780914710909148100C
:1031F000A0914910B0914A1060968CAF9DAFAEAFD0
:10320000BFAF609764962CAD3DAD4EAD5FAD64979A
:10321000BC01CD010E942DDE6B017C0120914B1081
:1032200030914C1040914D1050914E1068962CAF3B
:103230003DAF4EAF5FAF6897A4962CAD3DAD4EADA0
:103240005FADA49768966CAD7DAD8EAD9FAD689770
:103250000E942DDE4B015C018091140490911504B5
:10326000A0911604B09117046C968CAF9DAFAEAFD1
:10327000BFAF6C979C01AD0160914F1070915010E1
:1032800080915110909152100E942DDE2B013C0133
:103290002091531030915410409155105091561078
:1032A000AC962CAF3DAF4EAF5FAFAC97809118049A
:1032B00090911904A0911A04B0911B04A8968CAFA8
:1032C0009DAFAEAFBFAFA897A701960168AD79AD2E
:1032D0008AAD9BAD0E947CDAE0966CAF7DAF8EAF7D
:1032E0009FAFE097A50194016CAD7DAD8EAD9FAD14
:1032F0000E947CDA9B01AC01E0966CAD7DAD8EAD99
:103300009FADE0970E942EDEE0966CAF7DAF8EAF52
:103310009FAFE097A501940168AD79AD8AAD9BADF3
:103320000E947CDA4B015C01A70196016CAD7DAD7A
:103330008EAD9FAD0E947CDA9B01AC01C501B4014A
:103340000E942DDEE0962CAD3DAD4EAD5FADE09719
:103350000E94A1DE6B017C0120E030E0A9010E9407
:1033600017DA87FF0AC02BED3FE049EC50E4C701B4
:10337000B6010E942EDE6B017C01112351F02BED72
:103380003FE049EC50E4C701B6010E942DDE6B011D
:103390007C0120E030E0A901C701B6010E9417DAE4
:1033A000811128C060962CAD3DAD4EAD5FAD6097EC
:1033B00024966CAD7DAD8EAD9FAD24970E9417DA3B
:1033C000811118C068962CAD3DAD4EAD5FAD6897CC
:1033D0002C966CAD7DAD8EAD9FAD2C970E9417DA0B
:1033E000811108C06BEDC62E6FE0D62E69ECE62E7B
:1033F00060E4F62EA7019601A0966CAD7DAD8EAD72
:103400009FADA0970E947CDA4B015C0120E030E088
:10341000A901C301B2010E9417DA8823C9F0A501EE
:103420009401C501B4010E947CDA4B015C01A30147
:103430009201C301B2010E947CDA9B01AC01C5017B
:10344000B4010E942EDE0E9499E04B015C010DC088
:1034500020E030E0A901C501B4010E9454E087FFDB
:1034600004C0B7FAB094B7F8B0942FE632E143E85D
:103470005AE3C501B4010E9417DA87FF02C00C9419
:10348000172FC501B4010E94A3DF0E9477DF1B0143
:10349000672B19F422242394312CB10180E090E0B1
:1034A0000E941BDA4B015C019B01AC01C701B60114
:1034B0000E940ADF24966CAF7DAF8EAF9FAF24973A
:1034C000A5019401C301B2010E940ADFA0966CAF6E
:1034D0007DAF8EAF9FAFA097A8962CAD3DAD4EAD02
:1034E0005FADA897AC966CAD7DAD8EAD9FADAC9742
:1034F0000E942DDEA50194010E940ADFAC966CAFFC
:103500007DAF8EAF9FAFAC9724962CAD3DAD4EAD49
:103510005FAD2497CA01B9010E947CDA20E030E057
:1035200040E05FE30E947CDA9B01AC0160E070E068
:1035300080E89FE30E942DDE68966CAF7DAF8EAF72
:103540009FAF68976C962CAD3DAD4EAD5FAD6C975F
:1035500029873A874B875C87A8968CAD9DADAEAD29
:10356000BFADA8978D879E87AF87B88B609101020A
:1035700070910202072E000C880B990B0E941DDA35
:103580002091420230914302409144025091450201
:103590000E947CDA2AE037ED43E25CE30E947CDAA9
:1035A0006CAB7DAB8EAB9FAB0E9442629B01AC01CA
:1035B00028533F4F4F4F5F4F6C962CAF3DAF4EAFF0
:1035C0005FAF6C9748AC59AC6AAC7BAC41E050E063
:1035D0002E965FAF4EAF2E9759E129965FAF299790
:1035E0002E962EAD3FAD2E972215330509F44EC110
:1035F0000E94C1670E944262DC01CB016C962CAD37
:103600003DAD4EAD5FAD6C97821B930BA40BB50B1C
:10361000B7FD10C00E9442629B01AC0128533F4F8E
:103620004F4F5F4F6C962CAF3DAF4EAF5FAF6C9777
:103630000E94C95529963FAD2997315029963FAF31
:103640002997332309F445C068962CAD3DAD4EADA6
:103650005FAD68976CAD7DAD8EAD9FAD0E947CDA9D
:103660006B017C0124962CAD3DAD4EAD5FAD249732
:10367000B201C3010E947CDAA70196010E942EDEEE
:103680007B018C0168962CAD3DAD4EAD5FAD68976A
:10369000B201C3010E947CDA4B015C0124962CAD7F
:1036A0003DAD4EAD5FAD24976CAD7DAD8EAD9FADA4
:1036B0000E947CDA9B01AC01C501B4010E942DDEA1
:1036C0002B013C01C701D8018CAF9DAFAEAFBFAF9E
:1036D0005BC02E964EAD5FAD2E97BA0180E090E0B4
:1036E0000E941BDA24962CAD3DAD4EAD5FAD249704
:1036F0000E947CDA4B015C010E9407DF6B017C01B8
:10370000C501B4010E948FE04B015C01A701960145
:1037100068AD79AD8AAD9BAD0E947CDA2B013C018E
:10372000A501940128966CAD7DAD8EAD9FAD289717
:103730000E947CDA9B01AC01C301B2010E942EDE23
:103740002B013C01A501940168AD79AD8AAD9BAD1B
:103750000E947CDA4B015C01A701960128966CADB2
:103760007DAD8EAD9FAD28970E947CDA9B01AC01A8
:10377000C501B4010E942DDE6CAF7DAF8EAF9FAF4F
:1037800059E129965FAF29979201A30164966CAD28
:103790007DAD8EAD9FAD64970E942EDE69837A83E6
:1037A0008B839C832CAD3DAD4EAD5FADA4966CADCF
:1037B0007DAD8EAD9FADA4970E942EDE6D837E837E
:1037C0008F839887A0962CAD3DAD4EAD5FADA09791
:1037D00069857A858B859C850E942EDE69877A872C
:1037E0008B879C87AC962CAD3DAD4EAD5FADAC9755
:1037F0006D857E858F8598890E942EDE6D877E87F8
:103800008F87988B80912202882321F0CE01019628
:103810000E940153E0908A061CA61DA61EA61FA6A4
:1038200089819A81AB81BC8188A399A3AAA3BBA3F8
:103830008D819E81AF81B8858CA39DA3AEA3BFA3CC
:1038400089859A85AB85BC8588A799A7AAA7BBA7B8
:10385000AE01485D5F4FBE016C5D7F4FCE0180962B
:103860000E94C684CE018C966C018E010C5C1F4FA9
:103870009E01235F3F4FAE01485D5F4FBE016C5D0F
:103880007F4F0C970E942A74811151C0E0908A06E4
:1038900018AA19AA1AAA1BAA809147109091481039
:1038A000A0914910B0914A1088A399A3AAA3BBA3E1
:1038B00080914B1090914C10A0914D10B0914E10F2
:1038C0008CA39DA3AEA3BFA380914F1090915010E5
:1038D000A0915110B091521088A799A7AAA7BBA791
:1038E000AE01485D5F4FBE016C5D7F4FCE0180969B
:1038F0000E94C684DE01D0966D018E010C5C1F4FC4
:1039000023E530E1AE01485D5F4FBE016C5D7F4F46
:10391000CE0180960E942A7480E1E7E4F0E1ACE0F9
:10392000B4E001900D928A95E1F70C94172F2E9632
:10393000EEADFFAD2E9731962E96FFAFEEAF2E97E0
:103940004FCEE9EBF3E284918F010F5F1F4F882385
:1039500021F00E941896F801F6CFEDE1F2E0849193
:103960008F010F5F1F4F882311F40C94172F0E94B3
:103970001896F801F4CF0E9403C30C94172F0E94ED
:103980004EAB0C94172F80911702882311F40C94DE
:10399000172F89E40E941F98182F882321F00E9476
:1039A000C897E62E01C0E12C8AE40E941F98082FD8
:1039B000882331F00E94C897F62E111104C00BC065
:1039C000F12C1123C1F032E03E1510F00C94BE35FD
:1039D000E3E3F2E004C042E04F15D0F30CC0849161
:1039E0008F010F5F1F4F882311F40C94172F0E9433
:1039F0001896F801F4CF0E940E961123F1F0209151
:103A00001010309111105E2D5203B001539F700DB4
:103A100011248091140890911508680F791F072EC2
:103A2000000C880B990B0E941DDA6093471070936D
:103A300048108093491090934A100023F1F0209190
:103A40001210309113104F2D4203B001439F700D9F
:103A500011242091160830911708620F731F072E4A
:103A6000000C880B990B0E941DDA60934B10709329
:103A70004C1080934D1090934E1080E50E941F983B
:103A80008823E9F00E940B748823A9F11123D9F04F
:103A900020E030E040E151E460914710709148101F
:103AA0008091491090914A100E942EDE6093471039
:103AB000709348108093491090934A1004C080E599
:103AC0000E94D897E1CF0023B1F020E030E040EB36
:103AD00051E460914B1070914C1080914D10909179
:103AE0004E100E942EDE60934B1070934C1080930A
:103AF0004D1090934E1086E40E941F988823D9F0B1
:103B00000E94D2956B017C0120E030E0A9010E9467
:103B100054E0181684F420E030E040E752E4C70196
:103B2000B6010E940ADF60934202709343028093C1
:103B30004402909345020E948F590C94172F2093B2
:103B4000FE030C94172F3FE5232E32E0332E49E974
:103B5000C42E46E0D42EE12CF12C00E010E0D1017F
:103B60008D911D010E941F98882309F44EC00E9468
:103B7000D2952B013C01133059F0F701E95AFF4E61
:103B800020813181428153810E942DDE2B013C0135
:103B9000F701E45FFB4F2081318142815381C301F2
:103BA000B2010E942DDE4B015C012DEB37E346E8AC
:103BB00055EB0E9454E087FD0AC02DEB37E346E841
:103BC00055E3C501B4010E9417DA1816F4F4133056
:103BD00051F4409218045092190460921A047092A1
:103BE0001B0401E012C0A5019401F60160817181FE
:103BF000828193810E942EDED6016D937D938D93F9
:103C00009C931397812F0E94596F1F5FB4E0CB0ED6
:103C1000D11CE4E0EE0EF11C143009F0A0CF00231B
:103C200009F459C0C0901804D0901904E0901A0407
:103C3000F0901B0420E030E0A901C701B6010E940A
:103C40002EDE2091BD103091BE104091BF105091DA
:103C5000C0100E947CDA0E945FE060935D0A70935E
:103C60005E0A80935F0A9093600AC0924D0AD092D8
:103C70004E0AE0924F0AF092500A90912B0A8091DE
:103C80002C0A981719F00E94E38325C00E944184F2
:103C900080916F0081FB992790F981FF05C0809189
:103CA0006F008D7F80936F0040915D0A50915E0A96
:103CB00060915F0A7091600A4093F8055093F9058E
:103CC0006093FA057093FB05992329F080916F00AA
:103CD000826080936F000E94DDA30C94172F0E94D6
:103CE000E7C30C94172F8091611690916216863766
:103CF000910509F414C50CF0CAC08135910509F489
:103D00003BC40CF06CC08B31910509F421C2ACF5B9
:103D10008631910509F4F3C10CF58231910509F45E
:103D200046C484F4419711F00C94CE2E5F988A9883
:103D300047988091080181708093060147981298F6
:103D40000C94172F8431910509F496C1459711F011
:103D50000C94CE2E0E9468910C94172F88319105F7
:103D600009F4D7C10CF4D1C18931910509F4DCC142
:103D70004A9709F4DFC10C94CE2E8032910509F4E4
:103D80008FC29CF48D31910511F40C94172F0CF413
:103D900079C28E31910509F47FC24F9711F00C94CE
:103DA000CE2E0E943AA60C94172F8B34910509F45D
:103DB00088C244F48A9711F00C94CE2E0E94BCA5C0
:103DC0000C94172F8C34910509F47FC28D34910522
:103DD00011F00C94CE2E0E9484490C94172F8B3630
:103DE000910509F4B7C36CF58C35910509F42FC41E
:103DF00084F48335910509F4D5C30CF4CFC384351D
:103E0000910509F4D4C38535910509F405C40C94D2
:103E1000CE2E8836910509F45CC24CF484369105A7
:103E200011F00C94CE2E0E942B980C94172F8936EB
:103E3000910509F4DCC28A36910509F46DC30C942E
:103E4000CE2E8037910509F49EC284F48D369105FB
:103E500009F40FC30CF493C28E36910509F43DC2E8
:103E60008F36910509F43DC20C94CE2E8237910510
:103E700009F4F1C30CF48FC28337910509F4F1C33F
:103E80008537910511F40C94172F0C94CE2E8F3298
:103E9000F1E09F0711F40C94B9280CF066C08C3C3B
:103EA000910509F4D1C49CF58B39910509F4BAC286
:103EB00084F48837910509F43AC40CF434C4893782
:103EC000910509F43BC48C38910509F4F0C20C94B7
:103ED000CE2E883C910509F437C434F48E3B91050D
:103EE00009F403C30C94CE2E893C910509F474C4E3
:103EF0008B3C910511F00C94CE2EE1EFEE2EE7E015
:103F0000FE2E0FE512E0F4E0DF2ED00E8EC48D3DC4
:103F1000910509F476C784F48E3C910509F48DC5AA
:103F20000CF40AC5833D910509F47BC68C3D9105CF
:103F300009F458C70C94CE2E8C3231E0930709F463
:103F4000FAC734F4823E910509F4CAC70C94CE2E08
:103F50008D3251E0950711F40C94C4278E329140B4
:103F600011F40C9465280C94CE2E853FB1E09B078C
:103F700011F40C94272E0CF044C08A39F1E09F070D
:103F800009F405C214F5803931E0930711F40C945B
:103F9000782C4CF48336914011F00C94CE2EE9EB42
:103FA000F3E20C94612C8139A1E09A0711F40C948E
:103FB0007B2C8239914011F00C94CE2E80E00E942F
:103FC000B96E0E94DDA30C94172F853AE1E09E079D
:103FD00011F40C94932D3CF4843A914011F40C9418
:103FE000812C0C94CE2E8C3A31E0930709F446C50F
:103FF000843F914011F00C94CE2E0E94078B0C94BC
:10400000172F833553E0950711F40C94682EB4F400
:10401000873FB1E09B0711F40C942D2E14F40C94FF
:104020002A2E883FF1E09F0711F40C94392E8A392B
:10403000924011F40C943C2E0C94CE2E8B3833E02D
:10404000930711F40C94172F4CF48438934011F01B
:104050000C94CE2E0E9483A20C94172F803AA3E0DA
:104060009A0709F421C1873E934011F00C94CE2E9B
:104070000E9470A20C94172FE1E6F2E084918F0168
:104080000F5F1F4F882321F00E941896F801F6CF8A
:104090001092FE0C40E050E0BA0181EB9AE00E94E1
:1040A0009CB98BE1E1EBFAE0DE01159601900D92EF
:1040B0008A95E1F78091AF0A9091B00A9C838B8337
:1040C00089EF92E09A83898340E050E0BE016F5F00
:1040D0007F4F80E090E00E945593CE0101960E94B0
:1040E0005455E2E5F2E084918F010F5F1F4F882362
:1040F00011F40C94172F0E941896F801F4CF109227
:10410000810A1092820A0C94172F0E94B5A70C9472
:10411000172F8091820A882319F081E08093810A09
:104120000E9436490C94172F1092810A0E946F4901
:104130000C94172F8091820A882311F40C94172F66
:1041400083E50E941F9881110C94212F0C94172F46
:1041500083E40E94D897882309F454C0EFE9F2E081
:1041600084918F010F5F1F4F882321F00E941896C2
:10417000F801F6CF80914C0C882391F0BE016F5F5F
:104180007F4F89E49CE00E94BE9B8E010F5F1F4F12
:10419000F80181918F01882381F10E941896F8CF50
:1041A000E2E7F2E084918F010F5F1F4F882329F12E
:1041B0000E941896F801F6CF80910E08882309F422
:1041C000D1C02EEAC22E22E0D22EE12CF12C20E02A
:1041D00080910E0890E00E2C02C0959587950A9468
:1041E000E2F780FDA7C0FFEFEF1AFF0A32E0C30E2F
:1041F000D11C45E0E416F10459F78AE00E941896B4
:104200000C94172F8091820A882371F18091810A82
:10421000882351F1ECE7F2E084918F010F5F1F4F8B
:10422000882321F00E941896F801F6CF6091FA0CCD
:104230007091FB0C8091FC0C9091FD0C4AE00E9467
:1042400022968FE20E9418966091F60C7091F70CFE
:104250008091F80C9091F90C4AE00E9422968AE035
:104260000E9418960C94172FEEE8F2E084918F01CB
:104270000F5F1F4F882311F40C94172F0E9418967C
:10428000F801F4CF40E060E080915F1690916016F5
:104290000E94DBBC0C94172F0E9406A70C94172FCA
:1042A0000E94F9A50C94172F80915F1690916016CB
:1042B00021E02093800A40E060E00E94DBBC0C9487
:1042C000172F0E9436490C94172F0E946F490C94A7
:1042D000172F0E9478A50C94172F0E9468A50C94A4
:1042E000172F83E50E94D897882359F083E50E9411
:1042F0001F98882319F00E94B67301C080E0809354
:104300000E08EEECF3E284918F010F5F1F4F8823BC
:1043100021F00E941896F801F6CFECEBF2E08491C0
:104320008F010F5F1F4F882309F446CF0E94189614
:10433000F801F5CFBB24B394B20E222319F08CE21E
:104340000E941896F60125913491F9018491890112
:104350000F5F1F4F882321F00E9418969801F5CF18
:104360002B2D41CFE8EBF2E084918F010F5F1F4FBF
:10437000882309F442CF0E941896F801F5CF1092D5
:1043800000020C94172F83EC92E00E9477550E9454
:104390000DA30C94172F83E50E941F98882369F0C2
:1043A0000E94B6738D3320F4809323020C94172F50
:1043B0008CE3809323020C94172FEEECF3E28491AC
:1043C0008F010F5F1F4F882321F00E941896F8017C
:1043D000F6CF4091230250E060E070E08CEC92E078
:1043E0000E947DC88AE00E9418960C94172F89E6D7
:1043F00090E00E94CA73811111C0E3EDF2E0849154
:104400008F010F5F1F4F882321F00E941896F8013B
:10441000F6CF0E9420648AE00E94189610928B06C4
:104420000C94C53583E50E941F98882311F40C94E1
:10443000172F0E94B673182F8D3308F01CE31093CA
:1044400098060E9442626B017C01212F30E0A8EEA9
:10445000B3E00E941EDEC60ED71EE81EF91EC092F3
:104460009406D0929506E0929606F09297060C94E8
:10447000172F8DE690E00E94CA7381110C94172FBC
:1044800080910E0883FF02C00C94172F83E50E94D1
:104490001F9861968FAF619781110C94322F82E53E
:1044A0000E941F9881110C94322F0C94172F809129
:1044B0000E0883FF02C00C94172F83E50E941F98FB
:1044C000882311F40C94172F0E94D2950E9472DF5A
:1044D0006E36710514F06EE670E070931F04609301
:1044E0001E040E944E660C94172F80910E0883FFC5
:1044F00002C00C94172F83E50E941F9861968FAF1E
:10450000619781110C94433182E50E941F988111BB
:104510000C9443310C94172F80E50E941F98811151
:1045200006C083E50E941F98882361F006C00E94A0
:10453000B67381110C94172FF4CF0E94C8976F3F68
:10454000710510F06FEF70E070931D0460931C0410
:104550000C94172F80E50E941F98811106C01092BD
:104560001D0410921C040C94172F0E94C897672BEF
:1045700011F00C94172FF3CF0E94E2660E94518431
:1045800010921D0410921C0468EE73E080E090E02D
:104590000E943E690E94DF350C94172F1092FD0394
:1045A0000C94172F81E08093FD030C94172F83E563
:1045B0000E941F988823A1F00E94D29520E030E04D
:1045C0004AE754E40E947CDA0E9477DF6093240279
:1045D0007093250280932602909327020C94172F44
:1045E00088E50E94D89781110C94303389E50E94A8
:1045F000D89781110C9430338AE50E94D8978111A5
:104600000C94303385E40E94D89781110C94303398
:104610000E9451840C94172F83E50E94D897882319
:1046200011F40C94172F0E94D29520E030E04AE755
:1046300054E40E947CDA0E9477DF609390067093C6
:10464000910680939206909393060C94172F0E94E4
:10465000CAA40C94172F0E9441840E94DDA30C94DD
:10466000172FE1ECF4E084918F010F5F1F4F882337
:1046700021F00E941896F801F6CF60E081EB94E0FB
:104680000E9499A361E08AEA94E00E9499A361E004
:104690008FE994E00E9499A361E08FE894E00E9482
:1046A00099A360E086E894E00E9499A361E08CE71A
:1046B00094E00E9499A361E082E794E00E9499A3AC
:1046C00061E08AE694E00E9499A361E08CE594E0C1
:1046D0000E9499A360E08EE494E00E9499A360E0B8
:1046E0008FE394E00E9499A360E081E394E00E944C
:1046F00099A360E08BE194E00E9499A360E08AE0D6
:1047000094E00E9499A360E085EF93E00E9499A352
:1047100061E082EE93E00E9499A30C94172F0E940F
:1047200047A30C94172F0E94AEC70C94172F81E05B
:1047300080934510809346100C94172F10924510CB
:10474000109246100C94172F88EC90E00E94CA73C8
:1047500081110C94172F84E40E94D8978823C1F10B
:104760000E94D29511E020E030E0A9010E9417DA02
:10477000811101C010E010937410112349F10E94BF
:10478000D295E091FF0624E0E29FF0011124E75862
:10479000FF4E608371838283938320E030E0A90120
:1047A0006091791070917A1080917B1090917C10BB
:1047B0000E9417DA81110CC080E090E0A0EEBFE308
:1047C0008093791090937A10A0937B10B0937C1013
:1047D0000E9403C40C94172FA1E9EA2EA0E1FA2E3F
:1047E0000FE512E0B4E0DB2ED00ED8018D918D01E3
:1047F0000E94D897882349F00E94D2950E9477DFC3
:10480000F7016083718382839383F4E0EF0EF11CE0
:10481000D012EBCF0E9428C90C94172FF4E0EF0EB2
:10482000F11CD01611F40C94172FD8018D918D0125
:104830000E94D897882391F30E94D295F701608354
:10484000718382839383EACF83E50E941F98882334
:10485000A1F00E94D2956093E9077093EA078093D4
:10486000EB079093EC076093E5077093E60780935E
:10487000E7079093E80710E001C011E080E50E948F
:104880001F98882359F00E94D2956093E90770938E
:10489000EA078093EB079093EC0710E082E50E9413
:1048A0001F98882359F00E94D2956093ED0770936A
:1048B000EE078093EF079093F00710E084E50E94E5
:1048C0001F98882361F00E94D2956093E50770934A
:1048D000E6078093E7079093E8070C94172F1123BE
:1048E00011F40C94172F4091E9075091EA07609159
:1048F000EB077091EC0784E995E00E949AC840911B
:10490000ED075091EE076091EF077091F00781E994
:1049100095E00E949AC84091E5075091E6076091A2
:10492000E7077091E8078EE895E00E949AC88AE050
:104930000E9418960C94172F82E40E94D89788231F
:1049400051F00E941A7460930108709302088093DA
:1049500003089093040883E50E94D897882351F0B8
:104960000E94D2956093090870930A0880930B08FF
:1049700090930C0884E50E94D897882351F00E94F8
:10498000D29560930508709306088093070890936A
:10499000080888E50E94D897882351F00E94D29594
:1049A0006093D1077093D2078093D3079093D40775
:1049B00089E50E94D897882351F00E94D295609390
:1049C000D5077093D6078093D7079093D8078AE5C9
:1049D0000E94D8978823F1F00E94D2956093D9075E
:1049E0007093DA078093DB079093DC072DEC3CECA7
:1049F0004CEC5DE30E9417DA181664F0E4EAF5E087
:104A000084918F010F5F1F4F882321F00E94189619
:104A1000F801F6CF85E40E94D897882311F40C940E
:104A2000172F0E94D2956093DD077093DE07809365
:104A3000DF079093E0070C94172F6FE5C62E62E016
:104A4000D62E76E4E72E74E0F72E10E0D6018D9195
:104A50006D010E94D897882351F00E94D295F701EA
:104A60006083718382839383812F0E94596F1F5FBC
:104A7000F4E0EF0EF11C133049F72DC90E948FC0EE
:104A800081110C94172F58EC852E5CE1952E2CE0AB
:104A900034E039AF28AFAE014F5F5F4F5A0101E2FA
:104AA0001DE11A0153E0500F5CAFF401659175915F
:104AB00085919491A8ADB9ADCD90DD90ED90FD902C
:104AC000B9AFA8AFA70196010E942DDE2B013C01D2
:104AD00020E030E040EA51EC0E9454E087FD10C035
:104AE00020E030E040EA51E4C301B2010E9417DA4D
:104AF000181634F0F10140825182628273820DC037
:104B0000F80184911816B4F7F7FAF094F7F8F094D6
:104B1000F101C082D182E282F382D101CD90DD9099
:104B2000ED90FD901D0120E030E040EA51ECC7011E
:104B3000B6010E9454E087FF03C0E9EBF3E20BC02B
:104B400020E030E040EA51E4C701B6010E9417DAE4
:104B5000181644F5F2CF84918F010F5F1F4F882301
:104B600021F00E941896F801F6CFE6EDF5E0849169
:104B70008F010F5F1F4F882321F00E941896F801C4
:104B8000F6CF88E290E099A388A388EC90E09DA7F7
:104B90008CA7BE01605E7F4FCE018C960E94B3C38E
:104BA0000C94172FB4E08B0E911C0F5F1F4FECADD0
:104BB000E0137BCF46E4E42E44E0F42E10E0F50150
:104BC00081919191A191B1915F01F70181939193AD
:104BD000A193B1937F01812F0E94596F1F5F133002
:104BE00071F70E94DDA383E992E09DA78CA704E6FC
:104BF00010E019A308A3BE01645D7F4FCE0180962B
:104C00000E94B3C38AEB92E09DA78CA719A308A3C7
:104C1000BE01645D7F4FCE0180960E94B3C30C94A9
:104C2000172FEEECF3E284918F010F5F1F4F882363
:104C300021F00E941896F801F6CF83E50E94D897DC
:104C4000882321F00E940B7480932202ECE1F6E0AD
:104C500084918F010F5F1F4F882321F00E941896C7
:104C6000F801F6CF80912202811103C0E8E1F6E05D
:104C700002C0E4E1F6E084918F010F5F1F4F8823AB
:104C800021F00E941896F801F6CFECE0F6E084914E
:104C90008F010F5F1F4F882321F00E941896F801A3
:104CA000F6CF2091571030915810409159105091E3
:104CB0005A106091A5067091A6068091A706909162
:104CC000A8060E942EDEAB01BC018AE096E00E949D
:104CD0009AC820915B1030915C1040915D1050910A
:104CE0005E106091A9067091AA068091AB06909122
:104CF000AC060E942EDEAB01BC0187E096E00E946C
:104D00009AC820915F1030916010409161105091CD
:104D100062106091AD067091AE068091AF069091E1
:104D2000B0060E942EDEAB01BC0184E096E00E943A
:104D30009AC8ECEFF5E084918F010F5F1F4F882335
:104D400021F00E941896F801F6CF2091571030916B
:104D500058104091591050915A106091280270914A
:104D6000290280912A0290912B020E942EDEAB0133
:104D7000BC018AEF95E00E949AC820915B103091A7
:104D80005C1040915D1050915E1060912C0270910A
:104D90002D0280912E0290912F020E942EDEAB01F7
:104DA000BC0187EF95E00E949AC820915F10309176
:104DB00060104091611050916210609130027091CA
:104DC000310280913202909133020E942EDEAB01BB
:104DD000BC0184EF95E00E949AC88AE00E94189670
:104DE0000C94172F83E50E941F98882311F40C94CC
:104DF000172F0E94C89770930202609301020C94CF
:104E0000172F8DED90E00E94CA7381110C94172F1B
:104E100083E50E941F988823D9F10091FF0610E0D6
:104E20000E94C897000F111FF801EF5AFD4F7183C0
:104E300060838091FF0690E08C01000F111F000F2E
:104E4000111F9801295C3D4F7901880F991FFC01C2
:104E5000EF5AFD4F60817181072E000C880B990B72
:104E60000E941DDA2AE037ED43E25CE30E947CDA1F
:104E7000F801EB58FF4E20813181428153810E941D
:104E80007CDAD7016D937D938D939C931397CFC755
:104E9000EEECF3E284918F010F5F1F4F882321F026
:104EA0000E941896F801F6CF85E40E94189680912A
:104EB000FF06805D0E941896E091FF06F0E0EE0F7D
:104EC000FF1FEF5AFD4F608171818CE296E00E94D6
:104ED000B7C885E20E9418968AE00E941896A7C774
:104EE00080E50E94D897882309F4A1C70E94C8973B
:104EF0006B017C0183E50E941F98882321F00E94AA
:104F0000C8978B0102C00FEF1FEFC80101960397EE
:104F100008F08DC7D7FC8BC79C2DE4E3F6E080E357
:104F20008E0F2491921711F40C94623331968E13E4
:104F3000F8CF0C94653383E50E941F98882319F0FD
:104F40000E94C89702C064E071E079A368A380E57D
:104F50000E941F98882339F00E94C8976938B3E1EE
:104F60007B0730F402C068EE73E07A83698304C083
:104F700088E893E19A838983BE01605E7F4FCE010A
:104F800001960E94B3C353C785E40E941F98811104
:104F900010C080E50E94D897882391F00E94D29596
:104FA00060930006709301068093020690930306B7
:104FB00007C00E94B673882361F3E9EBF3E26EC089
:104FC00089E40E94D897882381F00E94D2952CEA28
:104FD00035EC47E25EE30E947CDA6093FC05709357
:104FE000FD058093FE059093FF0584E40E94D89709
:104FF000882381F00E94D2952CEA35EC47E25EE3EB
:105000000E940ADF609304067093050680930606EB
:1050100090930706EEECF3E284918F010F5F1F4F30
:10502000882321F00E941896F801F6CF40910006DF
:105030005091010660910206709103068CE696E09D
:105040000E949AC82CEA35EC47E25EE36091FC05C9
:105050007091FD058091FE059091FF050E940ADF89
:10506000AB01BC0188E696E00E949AC82CEA35ECB8
:1050700047E25EE3609104067091050680910606A2
:10508000909107060E947CDAAB01BC0184E696E0B1
:105090000E949AC88AE00E941896C9C684918F011E
:1050A0000F5F1F4F882321F00E941896F801F6CF5A
:1050B000E0E7F6E084918F010F5F1F4F882309F42A
:1050C000B6C60E941896F801F5CF83E50E94D897DE
:1050D000182F882371F00E94D2950E9472DF70937E
:1050E0003C0260933B0221E0672B09F020E0209313
:1050F0000D0880E50E94D897882359F020913B0243
:1051000030913C02232B11F00E940B7480930D0808
:105110008EC611118CC6EEECF3E284918F010F5F05
:105120001F4F882321F00E941896F801F6CF809136
:105130000D08811103C06FE173E002C06BED73E0F5
:1051400087E996E00E94D0C860913B0270913C02D2
:1051500086E896E00E94B7C8E2E8F6E084918F0105
:105160000F5F1F4F882309F462C60E941896F8014A
:10517000F5CF85E40E941F98882321F00E94C897EC
:105180007B0102C0E12CF12C83E40E941F9888234C
:1051900031F00E94C897EA966FAFEA9704C025E005
:1051A000EA962FAFEA9785E50E941F98882319F0A9
:1051B0000E940B7403C085E50E94D897CB57DF4F40
:1051C0008883C558D040F7FC07C0812C912CB6E1EC
:1051D000AB2EB3E4BB2E06C0812C912CACE8AA2EDA
:1051E000A2E4BA2E83E50E941F98882321F00E9432
:1051F000D2954B015C01E114F10411F41092FF0609
:1052000010928B060E9442622B013C01DC01CB0113
:105210008C53964FAF4FBF4F8093F5069093F60691
:10522000A093F706B093F806EE2069F0E9E1F8E004
:1052300084918F010F5F1F4F882309F4F8C50E94E6
:105240001896F801F5CFE3E4F8E084917F013FEF91
:10525000E31AF30A882321F00E941896F701F5CF8C
:10526000C501B4010E9472DF072E000C880B990B58
:105270000E941DDA25966FAF259721967FAF219763
:1052800029968FAF29972D969FAF2D97D301C201F5
:10529000805E914BAF4FBF4FC257DF4F88839983DA
:1052A000AA83BB83CE58D0400E94E2668FE78093EA
:1052B000FD0681E080930002C358DF4F4882598287
:1052C0006A827B82CD57D040CA57DF4F48825982CD
:1052D0006A827B82C658D040ED961FAEED97C657C6
:1052E000DF4F188219821A821B82CA58D040A196B9
:1052F0001FAEA19790E465969FAF6597ACE1699664
:10530000AFAF6997B6E4A596BFAFA5976D961FAEF0
:105310006D97A9961FAEA997AD961FAEAD97E19672
:105320001FAEE197E9961CAE1DAE1EAE1FAEE9970B
:10533000E5961CAE1DAE1EAE1FAEE597C12CD12C5E
:1053400076012FE730E040E050E02CAF3DAF4EAFAC
:105350005FAF8FE790E0A0E0B0E088AF99AFAAAF71
:10536000BBAFCF57DF4F188219821A821B82C158F8
:10537000D04091E0EC969FAFEC9762961FAE1EAEC8
:10538000629710E0212C312C00E0EA96AFADEA974D
:105390000A2E000CBB0BEB96BFAFAEAFEB97809124
:1053A0000002882309F435C10E9442624B015C016E
:1053B0008091FA06882309F408C10E94A26710911F
:1053C0002604209027043090280400912904212FDE
:1053D000322D432D502F6D966FAD6D97A9967FADF1
:1053E000A997AD968FADAD97E1969FADE1970E94DD
:1053F00017DA87FF0CC06D961FAF6D97A9962FAE79
:10540000A997AD963FAEAD97E1960FAFE197212FEB
:10541000322D432D502FA1966FADA19765967FAD8C
:10542000659769968FAD6997A5969FADA5970E94E0
:1054300054E0181664F4A1961FAFA19765962FAE9D
:10544000659769963FAE6997A5960FAFA59780912E
:10545000F5069091F606A091F706B091F806A50121
:105460009401281B390B4A0B5B0B57FD10C00E949F
:105470009748D501C4018C53964FAF4FBF4F8093CF
:10548000F5069093F606A093F706B093F806EC960F
:105490003FADEC9725962FAD2597332309F46CC0CB
:1054A00021963FAD219729964FAD29972D965FAD57
:1054B0002D97612F722D832D902F0E9454E0181686
:1054C0000CF083C0D501C40184199509A609B70958
:1054D000CE56DF4F88839983AA83BB83C259D040BD
:1054E00088589341A109B109B7FD6FC088AD99AD46
:1054F000AAADBBAD2CAD3DAD4EAD5FAD821B930BE8
:10550000A40BB50BB595A795979587958093FD0648
:10551000CE56DF4F88819981AA81BB81C259D04084
:10552000CF57DF4F88839983AA83BB83C158D0406C
:1055300025969FAD25976D969FAF6D972196AFAD40
:105540002197A996AFAFA9972996BFAD2997AD9698
:10555000BFAFAD972D96EFAD2D97E196EFAFE197E9
:10556000C358DF4F88829982AA82BB82CD57D04030
:10557000EC961FAEEC9729C021963FAD2197299656
:105580004FAD29972D965FAD2D97612F722D832DED
:10559000902F0E9417DA87FF18C0D501C401C358A5
:1055A000DF4F288139814A815B81CD57D040821BF2
:1055B000930BA40BB50BAC01BD01485853416109D5
:1055C000710977FD02C00C948D3320E030E040EA91
:1055D00051E425966FAD259721967FAD21972996A9
:1055E0008FAD29972D969FAD2D970E942EDE9B01A2
:1055F000AC01612F722D832D902F0E9454E018165C
:105600007CF4E5EAF7E084918F010F5F1F4F811171
:1056100003C00E94E2660BC40E941896F801F3CF03
:10562000D501C401CA57DF4F288139814A815B8186
:10563000C658D040821B930BA40BB50BB7FDA5C079
:105640000E9420648AE00E941896D501C40180530C
:10565000984FAF4FBF4FCA57DF4F88839983AA83B4
:10566000BB83C658D040ED969FADED9791116AC0AF
:10567000C657DF4F288139814A815B81CA58D040A3
:10568000612F722D832D902F0E9454E018160CF07C
:1056900044C020E030E040E050E4612F722D832DC3
:1056A000902F0E942EDEC657DF4F688379838A834E
:1056B0009B83CA58D040A5019401205E314B4F4FC7
:1056C0005F4FC257DF4F288339834A835B83CE58AD
:1056D000D04020E030E040EC50E425966FAD2597B7
:1056E00021967FAD219729968FAD29972D969FAD55
:1056F0002D970E942DDE9B01AC0181E0ED968FAFCE
:10570000ED97612F722D832D902F0E9454E0181673
:10571000E4F1ED961FAEED9738C0D501C401C25734
:10572000DF4F288139814A815B81CE58D040821B6E
:10573000930BA40BB50BB7FD28C044E857E066E90E
:1057400077E020C020E030E040EA51E425966FADDC
:10575000259721967FAD219729968FAD29972D9674
:105760009FAD2D970E942DDE9B01AC01612F722D04
:10577000832D902F0E9417DA87FF07C041E657E07C
:1057800064E777E080E00E942A48D501C401880FD1
:10579000991FAA1FBB1FC358DF4F288139814A8137
:1057A0005B81CD57D040821B930BA40BB50B8419A2
:1057B0009509A609B70981389F44A241B10568F04F
:1057C000E3E4F7E084918F010F5F1F4F882309F412
:1057D00020CF0E941896F801F5CF62964EAD5FADCE
:1057E0006297EB968EAD9FADEB97841795070CF003
:1057F000D6CDE6EEF6E084918F010F5F1F4F882330
:1058000021F00E941896F801F6CFB701A60182EDAB
:1058100096E00E949AC88AE00E941896E5964CADE0
:105820005DAD6EAD7FADE5978EEB96E00E949AC8B8
:105830008AE00E941896E9964CAD5DAD6EAD7FADE5
:10584000E9978AEA96E00E949AC88AE00E94189630
:10585000CB57DF4F9881C558D040992309F4E7C250
:10586000C0920006D0920106E0920206F092030672
:105870002CEA35EC47E25EE3E5966CAD7DAD8EAD8E
:105880009FADE5970E947CDA6093FC057093FD055F
:105890008093FE059093FF052CEA35EC47E25EE32A
:1058A000E9966CAD7DAD8EAD9FADE9970E940ADFA4
:1058B000609304067093050680930606909307068E
:1058C000B6C284918F010F5F1F4F882321F00E9481
:1058D0001896F801F6CFE7E5F8E084918F010F5FA5
:1058E0001F4F882309F4A3C20E941896F801F5CF30
:1058F0000E9441849CC281E00E94B96E0E94DDA397
:1059000096C283E50E94D897882349F00E940B74C1
:10591000082F811106C080E00E94EB7202C0009146
:105920006C1080910C0490910D04A0910E04B09124
:105930000F0489839A83AB83BC8380911004909178
:105940001104A0911204B09113048D839E83AF8340
:10595000B8878091140490911504A0911604B09119
:10596000170489879A87AB87BC8780911010909124
:105970001110892BC1F183E40E94D89781110C94F6
:105980001D3531C0930121964FAD219729965FAD0A
:105990002997682D7D2D8CAD25969FAD25970E946A
:1059A0002EDE20E030E040E05FE30E947CDAA201DE
:1059B00091010E942EDE4B015C012DEB37E346E89E
:1059C00055EB0E9454E087FF02C00C9480352DEB0C
:1059D00037E346E855E3C501B4010E9417DA18160B
:1059E00014F40C94803586E50E94D897882341F002
:1059F0008091101090911110892B11F00E94BBAA78
:105A00008AE50E94D897882321F00E94D2950E94AF
:105A1000FABF802F0E94EB72011103C0EEECF3E29B
:105A20001CC080916C108111F9CFE9EBF3E28491F5
:105A30008F010F5F1F4F882321F00E941896F801F5
:105A4000F6CFE6E8F8E084918F010F5F1F4F8823BF
:105A500029F30E941896F801F6CF84918F010F5F09
:105A60001F4F882321F00E941896F801F6CF8091ED
:105A70006C10811103C067E273E002C063E273E05F
:105A800088E798E00E94D0C88AE00E941896EEEC61
:105A9000F3E284918F010F5F1F4F882321F00E9452
:105AA0001896F801F6CFEBE6F8E084918F010F5FCE
:105AB0001F4F882321F00E941896F801F6CFC0905E
:105AC0006D10D0906E10E0906F10F090701020E08C
:105AD00030E0A901C701B6010E9454E018164CF449
:105AE00042E0C701B6010E94A2968AE00E94189681
:105AF0000CC0E6E6F8E084918F010F5F1F4F88230A
:105B000021F00E941896F801F6CF4CE050E06CE0CE
:105B100074E0CE0101960E944DE1892B09F487C102
:105B20000E94DDA384C189E40E941F98882321F08C
:105B30000E94C897062F01C00FEF8AE40E941F98A9
:105B4000882321F00E94C897162F01C01FEF8AE515
:105B50000E94D897F82E811105C081E50E94D89740
:105B6000D82E01C0D12C07FD02C017FF03C0E9EBFE
:105B7000F3E205C0F1101AC0D11018C0F8CF84911B
:105B80008F010F5F1F4F882321F00E941896F801A4
:105B9000F6CFE4ECF8E084918F010F5F1F4F88236C
:105BA00009F445C10E941896F801F5CF033018F0AA
:105BB000E9EBF3E206C01330D8F716C00E9418963E
:105BC000F80184918F010F5F1F4F8111F7CFE5EA34
:105BD000F8E084918F010F5F1F4F882309F427C1DC
:105BE0000E941896F801F5CFE02E000FFF08012F54
:105BF000110F110B0E94D295D701AA0FBB1FDD20F8
:105C000081F0FD01EE0DFF1DE00FF11FEE0FFF1FF4
:105C1000EE0FFF1FE85EFF4E2081318142815381EC
:105C200003C020E030E0A901EA0EFB1E0E0D1F1D8F
:105C3000000F111F000F111F085E1F4E0E942EDE65
:105C4000D8016D937D938D939C931397F0C00E9420
:105C500089B5EDC00E947BB4EAC083E50E94D89765
:105C6000882321F00E940B7491E089270E94DDAF08
:105C7000DEC00E94E9A2DBC08AE50E941F9888234B
:105C800059F00E94D2956093141070931510809370
:105C9000161090931710CBC0E7EEF8E084918F01B7
:105CA0000F5F1F4F882321F00E941896F801F6CF4E
:105CB00040911410509115106091161070911710AA
:105CC00084EE98E00E949AC88AE00E941896AFC0BD
:105CD0008AE50E941F98882309F438C00E94D29553
:105CE0006B017C0120E030E040EA51EC0E9454E07E
:105CF00087FD13C020E030E040EA51E4C701B6015F
:105D00000E9417DA18164CF0C0920704D0920804CB
:105D1000E0920904F0920A048AC0E9EBF3E284916C
:105D20008F010F5F1F4F81110DC0E8E1F9E08491F1
:105D30008F010F5F1F4F882309F479C00E941896C6
:105D4000F801F5CF0E941896F801E9CFEEECF3E2E6
:105D500084918F010F5F1F4F882321F00E941896B6
:105D6000F801F6CFE9E0F9E084918F010F5F1F4F52
:105D7000882321F00E941896F801F6CF409107047D
:105D8000509108046091090470910A0486E099E03A
:105D90000E949AC88AE00E94189649C00E94E7C3F0
:105DA00046C0F09061160E944184FF2029F1EEEC7C
:105DB000F3E284918F010F5F1F4F882321F00E942F
:105DC0001896F801F6CF84E50E9418966F2D70E0C2
:105DD00080E090E04AE00E94229680E20E941896BD
:105DE000E7E4F9E084918F010F5F1F4F8823F9F0FA
:105DF0000E941896F801F6CF10928A06EEECF3E2B4
:105E000084918F010F5F1F4F882321F00E94189605
:105E1000F801F6CF60918A0670E085E399E00E9470
:105E2000B7C88AE00E94189602C00E94E7C3109289
:105E30008B060E941ACBA9C60E94FBA80E948F590C
:105E4000F6CF0E94C897AB01BC014093FA0C509367
:105E5000FB0C6093FC0C7093FD0C89E49CE00E94A9
:105E60009CB9E5CF0E94D2950E9472DF7093250401
:105E70006093240480E00E9498660E94D29520E0FE
:105E800030E044EB52E40E9417DA18161CF00E942E
:105E9000844902C00E943649E2E0F3E084918F0118
:105EA000882351F0082E000C990B0E941A910F5F65
:105EB0001F4FF8018491F4CF8DE090E00E941A9179
:105EC0008AE090E00E941A91E6EDF2E084918F0161
:105ED0000F5F1F4F882321F00E941896F801F6CF1C
:105EE0000E94F8C881E08093000210928B061CAEDD
:105EF0001DAE1EAE1FAEA4961CAE1DAE1EAE1FAED6
:105F0000A49718AE65961FAE6597FCE36996FFAF40
:105F100069972CE1A5962FAFA59736E46D963FAF14
:105F20006D97C12CD12C80E8E82E9FEBF92E812CA7
:105F3000912C54016091240470912504072E000CCB
:105F4000880B990B0E941DDA162F072F782E692EC9
:105F5000262F372F482F592FB601C7010E9417DA75
:105F6000882301F1209126043091270440912804D0
:105F700050912904612F702F872D962D0E9417DADA
:105F8000881F8827881F88AF61964FAD619744238B
:105F900069F0882359F080910002E7E7F3E08491EB
:105FA0008F0127C11C2D0D2D7E2C6F2C0E9442626B
:105FB0006B017C01DC01CB01A4962CAD3DAD4EAD57
:105FC0005FADA497821B930BA40BB50BB7FD3DC02F
:105FD000D701C60188519C4FAF4FBF4FA4968CAFDD
:105FE0009DAFAEAFBFAFA4970E942064EBE7F3E094
:105FF00084912F019FEF491A590A882321F00E94AA
:106000001896F201F5CF81149104A104B104B9F0FE
:10601000D501C401805F984DAF4FBF4FBC01CD018A
:106020006C197D098E099F0928EE33E040E050E0AD
:106030000E94F2DDCA01B9010E94889603C08FE375
:106040000E9418968AE00E9418960E94C9550E94E4
:10605000426260938C0670938D0680938E069093B7
:106060008F06A09126042596AFAF2597B0912704FF
:106070002196BFAF2197E09128042996EFAF299789
:10608000F09129042D96FFAF2D9799D525962FAD28
:10609000259721963FAD219729964FAD29972D96AB
:1060A0005FAD2D97612F702F872D962D0E942DDECD
:1060B0001B012C0120E030E0A9010E9454E087FF81
:1060C00004C057FA509457F8509481149104A104D5
:1060D000B10459F420E030E040E85FE3C201B101CF
:1060E0000E9417DA87FF0DC00AC020E030E040E4CC
:1060F00050E4C201B1010E9454E0181614F44601A4
:10610000570128AD222309F458C08CAD9DADAEAD2A
:10611000BFAD892B8A2B8B2B61F0D701C6012CAD2B
:106120003DAD4EAD5FAD821B930BA40BB50BB7FD20
:1061300044C025962FAD259721963FAD21972996EE
:106140004FAD29972D965FAD2D9765966FAD6597ED
:1061500069967FAD6997A5968FADA5976D969FAD12
:106160006D970E942DDE20E030E040EC5FE30E945E
:1061700017DA87FD10CFD701C601805A9541AF4F7E
:10618000BF4F8CAF9DAFAEAFBFAF25969FAD2597EC
:1061900065969FAF65972196AFAD21976996AFAF92
:1061A00069972996BFAD2997A596BFAFA5972D965C
:1061B000EFAD2D976D96EFAF6D978091000288231C
:1061C00009F4E9CE81149104A104B10429F4C12E8B
:1061D000D02EE72CF62CAECEF0E1CF1AF7E2DF0A94
:1061E000E108F108C818D908EA08FB08F7FED3CE81
:1061F000EECF882351F0082E000C990B0E941A91C3
:106200000F5F1F4FF8018491F4CF8DE090E00E9462
:106210001A918AE090E00E941A91E6E4F3E08491FA
:106220008F010F5F1F4F882321F00E941896F801FD
:10623000F6CF80918E0E813009F0F9CDE2E4F3E0E3
:1062400084918F01882351F0082E000C990B0E9435
:106250001A910F5F1F4FF8018491F4CF8DE090E009
:106260000E941A918AE090E00E941A91E6E0F3E021
:1062700084918F010F5F1F4F882309F4D8CD0E94AE
:106280001896F801F5CF0E94D2950E9472DF6E3603
:1062900071050CF0E2C170931F0460931E040E940C
:1062A0004E660E94D29520E030E040EA50E40E9421
:1062B00054E0181614F40E943649E8EAF3E0849199
:1062C0008F01882351F0082E000C990B0E941A911F
:1062D0000F5F1F4FF8018491F4CF8DE090E00E9492
:1062E0001A918AE090E00E941A91EFE7F3E084911E
:1062F0008F010F5F1F4F882321F00E941896F8012D
:10630000F6CF81E08093000210928B0680918A067E
:106310008093FF061CAE1DAE1EAE1FAEA4961CAE33
:106320001DAE1EAE1FAEA49718AE65961FAE659744
:10633000FCE36996FFAF69972CE1A5962FAFA5976F
:1063400036E46D963FAF6D97C12CD12C10E8E12E4D
:106350000FEBF02E812C912C540160911E04709152
:106360001F04072E000C880B990B0E941DDA162FB4
:10637000072F782E692E262F372F482F592FB60139
:10638000C7010E9417DA8823F1F020912004309190
:1063900021044091220450912304612F702F872DF6
:1063A000962D0E9417DA881F8827881F88AF61966C
:1063B0004FAD6197442359F0882349F0EAEDF3E0AB
:1063C00084918F0127C11C2D0D2D7E2C6F2C0E94D6
:1063D00042626B017C01DC01CB01A4962CAD3DAD8A
:1063E0004EAD5FADA497821B930BA40BB50BB7FD0D
:1063F0003DC0D701C60188519C4FAF4FBF4FA496F7
:106400008CAF9DAFAEAFBFAFA4970E942064EEEDFE
:10641000F3E084912F019FEF491A590A882321F054
:106420000E941896F201F5CF81149104A104B104E1
:10643000B9F0D501C401805F984DAF4FBF4FBC018B
:10644000CD016C197D098E099F0928EE33E040E0EB
:1064500050E00E94F2DDCA01B9010E94889603C093
:106460008FE30E9418968AE00E9418960E94C955F0
:106470000E94426260938C0670938D0680938E0614
:1064800090938F06A09120042596AFAF2597B091E9
:1064900021042196BFAF2197E09122042996EFAF06
:1064A0002997F09123042D96FFAF2D9788D3259639
:1064B0002FAD259721963FAD219729964FAD29976E
:1064C0002D965FAD2D97612F702F872D962D0E94F1
:1064D0002DDE1B012C0120E030E0A9010E9454E0D8
:1064E00087FF04C057FA509457F8509481149104D0
:1064F000A104B10459F420E030E040E85FE3C201B8
:10650000B1010E9417DA87FF0DC00AC020E030E019
:1065100040E450E4C201B1010E9454E0181614F4A2
:106520004601570128AD222309F458C08CAD9DAD1A
:10653000AEADBFAD892B8A2B8B2B61F0D701C60185
:106540002CAD3DAD4EAD5FAD821B930BA40BB50BD7
:10655000B7FD44C025962FAD259721963FAD2197D5
:1065600029964FAD29972D965FAD2D9765966FAD06
:10657000659769967FAD6997A5968FADA5976D963E
:106580009FAD6D970E942DDE20E030E040EC5FE390
:106590000E9417DA87FD12CFD701C601805A9541B4
:1065A000AF4FBF4F8CAF9DAFAEAFBFAF25969FAD86
:1065B000259765969FAF65972196AFAD2197699610
:1065C000AFAF69972996BFAD2997A596BFAFA5979D
:1065D0002D96EFAD2D976D96EFAF6D9780910002E0
:1065E000882309F4EBCE81149104A104B10429F4A9
:1065F000C12ED02EE72CF62CB0CEF0E1CF1AF7E268
:10660000DF0AE108F108C818D908EA08FB08F7FE14
:10661000D5CEEECF882351F0082E000C990B0E94A6
:106620001A910F5F1F4FF8018491F4CF8DE090E035
:106630000E941A918AE090E00E941A91ECEAF3E03D
:1066400084918F010F5F1F4F882321F00E941896BD
:10665000F801F6CF80910002EACB6EE670E01BCE27
:106660000E94418488E50E94D897882331F05F9A80
:1066700080910B048E7F80930B0489E50E94D8974C
:10668000882339F08A9A479A80910B048D7F8093F2
:106690000B048AE50E94D897882361F08091080155
:1066A0008095817080930601479A80910B048B7FBF
:1066B00080930B0485E40E94D897882309F4B7CB14
:1066C000129AB5CB0E94A1A5B2CB0E944184BC2CEA
:1066D00060E08C2D0E94BE600F3FFFEF1F0759F452
:1066E0008C2D0E94676031E020E0892B09F030E0BA
:1066F000032F122F05C00130110561F000E010E0FA
:106700008B2D0E9467608017910709F490CB0E943F
:10671000C955F6CF01E010E0F3CF62964EAD5FAD04
:106720006297452B09F44DC1CF57DF4F4880598000
:106730006A807B80C158D040480E591E6A1E7B1E5D
:10674000CF57DF4F288139814A815B81C158D040C2
:10675000281B390B4A0B5B0BCA01B9012CAD3DADAF
:106760004EAD5FAD0E94E3DDA30192010E941DE1E9
:1067700088AD99ADAAADBBAD820F931FA41FB51F05
:1067800084319105A105B1051CF188AF99AFAAAF7D
:10679000BBAF8C3E9105A105B10544F08BEE90E0B6
:1067A000A0E0B0E088AF99AFAAAFBBAF28AD39ADDC
:1067B0004AAD5BAD2038310541055105D4F08EEF6F
:1067C00090E0A0E0B0E0821B930BA40BB50B0CC0D3
:1067D00024E130E040E050E028AF39AF4AAF5BAF92
:1067E00084E190E0A0E0B0E08CAF9DAFAEAFBFAF72
:1067F00008C028AD39AD4AAD5BAD2CAF3DAF4EAF53
:106800005FAF48AD59AD6AAD7BAD81E198E00E94C4
:10681000B6D54CAD5DAD6EAD7FAD8CE098E00E941D
:10682000B6D5A1964FADA19765965FAD6597699670
:106830006FAD6997A5967FADA59785E098E00E941A
:106840009AC86D964FAD6D97A9965FADA997AD9615
:106850006FADAD97E1967FADE1978EEF97E00E9427
:106860009AC862964EAD5FAD6297433051050CF405
:10687000A8C06CAD7DAD8EAD9FAD0E941DDA20E04D
:1068800030E040E850E40E947CDA6B017C01A19684
:106890002FADA19765963FAD659769964FAD699706
:1068A000A5965FADA5976D966FAD6D97A9967FADD7
:1068B000A997AD968FADAD97E1969FADE1970E94F8
:1068C0002DDE2BED3FE049E450E40E947CDA20E02D
:1068D00030E040E05FE30E947CDA9B01AC01C7013D
:1068E000B6010E940ADF6B017C01C301B2010E9464
:1068F0001DDA2FE632E143E85AE30E947CDA2B01ED
:106900003C01B701A60188EF97E00E949AC8B30145
:10691000A20182EF97E00E949AC82AE939E949E189
:106920005FE3C701B6010E947CDA6B017C019B0129
:10693000AC010E942EDEA30192010E940ADFE596BF
:106940006CAF7DAF8EAF9FAFE597A3019201C701FA
:10695000B6010E947CDA20E030E040E05EE30E9475
:106960007CDAE9966CAF7DAF8EAF9FAFE997E2EE30
:10697000F7E084913F015FEF651A750A882321F0E3
:106980000E941896F301F5CFB701A6018CED97E0B0
:106990000E949AC8E5964CAD5DAD6EAD7FADE597B2
:1069A00086ED97E00E949AC8E9964CAD5DAD6EAD5C
:1069B0007FADE99780ED97E00E949AC88AE00E9437
:1069C000189688AD99ADAAADBBAD2CAD3DAD4EAD21
:1069D0005FAD820F931FA41FB51FB595A79597951F
:1069E00087958093FD0662964EAD5FAD62974F5FCF
:1069F0005F4F62965FAF4EAF629725965FAD25976A
:106A0000A1965FAFA19721968FAD219765968FAF25
:106A1000659729969FAD299769969FAF69972D969F
:106A2000AFAD2D97A596AFAFA59724013501B1E085
:106A3000EC96BFAFEC970C94E52A0E94D2951B010F
:106A40002C0113E0612C712C28EC21962FAF21979B
:106A500032EC29963FAF2997812CD12C48EC4CAFD2
:106A600052E425965FAF2597115010F40C94C22C78
:106A7000E3E0E8AF812F90E07C01EE0CFF1CE80E14
:106A8000F91EB8ADB150B8AFBF3F71F3F701A8AD73
:106A9000EA0FF11DEE0FFF1FEE0FFF1FE85EFF4E26
:106AA0009080A180B280C380292D3A2D4B2D5C2D82
:106AB000682D7D2D8CAD25969FAD25970E9454E0C5
:106AC000181634F4892CDA2CBCAE2596CFAE259757
:106AD000292D3A2D4B2D5C2DB30121968FAD219799
:106AE00029969FAD29970E9417DA87FFCACF692C94
:106AF0007A2C2196BFAE21972996CFAE2997C1CF88
:106B000080E00E94EB7213E04CE0D42E1150D19E35
:106B1000C00111249C01285E3F4E7901A50194011A
:106B2000D70118966D917D918D919C911B970E9434
:106B30002DDEF7016087718782879387A501940115
:106B400064817581868197810E942DDED70114961C
:106B50006D937D938D939C931797A50194016D91EF
:106B60007D918D919C910E942DDEF7016083718350
:106B7000828393831111CACF0C94F32C01110C94CE
:106B8000EB1C0E940E960C94FF1CCB56DF4F0FB6E9
:106B9000F894DEBF0FBECDBFDF91CF911F910F9153
:106BA000FF90EF90DF90CF90BF90AF909F908F902D
:106BB0007F906F905F904F903F902F9008952F920D
:106BC0003F924F925F926F927F928F929F92AF927D
:106BD000BF92CF92DF92EF92FF920F931F93CF93CA
:106BE000DF93CDB7DEB76F970FB6F894DEBF0FBE59
:106BF000CDBFC0902604D0902704E0902804F090E8
:106C0000290420E030E040EA50E4C701B6010E94C8
:106C100017DA87FD24C120E030E041E953E4C701E1
:106C2000B6010E9454E018160CF419C110929D0E82
:106C300010929C0E8091090140919B0E042E000C35
:106C4000550B817021E0822790E04817590709F41D
:106C500052C0809109018170822780939B0E882306
:106C600031F10E946891E7EDF0E184918F01882372
:106C700051F0082E000C990B0E941A910F5F1F4FC4
:106C8000F8018491F4CF8DE090E00E941A918AE09F
:106C900090E00E941A91ECEAF0E184918F010F5F7D
:106CA0001F4F882341F10E941896F801F6CFE5E0C6
:106CB000F1E184918F01882351F0082E000C990B8B
:106CC0000E941A910F5F1F4FF8018491F4CF8DE05D
:106CD00090E00E941A918AE090E00E941A91EBEDF8
:106CE000F0E184918F010F5F1F4F882321F00E94F4
:106CF0001896F801F6CF80918E0E833009F457C0B4
:106D00002CF4882351F08130D9F073C0843009F419
:106D100049C0853009F458C06CC08091810A88232D
:106D200009F467C081E080938E0E0E9442626093F6
:106D3000920E7093930E8093940E9093950E59C07B
:106D40008091810A811155C080914C0C882321F0DB
:106D500082E080938E0E4DC010928E0EE8EAF0E134
:106D600084918F01882351F0082E000C990B0E940A
:106D70001A910F5F1F4FF8018491F4CF8DE090E0DE
:106D80000E941A918AE090E00E941A91E0E8F0E1F6
:106D900084918F010F5F1F4F882359F10E9418962D
:106DA000F801F6CF8091DB0E882391F222C080910A
:106DB000810A81111EC080912B0A90912C0A891B97
:106DC0008F7009F483C015C08091810A811111C0B0
:106DD00080912B0A90912C0A891B8F7009F4ACC00A
:106DE00008C086E090E190931C0880931B080E94E5
:106DF000C16F8091830E9091840E0397E4F080918F
:106E0000830E9091840E009711F40C941A4601970A
:106E10009093840E8093830E8091850E9091860EC0
:106E2000019664E070E00E940AE19093860E8093E0
:106E3000850E0C941A468AE0C82ED12CE12CF12C38
:106E400089EE9FE00E94BA9518161906C4F6809143
:106E5000830E9091840E04970CF495C0D0CF80914E
:106E60009C0E90919D0E8136FAEE9F0748F110928C
:106E70009D0E10929C0EEFE3F1E184918F01882327
:106E800051F0082E000C990B0E941A910F5F1F4FB2
:106E9000F8018491F4CF8DE090E00E941A918AE08D
:106EA00090E00E941A91E9E0F1E184918F010F5F77
:106EB0001F4F882309F4BECE0E941896F801F5CF23
:106EC000019690939D0E80939C0EB4CE8CE690E13B
:106ED00090931C0880931B080E94C16F8091DB0E69
:106EE000882311F082E001C084E080938E0EE8E6F2
:106EF000F0E184918F01882351F0082E000C990B4A
:106F00000E941A910F5F1F4FF8018491F4CF8DE01A
:106F100090E00E941A918AE090E00E941A91E9E3C1
:106F2000F0E184918F010F5F1F4F882309F461CF37
:106F30000E941896F801F5CFE5E3F0E184918F0106
:106F4000882351F0082E000C990B0E941A910F5FB4
:106F50001F4FF8018491F4CF8DE090E00E941A91C8
:106F60008AE090E00E941A9110928E0EEAE0F0E121
:106F700084918F010F5F1F4F882309F432CF0E9445
:106F80001896F801F5CF89EE9FE00E947E958093D8
:106F9000890E20918A0E30918B0E8A3049F08D3007
:106FA00039F08A3329F02F35310514F40C9444421A
:106FB0002115310509F423CF8091870E9091880E19
:106FC000A0E6BA2EB89E8001B99E100D1124200FA4
:106FD000311FF901ED5FF24F108298012D5F324FA2
:106FE000390161E470E0C9010E9488E1009711F461
:106FF0000C94284290938D0E80938C0E86199709DD
:10700000800F911F60E070E08C5F924F0E94DDD591
:107010000E9472DF2B013C0168307105B4F06431CD
:10702000710509F491C68091870E9091880EB89EE3
:10703000B001B99E700D11246D5F724F81EF9FE01A
:107040000E94D0C88AE00E941896052C000C6608A1
:10705000770832E24316510410F00C942842F201F2
:107060008827EE58FF4F8F4F0C9439E1ECEEFFE08C
:1070700084918F01882351F0082E000C990B0E94F7
:107080001A910F5F1F4FF8018491F4CF20E030E098
:1070900040E05FE36091260470912704809128040A
:1070A000909129041EC0E7EEFFE084918F018823B0
:1070B00051F0082E000C990B0E941A910F5F1F4F80
:1070C000F8018491F4CF6091240470912504072E77
:1070D000000C880B990B0E941DDA20E030E040E0A4
:1070E0005FE30E942EDE0E9472DFCB010E949D9A18
:1070F0000E94DBBE8DE090E00E941A918AE090E051
:107100000E941A910C942842E2EEFFE084918F01D4
:10711000882351F0082E000C990B0E941A910F5FE2
:107120001F4FF8018491F4CF20E030E040E05FE3AE
:107130006091200470912104809122049091230495
:10714000D0CFEDEDFFE084918F01882351F0082E20
:10715000000C990B0E941A910F5F1F4FF801849148
:10716000F4CF60911E0470911F04B1CF20911C04D4
:1071700030911D0444E6429FC001439F900D1124AD
:107180006FEF70E00E940AE15B016536710518F04F
:10719000F4E6AF2EB12CE8EDFFE084918F01882357
:1071A00051F0082E000C990B0E941A910F5F1F4F8F
:1071B000F8018491F4CFB50180E090E011C6E4EDD0
:1071C000FFE084918F01882351F0082E000C990B69
:1071D0000E941A910F5F1F4FF8018491F4CF80E253
:1071E00090E00E941A91E0EDFFE084918F018823E6
:1071F00051F0082E000C990B0E941A910F5F1F4F3F
:10720000F8018491F4CF60910C0470910D04809189
:107210000E0490910F040E9427BF80E290E00E942C
:107220001A91ECECFFE084918F01882351F0082E35
:10723000000C990B0E941A910F5F1F4FF801849167
:10724000F4CF609110047091110480911204909118
:1072500013040E9427BF80E290E00E941A91E8EC9C
:10726000FFE084918F01882351F0082E000C990BC8
:107270000E941A910F5F1F4FF8018491F4CF609123
:1072800014047091150480911604909117040E94C3
:1072900027BF80E290E00E941A912CCF8091810A52
:1072A000882309F450C0E3ECFFE084918F01882328
:1072B00051F0082E000C990B0E941A910F5F1F4F7E
:1072C000F8018491F4CF8091820A882359F180914A
:1072D0004C0C882329F18091F60C9091F70CA09129
:1072E000F80CB091F90C0097A105B105C1F0BC01F3
:1072F000CD016D597F4F8F4F9F4F24E630E040E026
:1073000050E00E94F2DD6091FA0C7091FB0C8091CC
:10731000FC0C9091FD0C0E94F2DD822F01C080E0F8
:1073200090E0E4CEEFEBFFE084918F01882309F435
:10733000E1CE082E000C990B0E941A910F5F1F4F8F
:10734000F8018491F3CFE7EBFFE084918F0188236C
:1073500009F4D0CE082E000C990B0E941A910F5FF1
:107360001F4FF8018491F3CFE2EBFFE084918F018E
:10737000882351F0082E000C990B0E941A910F5F80
:107380001F4FF8018491F4CF8091920E9091930E4B
:10739000A091940EB091950E892B8A2B8B2B09F41A
:1073A0007FC00E94426220E63AEE40E050E00E9438
:1073B000F2DD29013A016091920E7091930E809155
:1073C000940E9091950E20E63AEE40E050E00E9437
:1073D000F2DD421A530AC2016CE370E00E94F6E04B
:1073E000CB0199272AE030E0B9010E940AE1482F39
:1073F000CB01B9010E940AE1805D8093FF03405DEB
:1074000040930004109201048FEF93E00E94DBBED2
:1074100080E290E00E941A91E0EBFFE084918F01FE
:10742000882351F0082E000C990B0E941A910F5FCF
:107430001F4FF8018491F4CF80E290E00E941A91EE
:10744000C2016CE370E00E94F6E0EAE0F0E0BF0108
:107450000E940AE1282FCB01BF010E940AE1805D52
:107460008093FF03205D20930004109201048FEFAE
:1074700093E00E94DBBE80E290E00E941A91EEEA67
:10748000FFE084918F01882309F434CE082E000C8C
:10749000990B0E941A910F5F1F4FF8018491F3CF4F
:1074A00080E290E00E941A91E6EAFFE084918F0169
:1074B000882309F41FCE082E000C990B0E941A9104
:1074C0000F5F1F4FF8018491F3CF1092BC0E809193
:1074D000090180FF11C0E2EAFFE084918F01882357
:1074E00009F408CE082E000C990B0E941A910F5F28
:1074F0001F4FF8018491F3CF83E50E94B7BE882324
:1075000041F00E94D2BE0E9477DF7093910E60938B
:10751000900EEEE9FFE084918F01882351F0082E50
:10752000000C990B0E941A910F5F1F4FF801849174
:10753000F4CF8DE090E00E941A918AE090E00E94E2
:107540001A918091DA0E882309F4F3C08091900E8D
:107550009091910E009741F0049709F0A6C2EFE6D2
:10756000FAE084918F01C1C0E6EFFAE084918F01C7
:10757000882351F0082E000C990B0E941A910F5F7E
:107580001F4FF8018491F4CF8DE090E00E941A9192
:107590008AE090E00E941A91EFEEFAE084918F0168
:1075A000882351F0082E000C990B0E941A910F5F4E
:1075B0001F4FF8018491F4CF8DE090E00E941A9162
:1075C0008AE090E00E941A91E8EDFAE084918F0140
:1075D000882351F0082E000C990B0E941A910F5F1E
:1075E0001F4FF8018491F4CF8DE090E00E941A9132
:1075F0008AE090E00E941A91E1ECFAE084918F0118
:10760000882351F0082E000C990B0E941A910F5FED
:107610001F4FF8018491F4CF8DE090E00E941A9101
:107620008AE090E00E941A91EDEAFAE084918F01DD
:10763000882351F0082E000C990B0E941A910F5FBD
:107640001F4FF8018491F4CF8DE090E00E941A91D1
:107650008AE090E00E941A91E9E9FAE084918F01B2
:10766000882351F0082E000C990B0E941A910F5F8D
:107670001F4FF8018491F4CF8DE090E00E941A91A1
:107680008AE090E00E941A91EBE8FAE084918F0181
:10769000882351F0082E000C990B0E941A910F5F5D
:1076A0001F4FF8018491F4CF8DE090E00E941A9171
:1076B0008AE090E00E941A91EDE7FAE084918F0150
:1076C000882351F0082E000C990B0E941A910F5F2D
:1076D0001F4FF8018491F4CF8DE090E00E941A9141
:1076E0008AE090E00E941A91E0C1882351F0082EB0
:1076F000000C990B0E941A910F5F1F4FF8018491A3
:10770000F4CF8DE090E00E941A918AE090E00E9410
:107710001A91E1E6FAE084918F018823E9F2082EBC
:10772000000C990B0E941A910F5F1F4FF801849172
:10773000F4CF8091820A882309F48EC181E080937E
:10774000FE0C1092000D1092FF0C40E050E0BA01C8
:1077500080ED9AE00E949CB98BE1E0EDFAE0DE0159
:10776000159601900D928A95E1F78091CE0A90913D
:10777000CF0A9C838B8389EF92E09A83898340E0D0
:1077800050E0BE016F5F7F4F80E090E00E94559314
:10779000CE0101960E9454556090FF0C7090000D30
:1077A0000091900E1091910EC301801B910B0497D4
:1077B00020F03801F3E06F0E711C6BE2262E6AE0B8
:1077C000362E72E5872E7AE0972EE3E44E2EEAE01D
:1077D0005E2E6016710608F468C10115110509F0E6
:1077E000A1C064E87AE080ED9AE00E94BE9B6BE263
:1077F00073E084E89AE00E9493E1892B09F04AC083
:10780000F401849152E5A52E5AE0B52E882359F053
:10781000082E000C990B0E941A91FFEFAF1ABF0AB5
:10782000F5018491F3CF8DE090E00E941A918AE0F7
:1078300090E00E941A91F201849143E4A42E4AE060
:10784000B42E882359F0082E000C990B0E941A912F
:10785000FFEFAF1ABF0AF5018491F3CF8DE090E0FE
:107860000E941A918AE090E00E941A914AE060E03A
:1078700070E0CB010E942296E3E3FAE084915F017D
:107880002FEFA21AB20A882309F4E3C00E941896C7
:10789000F501F4CFEFE2FAE084915F01882359F01B
:1078A000082E000C990B0E941A91FFEFAF1ABF0A25
:1078B000F5018491F3CF8DE090E00E941A918AE067
:1078C00090E00E941A91F10184913BE2A32E3AE0EC
:1078D000B32E882359F0082E000C990B0E941A91A0
:1078E000FFEFAF1ABF0AF5018491F3CF8DE090E06E
:1078F0000E941A918AE090E00E941A914AE060E0AA
:1079000070E0CB010E942296E6E2FAE084915F01EA
:107910002FEFA21AB20A882309F49BC00E9418967E
:10792000F501F4CF60E070E0C80101970E94D4BB7C
:107930008091830A882309F460C0E4E2FAE084912C
:107940005F01882359F0082E000C990B0E941A91B0
:10795000FFEFAF1ABF0AF5018491F3CF84E89AE0F4
:107960000E94DBBE8DE090E00E941A918AE090E0D8
:107970000E941A91E2E2FAE084915F01882359F0B3
:10798000082E000C990B0E941A91FFEFAF1ABF0A44
:10799000F5018491F3CF81E99AE00E94DBBE8DE08E
:1079A00090E00E941A918AE090E00E941A91C8012A
:1079B000A0E0B0E04AE0BC01CD010E942296E0E2E6
:1079C000FAE084915F012FEFA21AB20A811105C07B
:1079D00021E9A22E2AE0B22E04C00E941896F501D9
:1079E000F0CFF50181915F01882319F00E9418966C
:1079F000F8CF8AE00E9418962CC084E89AE00E9492
:107A0000DBBE8DE090E00E941A918AE090E00E9437
:107A10001A9181E99AE00E94DBBE8DE090E00E941D
:107A20001A918AE090E00E941A91C801A0E0B0E0AB
:107A30004AE0BC01CD010E94229691E9A92E9AE06C
:107A4000B92EF50181915F01882399F20E94189661
:107A5000F8CF0F5F1F4FBDCEE1E1FAE084918F01B7
:107A6000882351F0082E000C990B0E941A910F5F89
:107A70001F4FF8018491F4CF8DE090E00E941A919D
:107A80008AE090E00E941A91E2E0FAE084918F018E
:107A9000882309F421CE082E000C990B0E941A911C
:107AA0000F5F1F4FF8018491F3CFEAE9FFE0849163
:107AB0008F01882309F41ECB082E000C990B0E941D
:107AC0001A910F5F1F4FF8018491F3CF8091810AC3
:107AD000882339F00E941E91BBC48091810A8823BB
:107AE00089F10E94E5BFB4C480918E0E823019F0F6
:107AF000833609F0ADC40E94A292E6E9FFE08491CA
:107B00008F01882351F0082E000C990B0E941A91C6
:107B10000F5F1F4FF8018491F4CF8DE090E00E9439
:107B20001A918AE090E00E941A91EBE6FFE08491BE
:107B30008F010F5F1F4F882309F48AC40E94189693
:107B4000F801F5CF80918E0E833609F081C4C9CF3C
:107B500082E69FE00E94775580912B0A90912C0A33
:107B6000891B8F7009F074C480918E0E823009F4E5
:107B70006FC4833609F0A1C46BC480912B0A909125
:107B80002C0A891B8F7009F063C480918E0E82309D
:107B900009F45EC4833609F45BC480914C0C8111F6
:107BA0000AC556C483E50E94B7BE811126C083E48E
:107BB0000E94B7BE882309F44BC480912B0A909190
:107BC0002C0A891B8F7009F043C420E030E040E2AA
:107BD00051E4609114047091150480911604909101
:107BE00017040E9417DA87FF08C089EC9EE0909383
:107BF0001C0880931B080E94C16F0E94D2BE20E027
:107C000030E0A9010E9417DA87FD0FC00E94D2BEA2
:107C100020E030E849E853E40E9454E0181644F0AC
:107C20000E94D2BE0E9477DF05C060E070E002C013
:107C300063E171E0709325046093240480E00E9466
:107C4000986606C483E50E94B7BE882309F400C481
:107C50000E94D2BE20E030E0A9010E9417DA87FD21
:107C600011C00E94D2BE20E030E046E153E40E9401
:107C700054E018164CF00E94D2BE0E9477DF362FD7
:107C8000272F04C030E001C036E920E0832F922F77
:107C90008E36910514F08EE690E090931F04809349
:107CA0001E040E944E66D4C383E50E94B7BE88239B
:107CB000D9F00E94D2BE20E030E04FE753E40E94AA
:107CC0007CDA20E030E048EC52E40E940ADF0E94B7
:107CD00077DF6F3F710519F010F06FEF70E0709370
:107CE0001D0460931C0406CA8FEF90E090931D045E
:107CF00080931C04FFC980912B0A90912C0A891B48
:107D00008F7009F0F7C98091810A8111F3C90E942F
:107D10000DA35F9A80910B048E7F80930B048A9A47
:107D2000479A80910B048D7F80930B04809108010A
:107D30008095817080930601479A80910B048B7F18
:107D400080930B04129AD6C983E50E94B7BE88239C
:107D500019F10E94D2BE20E030E040E252E40E94DD
:107D600017DA87FD0FC00E94D2BE20E030EC49E751
:107D700054E40E9454E0181644F00E94D2BE0E94BF
:107D800072DF05C068E270E002C067EE73E07093D6
:107D90000202609301025CC3E3ECFEE084918F0178
:107DA000882351F0082E000C990B0E941A910F5F46
:107DB0001F4FF8018491F4CF80900102909002024D
:107DC000092C000CAA08BB08B7FE0CC08DE20E946B
:107DD0001CBF66277727CB01681979098A099B0997
:107DE0004AE003C04AE0C501B4010E94DCBE82C97A
:107DF00080912B0A90912C0A891B8F7009F028C35F
:107E000080918E0E823009F423C3833609F0EEC2CE
:107E10001FC380912B0A90912C0A891B8F7009F047
:107E200069C980918E0E823009F464C9833609F0E5
:107E3000F7C360C980912B0A90912C0A891B8F701F
:107E400009F006C380918E0E823009F401C3833697
:107E500009F03CC5FDC280912B0A90912C0A891B28
:107E60008F7009F0F5C280918E0E823009F4F0C255
:107E7000833609F066C5ECC280912B0A90912C0ADA
:107E8000891B8F7009F0E4C280918E0E823009F454
:107E9000DFC2833609F090C5DBC28091BC0E811130
:107EA00003C00E94689125C18E3271F58091BD0E8C
:107EB0008E3209F0A6C08091210C882309F419C1E3
:107EC00081508093210C882361F090E001974FE16D
:107ED000489F9001499F300D1124C9018551954F4C
:107EE00002C08DEA9AE02BE1FC013496A0EDBAE0E5
:107EF00001900D922A95E1F7FC0182819381909384
:107F0000CF0A8093CE0AF5C08C3309F07AC06DE2B7
:107F100073E08CEB9EE00E9493E1892B21F481E0D9
:107F20008093DA0EE6C06CE373E08CEB9EE00E9477
:107F300093E1892B79F4E5EEF9E084918F010F5FED
:107F40001F4F882321F00E941896F801F6CF88ED84
:107F500099E044C063E573E08CEB9EE00E9493E1FE
:107F6000892B79F4E7EBF9E084918F010F5F1F4FC4
:107F7000882321F00E941896F801F6CF8FEA99E045
:107F80002DC067E673E08CEB9EE00E9493E1892BA5
:107F900079F4E4E9F9E084918F010F5F1F4F8823A2
:107FA00021F00E941896F801F6CF8FE899E016C0EC
:107FB00065E773E08CEB9EE00E9493E1892BA9F4C6
:107FC000E4E7F9E084918F010F5F1F4F882321F0D0
:107FD0000E941896F801F6CF8FE699E090931C085E
:107FE00080931B080E94C16F84C063E873E08CEB30
:107FF0009EE00E9493E1892B09F07BC01092DA0E7B
:1080000078C01D8218861C821B8289EF92E09A83B9
:1080100089838091D30A811103C06DEA7AE002C09E
:108020006CEC7AE06115710519F06C5F7F4F02C04E
:1080300060E070E021E04CEB5EE0CE0105960E942E
:1080400082A1882361F18BE1FE013596A0EDBAE0B3
:1080500001900D928A95E1F72B813C813093CF0AF4
:108060002093CE0A8091210C8A3008F03EC091E026
:10807000980F9093210CFFE18F9FC0011124DC0128
:10808000A151B54F4BE1E0EDFAE001900D924A9518
:10809000E1F7FC01E551F54F3383228326C0EEEC76
:1080A000F3E284918F010F5F1F4F882321F00E941C
:1080B0001896F801F6CFE9E5F9E084918F010F5F9A
:1080C0001F4F811103C00CEB1EE004C00E941896E4
:1080D000F801F3CFF80181918F01882319F00E94F4
:1080E0001896F8CF8AE00E941896CE0101960E9459
:1080F00054551092BC0E8091090180FFA9C1E0EE99
:10810000FDE084918F01882351F0082E000C990B1B
:108110000E941A910F5F1F4FF8018491F4CF8DE0F8
:1081200090E00E941A918AE090E00E941A91E2EB9E
:10813000FDE084918F010F5F1F4F882309F488C1F0
:108140000E941896F801F5CF8FE40E94B7BE811106
:108150000C947A3883E40E94B7BE0C947A3883E595
:108160000E94B7BE882369F0E5E9FDE084918F01A4
:108170000F5F1F4F882309F4C5C00E941896F801AD
:10818000F5CF8FE40E94B7BE882379F0E3E6FDE0E7
:1081900084918F010F5F1F4F882321F00E94189652
:1081A000F801F6CF8BE29DE013C084E50E94B7BED4
:1081B0008823A9F0E6E0FDE084918F010F5F1F4F57
:1081C000882321F00E941896F801F6CF8EED9CE0EE
:1081D00090931C0880931B080E94C16F93C083E496
:1081E0000E94B7BE882379F0EAEBFCE084918F010E
:1081F0000F5F1F4F882321F00E941896F801F6CFD9
:1082000081E99CE0E5CF81E50E94B7BE882379F043
:10821000EDE6FCE084918F010F5F1F4F882321F072
:108220000E941896F801F6CF85E49CE0D1CF88E44F
:108230000E94B7BE882389F1E6E2FCE084918F01B9
:108240000F5F1F4F882321F00E941896F801F6CF88
:10825000E2E2FCE084918F01882351F0082E000CAB
:10826000990B0E941A910F5F1F4FF8018491F4CF70
:108270008DE090E00E941A918AE090E00E941A91AD
:10828000EFEEFBE084918F010F5F1F4F882309F40D
:1082900039C00E941896F801F5CF8CE40E94B7BE51
:1082A000882381F1E3EDFBE084918F010F5F1F4F85
:1082B000882321F00E941896F801F6CFEFECFBE03E
:1082C00084918F01882351F0082E000C990B0E9495
:1082D0001A910F5F1F4FF8018491F4CF8DE090E069
:1082E0000E941A918AE090E00E941A91EFE8FBE068
:1082F00084918F010F5F1F4F882321F00E941896F1
:10830000F801F6CFE6E1FEE084918F01882311F4B5
:108310000C947A38082E000C990B0E941A910F5F6A
:108320001F4FF8018491F2CF80912B0A90912C0A73
:10833000891B8F7011F00C947A3880918E0E8230E8
:1083400011F40C947A38833609F068C30C947A38A7
:1083500083E50E94B7BE882309F47AC0EFE2FBE010
:1083600084918F010F5F1F4F882321F00E94189680
:10837000F801F6CF87E09BE090931C0880931B08E0
:108380000E94C16FE6E1FEE084918F01882311F421
:108390000C947A38082E000C990B0E941A910F5FEA
:1083A0001F4FF8018491F2CFE2E0FBE084918F014E
:1083B000882351F0082E000C990B0E941A910F5F30
:1083C0001F4FF8018491F4CFEDEFFAE084918F0113
:1083D000882311F40C947A38082E000C990B0E9413
:1083E0001A910F5F1F4FF8018491F2CF88E50E9428
:1083F000B7BE811106C089E50E94B7BE882309F483
:1084000001C188E50E94B7BE882341F08DEB9EE054
:1084100090931C0880931B080E94C16F89E50E94FD
:10842000B7BE882341F087EB9EE090931C088093B1
:108430001B080E94C16F8AE50E94B7BE882341F0E5
:1084400081EB9EE090931C0880931B080E94C16FF3
:108450008091870E9091880E019664E070E00E94F2
:108460000AE19093880E8093870E8091830E9091FD
:10847000840E01969093840E8093830E10928B0E3F
:1084800010928A0E0C9420374091870E5091880EDE
:10849000B9016F5F7F4F70938B0E60938A0E90E6E9
:1084A000949FF001959FF00D11242E0F3F1FF901AD
:1084B000ED5FF24F80830C94203700918C0E109169
:1084C0008D0E580124E0A20EB11C6AE270E0C501D5
:1084D0000E9488E1F80124812F3221F4B8016B5FFA
:1084E0007F4F03C02C3339F4B5018CEB9EE00E9422
:1084F0009CE10C947A381092BC0E009719F0FC01A4
:108500003197108280918C0E90918D0E40E061E049
:1085100004960E94DBBC80914C0C882331F1EEE57F
:10852000FFE084918F01882351F0082E000C990BF5
:108530000E941A910F5F1F4FF8018491F4CF8DE0D4
:1085400090E00E941A918AE090E00E941A91EFE276
:10855000FFE084918F010F5F1F4F882311F40C946B
:108560007A380E941896F801F4CFEBE2FFE084918C
:108570008F01882351F0082E000C990B0E941A914C
:108580000F5F1F4FF8018491F4CF8DE090E00E94BF
:108590001A918AE090E00E941A91E0E0FFE0849155
:1085A0008F010F5F1F4F882311F40C947A380E94BB
:1085B0001896F801F4CF0E94A292ECEFFEE08491AD
:1085C0008F01882351F0082E000C990B0E941A91FC
:1085D0000F5F1F4FF8018491F4CF8DE090E00E946F
:1085E0001A918AE090E00E941A91E0EDFEE08491F9
:1085F0008F010F5F1F4F882309F42ACF0E9418961E
:10860000F801F5CF8AE50E94B7BE8111FACE83E466
:108610000E94B7BE882309F41BCF8DEA9EE012CFDB
:1086200086E40E94B7BE882309F44DC10E94D2BEE1
:108630000E9477DF8B0189EA9EE090931C0880936B
:108640001B080E94C16F88E50E94B7BE882309F409
:1086500051C00E94D2BE2B013C012DEC3CEC4CE4FD
:108660005EE30E9417DA9E012F5F3F4F59011816F3
:1086700074F020E030E0A901C301B2010E9454E08F
:1086800018162CF41F930F938EE99EE005C12DEC74
:108690003CEC4CEC5DEBC301B2010E9417DA1816FA
:1086A0007CF020E030E040E85FEBC301B2010E94C3
:1086B00054E018162CF41F930F9382E99EE0ECC04F
:1086C0001F930F93C301B2010E9472DF7F936F93D8
:1086D00088E89EE09F938F93BF92AF920E94E8D963
:1086E0000FB6F894DEBF0FBECDBFCE0101960E943B
:1086F000996FDFC089E50E94B7BE882309F441C0A5
:108700000E94D2BE2B013C012DEC3CEC4CE45EE31C
:108710000E9417DAFE0131965F01181674F020E00E
:1087200030E0A901C301B2010E9454E018162CF4F4
:108730001F930F938DE79EE0AFC02DEC3CEC4CEC0B
:108740005DEBC301B2010E9417DA18167CF020E03D
:1087500030E040E85FEBC301B2010E9454E018161C
:108760002CF41F930F9381E79EE096C01F930F9305
:10877000C301B2010E9472DF7F936F9387E69EE090
:10878000A9CF8AE50E94B7BE882309F441C00E94A0
:10879000D2BE2B013C012DEC3CEC4CE45EE30E948C
:1087A00017DAFE0131965F01181674F020E030E010
:1087B000A901C301B2010E9454E018162CF41F93C2
:1087C0000F938CE59EE068C02DEC3CEC4CEC5DEB2F
:1087D000C301B2010E9417DA18167CF020E030E0E5
:1087E00040E85FEBC301B2010E9454E018162CF47C
:1087F0001F930F9380E59EE04FC01F930F93C3011B
:10880000B2010E9472DF7F936F9386E49EE062CF95
:1088100085E40E94B7BE882309F44BC00E94D2BEF3
:108820002B013C012DEC3CEC4CE45EE30E9417DA9A
:10883000FE0131965F01181674F020E030E0A901C6
:10884000C301B2010E9454E018162CF41F930F9339
:108850008BE39EE021C02DEC3CEC4CEC5DEBC301C6
:10886000B2010E9417DA18167CF020E030E040E8F0
:108870005FEBC301B2010E9454E018162CF41F9361
:108880000F938FE29EE008C0C301B2010E9472DF25
:108890007F936F9384E29EE09F938F93BF92AF92FA
:1088A0000E94E8D90F900F900F900F900F900F90AB
:1088B0001CCF80E29EE090931C0880931B080E94CE
:1088C000C16F0C947A3800E010E0B5CE20E030E0C3
:1088D00040E251E4609114047091150480911604F3
:1088E000909117040E9417DA87FF08C089E19EE083
:1088F00090931C0880931B080E94C16F82E390E054
:1089000090931F0480931E040E944E6688EC90E0B2
:10891000909325048093240480E00E949866E6E109
:10892000FEE084918F01882311F40C947A38082E8C
:10893000000C990B0E941A910F5F1F4FF801849150
:10894000F2CF20E030E040E251E4609114047091F5
:10895000150480911604909117040E9417DA87FF7E
:1089600008C08FE09EE090931C0880931B080E9433
:10897000C16F80E590E090931F0480931E040E94D5
:108980004E6680EF90E0909325048093240480E06D
:108990000E949866E6E1FEE084918F01882311F43D
:1089A0000C947A38082E000C990B0E941A910F5FD4
:1089B0001F4FF8018491F2CF1092250410922404E5
:1089C00080E00E94986610921F0410921E040E947C
:1089D0004E66EBE0FEE084918F01882351F0082E73
:1089E000000C990B0E941A910F5F1F4FF8018491A0
:1089F000F4CF8DE090E00E941A918AE090E00E940E
:108A00001A91E4EEFDE084918F010F5F1F4F8823E0
:108A100009F41ECD0E941896F801F5CF83E50E9457
:108A2000B7BE882309F479C0EAE8FBE084918F019E
:108A3000882351F0082E000C990B0E941A910F5FA9
:108A40001F4FF8018491F4CF20E030E048EC52E46D
:108A500060910704709108048091090490910A04C0
:108A60000E947CDA20E030E040E05FE30E942EDEEE
:108A70000E9472DFCB010E949D9A0E94DBBE8DE0B6
:108A800090E00E941A918AE090E00E941A91EDE530
:108A9000FBE084918F010F5F1F4F882321F00E941C
:108AA0001896F801F6CFE8E5FBE084918F010F5F9F
:108AB0001F4F882321F00E941896F801F6CF20E07E
:108AC00030E048EC52E46091070470910804809112
:108AD000090490910A040E947CDA20E030E040E032
:108AE0005FE30E942EDE0E9472DFCB010E949D9AFE
:108AF0008C01F80181918F01882319F00E9418964A
:108B0000F8CFE5E5FBE084918F010F5F1F4F8823CD
:108B100021F00E941896F801F6CF84E40E94B7BEB7
:108B2000882311F40C947A380E94D2BE20E030E001
:108B300048EC52E40E940ADF20E030E048EC52E4C6
:108B40000E947CDA0E9472DF2B013C0197FD0EC06F
:108B500020E137E240E050E00E941DE1CA01B90186
:108B6000A70196010E941DE1605D09C070946094A8
:108B700050944094411C511C611C711C6DE2609327
:108B80000004C301B20128EE33E040E050E00E944F
:108B90001DE1CA01B901A70196010E941DE1605DB6
:108BA00060930104C301B20124E630E040E050E0EC
:108BB0000E941DE1CA01B901A70196010E941DE1B1
:108BC000605D609302048EE280930304C301B201EE
:108BD000A70196010E941DE1162FCA01B901A70144
:108BE00096010E941DE1605D60930404105D109386
:108BF00005048EE49BE09F938F938E010F5F1F4FC0
:108C00001F930F930E94E8D960E074E0C8010E94AE
:108C10007DE1C8010E94996F89E49BE090931C0854
:108C200080931B080E94C16F0F900F900F900F90C0
:108C30000C947A386F960FB6F894DEBF0FBECDBF96
:108C4000DF91CF911F910F91FF90EF90DF90CF9028
:108C5000BF90AF909F908F907F906F905F904F905C
:108C60003F902F9008950E9441E11F920F920FB6FE
:108C70000F9211240BB60F922F933F934F935F9354
:108C80006F937F938F939F93AF93BF93EF93FF93D4
:108C900080912D0490912E04A0912F04B091300466
:108CA000892B8A2B8B2B59F180912C04E0912A047B
:108CB000F0912B0490818927808380912D049091DD
:108CC0002E04A0912F04B0913004181619061A062C
:108CD0001B060CF056C080912D0490912E04A0919B
:108CE0002F04B09130040197A109B10980932D049C
:108CF00090932E04A0932F04B093300442C080912F
:108D00000302E3E4F1E1E4919FEF90930302E23088
:108D1000C9F050F4EE2399F0E13081F590916F00A5
:108D20009D7F90936F002AC0E43019F1E0F0E530A8
:108D300029F5909173009D7F909373001FC010924E
:108D40006E001CC0909170009D7F9093700091E028
:108D50009093B0009091B100987F94609093B1008F
:108D60001092B3000BC0909171009D7F90937100A1
:108D700005C0909172009D7F9093720060E00E9408
:108D80008F60FF91EF91BF91AF919F918F917F91F4
:108D90006F915F914F913F912F910F900BBE0F906C
:108DA0000FBE0F901F9018952F923F924F925F9297
:108DB0006F927F928F929F92AF92BF92CF92DF92EB
:108DC000EF92FF92CF93DF9300D01F92CDB7DEB723
:108DD00060902404709025048090260490902704CD
:108DE000A0902804B0902904B301072C000C880B34
:108DF000990B0E941DDAA50194010E942DDE6B01E2
:108E00007C0160937206709373068093740690934E
:108E1000750620ED3CEC4CE45DE360910406709136
:108E2000050680910606909107060E947CDA1B01D8
:108E30002C0120916E0630916F0640917006509182
:108E40007106C501B4010E942DDE9B01AC01C20177
:108E5000B1010E947CDA1B012C0123E333E343E7D9
:108E60005FE360916A0670916B0680916C06909149
:108E70006D060E947CDA9B01AC01C201B1010E9427
:108E80002EDE69837A838B839C8360936A0670935A
:108E90006B0680936C0690936D0680926E0690929E
:108EA0006F06A0927006B092710620E030E040E2BA
:108EB00051E4C701B6010E9454E0181624F481E081
:108EC0008093690689C020E030E040E251ECC701A0
:108ED000B6010E9417DA87FD02C0672821F481E0FD
:108EE000809369069DC080916906882351F0109295
:108EF0006506109266061092670610926806109238
:108F000069062091000630910106409102065091B9
:108F10000306C701B6010E947CDA2B013C01609375
:108F200061067093620680936306909364062091B5
:108F30006506309166064091670650916806C70144
:108F4000B6010E942EDE4B015C01609365067093B2
:108F5000660680936706909368062091FC05309121
:108F6000FD054091FE055091FF050E947CDA9B01B2
:108F7000AC0160935D0670935E0680935F069093EC
:108F80006006C301B2010E942EDE29813A814B8125
:108F90005C810E942DDE2B013C0120E030E04FE798
:108FA00053E40E9454E020E030E0A9011816DCF4FC
:108FB000C701B6010E9454E0181674F4A701960187
:108FC000C501B4010E942DDE6093650670936606AC
:108FD0008093670690936806412C512C8FE7682E8A
:108FE00083E4782E20C0C301B2010E9417DA87FF04
:108FF0001AC020E030E0A901C701B6010E9417DACB
:1090000087FF0EC0A7019601C501B4010E942DDEA5
:109010006093650670936606809367069093680672
:10902000412C512C3201C301B2010F900F900F90CF
:109030000F90DF91CF91FF90EF90DF90CF90BF9096
:10904000AF909F908F907F906F905F904F903F90E8
:109050002F900895CF92DF92FF920F931F93CF939B
:10906000DF931F921F92CDB7DEB7F82E8A01809151
:109070001702882309F444C0E9EBF3E284916F01FD
:109080009FEFC91AD90A882341F069837A830E9425
:109090001896F60169817A81F1CFFB0184916F0105
:1090A0009FEFC91AD90A882321F00E941896F60169
:1090B000F5CFEDE1FBE184916F019FEFC91AD90A69
:1090C000882321F00E941896F601F5CFF7FC0BC01B
:1090D0006F2DFF0C770B880B990B0E9488968AE006
:1090E0000E9418960DC0E8E1FBE184916F019FEFAB
:1090F000C91AD90A882321F00E941896F601F5CFE3
:1091000080915C06811108C01092170281E0809363
:109110005C06C8010E9477550F900F90DF91CF91A8
:109120001F910F91FF90DF90CF900C94E266AF9269
:10913000BF92CF92DF92EF92FF920F931F93CF9344
:10914000DF9320E030E048E452E46091260470911F
:10915000270480912804909129040E9454E0181655
:109160004CF4E2E1FBE1E491C1E001C0CC0FEA95EF
:10917000EAF701C0C0E0E12CF12CA12CD0E0CC2416
:10918000C394D12CF701E45FF44EB490F701EE5E86
:10919000F44E0491B7FC24C08A2D90E0002E02C04A
:1091A000959587950A94E2F780FD1AC0BE01002EBE
:1091B00002C0759567950A94E2F761707727162FBC
:1091C0001195612F8B2D0E948F60612F70E08B2D88
:1091D0000E94FA60C60101C0880F0A95EAF7A82A22
:1091E0008FEFE81AF80A86E0E816F10459F6DF91E5
:1091F000CF911F910F91FF90EF90DF90CF90BF9094
:10920000AF9008950F931F9380914404813019F417
:109210000E94426208C060913C0470913D048091BC
:109220003E0490913F04009140041091410420912C
:10923000420430914304601B710B820B930B28EEA8
:1092400033E040E050E00E94F2DD809138049091DC
:109250003904A0913A04B0913B04BC01CD01620FE6
:10926000731F841F951F1F910F91089580914404CF
:10927000813099F1823051F4C5DF609338047093E6
:10928000390480933A0490933B0418C01092400430
:1092900010924104109242041092430410923C0434
:1092A00010923D0410923E0410923F041092380434
:1092B0001092390410923A0410923B0481E080939A
:1092C00044040E944262609340047093410480937E
:1092D00042049093430481E0089580E008958091D2
:1092E0004404813079F482E0809344040E94426215
:1092F00060933C0470933D0480933E0490933F043C
:1093000081E0089580E00895809144048150823086
:1093100010F080E00895109244040E94426260932D
:109320003C0470933D0480933E0490933F0481E09D
:10933000089590916F0091FB222720F991FF05C0BD
:1093400090916F009D7F90936F0034E0839FC001E8
:109350001124FC01E451FA4F4081518162817381F3
:10936000FC01E052FA4F408351836283738381E0B2
:109370008093DF05222329F080916F008260809323
:109380006F00089590916F0091FB222720F991FFC3
:1093900005C090916F009D7F90936F0094E0899F2E
:1093A000F0011124E451FA4F60817181828193812F
:1093B000222329F020916F00226020936F000895EE
:1093C000BC0120915A0630915B0640915A0650919B
:1093D0005B062417350711F09A01F7CF81E0621779
:1093E000730709F080E008950F930FB70F93009172
:1093F0006E000F930B7F00936E0000916F000D7F46
:1094000000936F000F930BB70F930CB70F921F923F
:109410002F933F934F935F936F937F938F939F937C
:10942000AF93BF93EF93FF9311244DD0FF91EF9132
:10943000BF91AF919F918F917F916F915F914F916C
:109440003F912F911F900F900CBF0F910BBF0F9169
:109450000260F89400936F000F9100936E000F91DB
:109460000FBF0F9118958091DD0580FF03C0899A89
:109470008FEF02C0899881E0809308068091DD0516
:1094800081FF03C08F988FEF02C08F9A81E0809395
:1094900009068091DD0582FF08C080910B01827072
:1094A0008093090143988FEF08C080910B0180954C
:1094B000827080930901439A81E080930A0600003C
:1094C0000000000008952F923F924F925F926F929A
:1094D0007F928F929F92AF92BF92CF92DF92EF9244
:1094E000FF920F931F93CF93DF9300D000D0CDB79F
:1094F000DEB7F8948FEF9FEF9093890080938800F8
:109500002AE02D83212C312C78948091560690915D
:109510005706A0915806B0915906892B8A2B8B2BA0
:1095200009F014C28091DF058823D1F01092DF0585
:1095300080915A0690915B06892B91F01092DE057E
:1095400010925B0610925A0690912B0A80912C0A79
:10955000981731F080912C0A8F5F8F7080932C0ABE
:1095600080915A0690915B06892B09F4EFC1009116
:109570005206109153062091540630915506909151
:10958000410640914E0650914F06609150067091F1
:109590005106401B510B620B730B892F90E0A0E02A
:1095A000B0E0481759076A077B0710F4DB01CA01CE
:1095B000482F800F911FA21FB31F809352069093D4
:1095C0005306A0935406B093550620918400309121
:1095D0008500225E3F4FC0902706D0902806E0907D
:1095E0002906F0902A068091170690911806A091FE
:1095F0001906B0911A068C0D9D1DAE1DBF1D8093DE
:10960000270690932806A0932906B0932A06B7FD53
:109610001CC0889AC090EC05D090ED05E090EE0556
:10962000F090EF0580910806082E000C990BAA0B0C
:10963000BB0B8C0D9D1DAE1DBF1D8093EC05909343
:10964000ED05A093EE05B093EF05C0902B06D090EA
:109650002C06E0902D06F0902E0680911B0690912E
:109660001C06A0911D06B0911E068C0D9D1DAE1D01
:10967000BF1D80932B0690932C06A0932D06B093CC
:109680002E06B7FD1CC08E9AC090F005D090F10553
:10969000E090F205F090F30580910906082E000C89
:1096A000990BAA0BBB0B8C0D9D1DAE1DBF1D80938E
:1096B000F0059093F105A093F205B093F305C090E7
:1096C0002F06D0903006E0903106F090320680915F
:1096D0001F0690912006A0912106B09122068C0DC4
:1096E0009D1DAE1DBF1D80932F0690933006A09345
:1096F0003106B0933206B7FD3EC09091DC058091F3
:109700000A069923C1F09091DA0592FF02C087FD05
:1097100005C09091D905992309F4A9C56091DA058E
:109720007091DB0573FF02C087FD0CC09091D805D6
:10973000911108C006C090910B019095987090937C
:109740000901419AC090F405D090F505E090F60526
:10975000F090F705082E000C990BAA0BBB0B8C0D93
:109760009D1DAE1DBF1D8093F4059093F505A0933C
:10977000F605B093F705C0903306D0903406E0901C
:109780003506F09036068091230690912406A0912C
:109790002506B09126068C0D9D1DAE1DBF1D809324
:1097A000330690933406A0933506B0933606B7FD82
:1097B0003AC08090F8059090F905A090FA05B09015
:1097C000FB05C0900B060C2C000CDD08EE08FF0812
:1097D000C80CD91CEA1CFB1CC092F805D092F905F4
:1097E000E092FA05F092FB05C0901306D0901406A3
:1097F000E0901506F09016068C199D09AE09BF0978
:109800008093330690933406A0933506B0933606C2
:109810009091DD0580913F0693FF02C0815001C009
:109820008F5F80933F06809184009091850082171E
:109830009307C8F38091270690912806A0912906E6
:10984000B0912A06B7FD15C0C0901306D09014063B
:10985000E0901506F09016068C199D09AE09BF0917
:109860008093270690932806A0932906B0932A0692
:10987000889880912B0690912C06A0912D06B0918E
:109880002E06B7FD15C0C0901306D0901406E090C8
:109890001506F09016068C199D09AE09BF09809334
:1098A0002B0690932C06A0932D06B0932E068E982F
:1098B00080912F0690913006A0913106B09132062A
:1098C000B7FD3AC0C0901306D0901406E09015067C
:1098D000F09016068C199D09AE09BF0980932F06DA
:1098E00090933006A0933106B09332068091DC0548
:1098F0008823E1F08091DA0582FF04C080910A0696
:1099000087FD05C08091D905882309F4B7C48091EB
:10991000DA059091DB0593FF04C080910A0687FD6C
:109920000BC08091D805811107C005C080910B0143
:109930008870809309014198415041F080918400E2
:109940009091850082179307C8F343CE809113024C
:1099500090911402A0911502B0911602892B8A2BC6
:109960008B2B09F094C080914006882309F455C0E0
:10997000C0905206D0905306E0905406F0905506E1
:1099800040913B0650913C0660913D0670913E0629
:1099900080913F064C155D056E057F0588F420918A
:1099A0000C0630910D06E0911006F0911106E217B9
:1099B000F30730F4815080933F062150310915C0E0
:1099C000C416D506E606F706E8F420910C06309199
:1099D0000D0640910E0650910F062417350790F49E
:1099E0008F5F80933F062F5F3F4F30930D0620938C
:1099F0000C0640910F02509110026091110270917B
:109A000012020EC08FEF9FEFDC0180930F02909344
:109A10001002A0931102B09312024FEF5FEFBA0150
:109A200080913F0687FD02C0169A01C016982091CA
:109A3000840030918500225E3F4F80913F0688234D
:109A4000F1F0149A80918400909185008217930719
:109A5000C8F380913F0687FF02C08F5F01C081502D
:109A600080933F06149880913F06882331F38091BC
:109A700084009091850082179307C8F3DCCF409350
:109A80001302509314026093150270931602809192
:109A9000560690915706A0915806B0915906892B09
:109AA0008A2B8B2B09F06CC3A0915A06B0915B06F0
:109AB000109739F1C0905206D0905306E0905406AA
:109AC000F090550640914E0650914F066091500619
:109AD00070915106C416D506E606F706C8F0109236
:109AE000DE0510925B0610925A0690912B0A809127
:109AF0002C0A981731F080912C0A8F5F8F70809319
:109B00002C0AA0ED8A2EA7E09A2EA12CB12C81C19F
:109B100040914A0650914B0660914C0670914D065B
:109B20004C155D056E057F0508F46EC04091460634
:109B3000509147066091480670914906D2960D9162
:109B40001D912D913C91D597EE27419FF12D529F6C
:109B5000C001629F900D619F800D911D429FF00D8D
:109B6000811D9E1F519FF00D811D9E1F609FF00D56
:109B7000811D9E1F509FF10D8E1F9E1FF6958E1FFB
:109B80009E1F349F800D911D359F900D1124FD0166
:109B9000EA5BFF4F0081118122813381080F191F79
:109BA000211D311D00934206109343062093440665
:109BB00030934506349780809180A280B3808016D0
:109BC0009106A206B30640F48092420690924306A4
:109BD000A0924406B09245068090420690904306BB
:109BE000A0904406B09045068CEE9AE177247394D9
:109BF000FC010591159125913491081519052A0547
:109C00003B0508F441C34BC320913B0630913C0611
:109C100040913D0650913E0629833A834B835C83F5
:109C20002C153D054E055F0508F068C040913706CC
:109C3000509138066091390670913A06D2960D918E
:109C40001D912D913C91D597EE27419FF12D529F6B
:109C5000C001629F900D619F800D911D429FF00D8C
:109C6000811D9E1F519FF00D811D9E1F609FF00D55
:109C7000811D9E1F509FF10D8E1F9E1FF6958E1FFA
:109C80009E1F349F800D911D359F900D11248C01D6
:109C900020E030E040904206509043066090440639
:109CA00070904506FD01E65BFF4F0415150526057E
:109CB000370580F480809180A280B380401A510AD9
:109CC000620A730A481459046A047B0438F42401B4
:109CD000350104C040805180628073808CEE9AE12F
:109CE00031E03E83FC0105911591259134910415D5
:109CF00015052605370508F44FC35BC380913F0661
:109D00008823D9F0D8964D915C91D99760E070E0A6
:109D100000910F0210911002209111023091120255
:109D2000041715072607370741F010921302109207
:109D30001402109215021092160240910B025091DB
:109D40000C0260910D0270910E0277FF5AC0AE5B5B
:109D5000BF4F8D919D910D90BC91A02D2CEE3AE1BD
:109D600041E0F901C590D590E590F490C816D90668
:109D7000EA06FB0658F4B695A79597958795440F84
:109D80002C5F3F4F5BE12830350759F74093410680
:109D900080329105A105B10508F4FAC38097A109A5
:109DA000B1098115E8E09E07A105B10508F4CBC310
:109DB00024E0929FF00111249F012451394EF901B2
:109DC000329645915491EE27859FB001849F610D95
:109DD0007E1F06946E1F7E1F1124AB0160E070E0B1
:109DE000F90185919491A0E0B0E0841B950BA60B3E
:109DF000B70B80930B0290930C02A0930D02B093CB
:109E00000E0280900B0290900C02A0900D02B09078
:109E10000E0280915A0690915B06892B09F0A8C129
:109E20000E9448C890935B0680935A06892B09F4D8
:109E30009FC160905A0670905B06D3018C9183FF9E
:109E40003FC0F30185899689A789B08D8093EC0581
:109E50009093ED05A093EE05B093EF05818D928D63
:109E6000A38DB48D8093F0059093F105A093F20536
:109E7000B093F305858D968DA78DB0A18093F405E1
:109E80009093F505A093F605B093F70581A192A1F3
:109E9000A3A1B4A18093F8059093F905A093FA05C6
:109EA000B093FB0590912B0A80912C0A981709F426
:109EB000B7CF80912C0A8F5F8F7080932C0AB0CF20
:109EC0005596CD90DD90ED90FC90589781E0C114AF
:109ED000D104E104F10409F480E0F301018D128D55
:109EE000238D348D011511052105310509F082609E
:109EF000D3015D964D915D916D917C919097411547
:109F000051056105710509F084608093DE051092AA
:109F10003706109238061092390610923A061092BF
:109F20004606109247061092480610924906F30121
:109F300085A196A1A7A1B0A580934E0690934F0648
:109F4000A0935006B0935106882499245401881A8E
:109F5000990AAA0ABB0A8092330690923406A0920C
:109F60003506B092360680922F0690923006A09267
:109F70003106B092320680922B0690922C06A09267
:109F80002D06B0922E068092270690922806A09267
:109F90002906B0922A06CC0CDD1CEE1CFF1CC092D8
:109FA0001706D0921806E0921906F0921A06000FD2
:109FB000111F221F331F00931B0610931C062093B2
:109FC0001D0630931E06440F551F661F771F4093D2
:109FD0001F0650932006609321067093220641A12C
:109FE00052A163A174A1440F551F661F771F4093B0
:109FF0002306509324066093250670932606880F47
:10A00000991FAA1FBB1F8093130690931406A09359
:10A010001506B0931606109252061092530610922F
:10A0200054061092550682A593A5A4A5B5A58093C4
:10A030004A0690934B06A0934C06B0934D0686A516
:10A0400097A5A0A9B1A980933B0690933C06A09345
:10A050003D06B0933E0681A58093120697A9909382
:10A060004006992361F024AD35AD3093110620935D
:10A07000100622AD33AD30930F0620930E06D301A8
:10A08000D6969C912091DD0592130AC020910A0278
:10A0900030E0482F082E000C550B4217530729F0CB
:10A0A0009093DD0580930A02DED90E9400C72FEF4E
:10A0B0003FEFA90120930B0230930C0240930D0255
:10A0C00050930E02F301EA5BFF4F80819181A281E0
:10A0D000B3818093420690934306A0934406B093C5
:10A0E00045062CEE3AE141E0F901C590D590E590A6
:10A0F000F490C816D906EA06FB0658F4B695A7955B
:10A1000097958795440F2C5F3F4FEBE128303E0732
:10A1100059F74093410680329105A105B10508F435
:10A120005FC28097A109B109811538E09307A105A5
:10A13000B10508F432C244E0949F900111242451E7
:10A14000394EF901329645915491EE27859FB00121
:10A15000849F610D7E1F06946E1F7E1F1124F901DE
:10A1600085909490A12CB12C861A970AA108B10869
:10A170008092560690925706A0925806B0925906C1
:10A1800000915606109157062091580630915906B5
:10A1900040911302509114026091150270911602C1
:10A1A0007801F22FE32F401751076207730718F465
:10A1B0007A01F62FE72FC701AF2FBE2F0097E1E0FE
:10A1C000AE07B10520F08FEF9FEFA0E0B0E0081BD5
:10A1D000190B2A0B3B0B009356061093570620933E
:10A1E0005806309359064F3FFFEF5F076F077F0711
:10A1F00061F0481B590B6A0B7B0B40931302509381
:10A2000014026093150270931602F8942091840052
:10A2100030918500205F3F4F4D8141504D83442355
:10A2200039F0280E391E2216330608F46DC901C014
:10A2300019013092890020928800789426960FB6F2
:10A24000F894DEBF0FBECDBFDF91CF911F910F916C
:10A25000FF90EF90DF90CF90BF90AF909F908F9046
:10A260007F906F905F904F903F902F9008959091C6
:10A270000B01909598709093090150CA80910B0141
:10A2800088708093090143CBB694A79497948794E0
:10A29000770C0496EBE188309E0709F0A9CC709208
:10A2A0004106F0E28F169104A104B10408F41CC128
:10A2B00090E2891A9108A108B1088114E8E09E068D
:10A2C000A104B104F8F0F4E09F9EC0011124845170
:10A2D000994EFC01329625913491F82DEE27F39F8B
:10A2E0008001F29F010D1E1F06940E1F1E1F1124D8
:10A2F000FC0185909490A12CB12C801A910AA108A0
:10A30000B10823C0950184013695279517950795C7
:10A31000F801EC7F9F0124513D4EF9018591949104
:10A32000F901329605911491E82DE770E09F9001B4
:10A33000E19F300D1124F3E036952795FA95E1F76A
:10A340004C01821A930AA12CB12C480D591D6A1D8B
:10A350007B1D4093460650934706609348067093D2
:10A36000490680914006882359F0472D50E060E06F
:10A3700070E0C416D506E606F70609F06CC084C086
:10A380002FEF3FEFA90120930F023093100240936B
:10A390001102509312029AC076946794579447948E
:10A3A0002E81220F2E8304963BE18830930709F01B
:10A3B00099CC2E812093410630E24316510461046A
:10A3C000710408F4BAC080E2481A510861087108A3
:10A3D000411498E059066104710408F48BC0E4E06C
:10A3E0005E9EC00111248451994EFC013296059164
:10A3F0001491F42DEE27F19F9001F09F210D3E1F47
:10A4000006942E1F3E1F1124FC0185909490A12CD0
:10A41000B12C821A930AA108B108480D591D6A1D72
:10A420007B1D40933706509338066093390670932E
:10A430003A06809140068823F1F149815A816B8167
:10A440007C812E81420F511D611D711D4C155D05D2
:10A450006E057F05C8F480913F06882309F4D9CCA6
:10A46000D8964D915C91D99760E070E000910F0211
:10A470001091100220911102309112020417150759
:10A480002607370709F4C5CC109213021092140264
:10A490001092150210921602D8968D919C91D99720
:10A4A000A0E0B0E080930F0290931002A0931102FD
:10A4B000B0931202AECC8FEF9FEFDC0180930F02BE
:10A4C00090931002A0931102B093120280913F0664
:10A4D000882309F49ECC1092130210921402109259
:10A4E00015021092160295CC10E2812E912CA12C0F
:10A4F000B12CDECE930182013695279517950795ED
:10A50000F801EC7FCF0184519D4EFC018590949021
:10A51000FC01329625913491E42DE770E29FC00151
:10A52000E39F900D112423E0969587952A95E1F7F6
:10A53000881A990AA12CB12C70CFF0E24F2E512C21
:10A54000612C712C40CFAC01BD0176956795579574
:10A550004795FA01EC7FAF0144515D4EFA01259118
:10A560003491FA013296459154918770849FB001DD
:10A57000859F700D1124CB01F3E096958795FA9590
:10A58000E1F7A901481B590BCA01A0E0B0E031CCAA
:10A5900080E290E0A0E0B0E001CCAC01BD01769596
:10A5A000679557954795FA01EC7F9F0124513D4EE1
:10A5B000F90185909490F901329625913491877034
:10A5C000829FA001839F500D1124CA0123E096951C
:10A5D00087952A95E1F7881A990AA12CB12CC8CD44
:10A5E00080E290E0A0E0B0E09CCD8EBD0DB407FE0F
:10A5F000FDCF08958FEF8EBD0DB407FEFDCF8EB554
:10A600000895CF92DF92EF92FF92CF93DF93EC0108
:10A61000C090A506D090A606E090A706F090A806E8
:10A62000A7019601688179818A819B810E9417DA4E
:10A6300087FF04C0C882D982EA82FB82C090A90643
:10A64000D090AA06E090AB06F090AC06A701960168
:10A650006C817D818E819F810E9417DA87FF04C003
:10A66000CC82DD82EE82FF82C0902802D090290247
:10A67000E0902A02F0902B02A7019601688179816F
:10A680008A819B810E9454E0181624F4C882D982E2
:10A69000EA82FB82C0902C02D0902D02E0902E0224
:10A6A000F0902F02A70196016C817D818E819F81A0
:10A6B0000E9454E0181624F4CC82DD82EE82FF82E0
:10A6C000C090AD06D090AE06E090AF06F090B00618
:10A6D000A7019601688579858A859B850E9417DA8E
:10A6E00087FF04C0C886D986EA86FB86C090300200
:10A6F000D0903102E0903202F0903302A70196012F
:10A70000688579858A859B850E9454E0181624F413
:10A71000C886D986EA86FB86DF91CF91FF90EF90BD
:10A72000DF90CF9008954F925F926F927F928F92B9
:10A730009F92AF92BF92CF92DF92EF92FF920F93D0
:10A740001F93CF93DF93D82EC82FD0E0FE01EF5D8B
:10A75000F24EC49082E0D81203C081E08093DC0501
:10A760007E01EE0CFF1CEE0CFF1CF701EB5EF24EBF
:10A7700045905590659074906C2D0C2C000C770BC7
:10A78000880B990B0E941DDA4B015C0120E030E040
:10A7900040EC5FE3C301B2010E947CDAA5019401A1
:10A7A0000E947CDAAB01BC0100E010E098018D2D25
:10A7B0000E9480A9F701E75FF24E259135914591FE
:10A7C0005491C501B4010E947CDA4B015C0120E088
:10A7D00030E0A9010E9417DA882309F448C000E09C
:10A7E00010E09801B501A40170588D2D0E9480A938
:10A7F000FE01EA5FF24EC491C11117C0EEECF3E224
:10A800008491EF012196882321F00E941896FE0181
:10A81000F7CFE4EEFCE18491EF012196882321F04B
:10A820000E941896FE01F7CFCAE0F701EC52F34EF2
:10A8300045905590659074906C2F70E080E090E0AA
:10A840000E941DDA9B01AC01C301B2010E940ADF24
:10A850002B013C01A5019401C501B4010E942EDE2B
:10A86000AB01BC01930182018D2D0E9480A982E081
:10A87000D81250C0409014105090151060901610CF
:10A880007090171020E030E0A901C301B2010E94CE
:10A8900054E05301420187FF04C0B7FAB094B7F8FF
:10A8A000B09420E030E0A901C501B4010E9417DA9C
:10A8B000882381F1C1E01C145CF0C0E020E030E0AE
:10A8C000A901C301B2010E9417DA87FF0EC009C0B7
:10A8D00020E030E0A901C301B2010E9454E0181643
:10A8E00024F481E08093D90503C081E08093D805EA
:10A8F000CC2321F0B7FAB094B7F8B09400E010E0A0
:10A900009801B501A40182E00E9480A91092D905A6
:10A910001092D8051092DC0581E090E00D2C01C06A
:10A92000880F0A94EAF790910B04982B90930B04EC
:10A9300090916310892B80936310F701E756F94FCC
:10A9400010821182128213828D2D0E94596FF7019D
:10A95000E853F34E85919591A591B491E701C45FB9
:10A96000DB4F88839983AA83BB830E94A472F7017B
:10A97000E95BFF4E88819981AA81BB8180839183A5
:10A98000A283B383DF91CF911F910F91FF90EF903E
:10A99000DF90CF90BF90AF909F908F907F906F90FF
:10A9A0005F904F9008954F925F926F927F928F9237
:10A9B0009F92AF92BF92CF92DF92EF92FF92CF938E
:10A9C0006B017C0149015A0120E030E040E151E493
:10A9D0000E942EDE2B013C0121E338E040EA50ECDE
:10A9E0000E9454E087FD50C022E430E042E553E489
:10A9F000C301B2010E9417DA18160CF445C020E01A
:10AA000030E040EB51E4C501B4010E942EDE2B0181
:10AA10003C012FE632E143E85AEB0E9454E087FD07
:10AA200033C022E430E042E553E4C301B2010E94A6
:10AA300017DA18164CF127EE3BEF4FE151E4C7014E
:10AA4000B6010E9454E087FD1FC022E430E048E4D4
:10AA500053E4C701B6010E9417DA1816ACF027EECE
:10AA60003BEF4FE151E4C501B4010E9454E087FD82
:10AA70000BC0C1E022E430E04CE353E4C501B40173
:10AA80000E9417DA18160CF4C0E08C2FCF91FF90BB
:10AA9000EF90DF90CF90BF90AF909F908F907F907E
:10AAA0006F905F904F90089529EF32E0FC01318361
:10AAB000208304960C9409965F9A80910B048E7FF4
:10AAC00080930B048A9A479A80910B048D7F809320
:10AAD0000B04809108018095817080930601479A4C
:10AAE00080910B048B7F80930B04129A0895E9EBFD
:10AAF000F3E28491EF012196882321F00E941896B9
:10AB0000FE01F7CFE8EAFCE18491EF01219688236A
:10AB100021F00E941896FE01F7CF0E94E266CCDF7A
:10AB2000E4EAFCE18491EF01882349F0082E000C4F
:10AB3000990B0E941A912196FE018491F5CF8DE028
:10AB400090E00E941A918AE090E00E941A91EDE74D
:10AB5000FCE18491EF012196882321F00E94189650
:10AB6000FE01F7CFFFEF2BE48DE1F1502040804054
:10AB7000E1F700C00000F8949FEFE4E3FCE091509F
:10AB8000E040F040E1F700C000000E94E266A895B6
:10AB9000FECF2F923F924F925F926F927F928F9251
:10ABA0009F92AF92BF92CF92DF92EF92FF920F935C
:10ABB0001F93CF93DF9300D0CDB7DEB70E94DF3570
:10ABC0000E9442626B017C0110912302112309F45F
:10ABD0006FC080918B06882309F46AC04091E1061A
:10ABE0005091E2066091E3067091E4064601570138
:10ABF000841A950AA60AB70AB7FC6CC0833031F1F3
:10AC000034F481300CF454C0EEECF3E206C084302E
:10AC100009F04EC0EEECF3E233C084915F012FEFF8
:10AC2000A21AB20A882321F00E941896F501F5CFE6
:10AC3000E4EAFBE184915F014FEFA41AB40A882390
:10AC400009F436C00E941896F501F4CFEEECF3E259
:10AC500084915F019FEFA91AB90A882321F00E940D
:10AC60001896F501F5CFEDE8FBE184915F012FEF38
:10AC7000A21AB20A8823E1F00E941896F501F5CFD6
:10AC800084915F014FEFA41AB40A882321F00E9437
:10AC90001896F501F5CFE5E7FBE184915F019FEFA1
:10ACA000A91AB90A882321F00E941896F501F5CF58
:10ACB000212F30E0A8EEB3E00E941EDEC60ED71EA4
:10ACC000E81EF91EC092E106D092E206E092E30689
:10ACD000F092E40689B182FB882780F98093DB0E2D
:10ACE0009091DC0E98170CF04AC08091DD0E909187
:10ACF000DE0EA091DF0EB091E00E0196A11DB11DF8
:10AD0000883BEDE39E07A105B1050CF450C01092FD
:10AD1000DD0E1092DE0E1092DF0E1092E00E80918A
:10AD2000810A882319F00E941E9124C0E0EEFBE105
:10AD300084918F01882351F0082E000C990B0E94FA
:10AD40001A910F5F1F4FF8018491F4CF8DE090E0CE
:10AD50000E941A918AE090E00E941A91E6EBFBE1D2
:10AD600084918F010F5F1F4F882321F00E94189656
:10AD7000F801F6CF8091DB0E8093DC0E20C089179E
:10AD8000F1F01092DD0E1092DE0E1092DF0E109296
:10AD9000E00E8093DC0EE4EEFBE184918F010F5F07
:10ADA0001F4F882361F00E941896F801F6CF809318
:10ADB000DD0E9093DE0EA093DF0EB093E00E809137
:10ADC0007310843010F40E9419700E944262C09087
:10ADD0009006D0909106E0909206F0909306C114F0
:10ADE000D104E104F10471F100918C0610918D06FB
:10ADF00020918E0630918F060C0D1D1D2E1D3F1DBE
:10AE00004B015C01801A910AA20AB30AB7FC1AC06E
:10AE1000E9EBF3E284918F010F5F1F4F882321F04C
:10AE20000E941896F801F6CF60914310709144107B
:10AE300083E49CE10E94D0C88AE00E9418968AE3CD
:10AE40009CE17BC0C0902402D0902502E0902602B5
:10AE5000F0902702C114D104E104F104E9F130912A
:10AE60002B0A20912C0A321749F060938C067093BC
:10AE70008D0680938E0690938F062EC000918C06CF
:10AE800010918D0620918E0630918F060C0D1D1DA0
:10AE90002E1D3F1DDC01CB01801B910BA20BB30BC0
:10AEA000B7FD1AC05F9A80910B048E7F80930B04CC
:10AEB0008A9A479A80910B048D7F80930B0480912E
:10AEC00008018095817080930601479A80910B0458
:10AED0008B7F80930B04129A8091F3069091F40675
:10AEE000909902C0019604C0181619062CF4019717
:10AEF0009093F4068093F3068091F3069091F40604
:10AF00008E3E9240DCF0E9EBF3E284918F010F5F1B
:10AF10001F4F882321F00E941896F801F6CFEAE12E
:10AF2000FCE184918F010F5F1F4F882321F00E9465
:10AF30001896F801F6CF81E19CE1D9DD0E944262CA
:10AF40000091EF061091F0062091F1063091F20683
:10AF50004B015C01801A910AA20AB30AB7FC4EC0E9
:10AF60008B019C010C53164F2F4F3F4F0093EF0660
:10AF70001093F0062093F1063093F2064F9BB0C178
:10AF80007A9BAEC12091060120FFAAC12091FE0646
:10AF90002111A6C1029BA4C10091EB061091EC0601
:10AFA0002091ED063091EE060115110521053105C0
:10AFB00099F0DC01CB01801B910BA20BB30B8056E7
:10AFC0009A4EA109B1098827B7FD83959927AA2729
:10AFD000BB27682F619501C060E0262F30E03093D9
:10AFE000EA062093E9068091020161118095807143
:10AFF00080930001B90187E00E94FA6090912B0ACA
:10B0000080912C0A981791F0E0912C0A28E5E29F94
:10B01000F0011124ED5EFE4E608180912C0A90912A
:10B020002B0A891729F08F5F8F70F9CF60911C046C
:10B0300070E089E00E94FA608091F906882309F4A3
:10B0400000C10091570210915802809059028B82E2
:10B0500090905A029A8260912404709125046E5F48
:10B060007F4F072E000C880B990B0E941DDA980168
:10B07000A4010E9417DA87FDE4C0F0902C0A212C6D
:10B08000312CE12C198280912B0AF81609F464C046
:10B090008F2D90E038E5A32EA89EF001A99EF00D1B
:10B0A0001124EF53FF4E458956896789708D452BD2
:10B0B000462B472B81F4418D528D638D748D452B2A
:10B0C000462B472B41F4458D568D678D70A1452B3E
:10B0D000462B472BE1F128E5B22EB89E9001B99E90
:10B0E000300D1124C9018F539F4E6C01FC01618109
:10B0F0007281838194810E9499E04B015C01F60189
:10B1000061A172A183A194A10E941BDA2B013C01D1
:10B11000F60165A176A187A190A50E941BDA9B018B
:10B12000AC01C301B2010E940ADFA50194010E9493
:10B130007CDA5B016C019B01AC01B1018E2D998120
:10B140000E9417DA87FF03C01501EC2CD98281E039
:10B150008F0D8F70F82E97CF20915B0230915C029B
:10B1600040915D0250915E02B1018E2D99810E9445
:10B170007CDA9B01AC01B8018B819A810E942EDEA2
:10B180006B017C0198014B815A810E9417DA87FD7F
:10B1900015C00091530210915402809055028B8289
:10B1A000909056029A829801A401B601C7010E94AC
:10B1B00054E018161CF08601EB82FA82C090E50676
:10B1C000D090E606E090E706F090E806A701960129
:10B1D000B8018B819A810E9417DA87FF1CC020E09A
:10B1E00037ED43EA5CE3B8018B819A810E947CDAF7
:10B1F0004B015C0128E431EE4AE75FE3C701B60189
:10B200000E947CDA9B01AC01C501B4010E942EDED4
:10B210008B018B839A83C801AB81BA818093E50649
:10B220009093E606A093E706B093E806B801CD0137
:10B230000E9472DF709325046093240480E00E94D2
:10B2400098660E94C16781E69AE00E94E669B09024
:10B250009806BB2009F44DC00E94426200919406FA
:10B26000109195062091960630919706DC01CB014E
:10B27000801B910BA20BB30BB7FD3BC00E94426237
:10B280006B017C012B2D30E0A8EEB3E00E941EDEA6
:10B29000DC01CB018C0D9D1DAE1DBF1D809394065E
:10B2A00090939506A0939606B09397060E9420640B
:10B2B0008AE00F900F900F90DF91CF911F910F9127
:10B2C000FF90EF90DF90CF90BF90AF909F908F90C6
:10B2D0007F906F905F904F903F902F900C941896B6
:10B2E0006093EB067093EC068093ED069093EE0668
:10B2F00053CE0F900F900F90DF91CF911F910F9130
:10B30000FF90EF90DF90CF90BF90AF909F908F9085
:10B310007F906F905F904F903F902F9008952F9265
:10B320003F924F925F926F927F928F929F92AF92D5
:10B33000BF92CF92DF92EF92FF920F931F93CF9322
:10B34000DF93CDB7DEB7CC54D1090FB6F894DEBF8A
:10B350000FBECDBF80912202882319F087E490E1CF
:10B3600050D980910E0883FDA9C0C0905310D09091
:10B370005410E0905510F090561020911804309120
:10B38000190440911A0450911B04C701B6010E9490
:10B3900017DA882309F492C060912604709127047B
:10B3A000809128049091290420910D0821112BC02F
:10B3B0000E9472DF20913B0230913C0262177307BA
:10B3C00014F5C0921804D0921904E0921A04F09275
:10B3D0001B04EEECF3E284917F019FEFE91AF90A76
:10B3E000882321F00E941896F701F5CFEAE5FBE1EA
:10B3F00084917F01AFEFEA1AFA0A882321F00E94B4
:10B400001896F701F5CF8090531090905410A090AB
:10B410005510B090561020911804309119044091A5
:10B420001A0450911B04C501B4010E942DDE6B016A
:10B430007C0120E030E0A9010E9454E087FF04C0B5
:10B44000F7FAF094F7F8F094E0918A06B4E0EB9FF5
:10B45000F0011124E95CFD4F20813181428153814B
:10B46000C701B6010E947CDA20E030E048E453E4F2
:10B470000E9454E0181614F5809218049092190452
:10B48000A0921A04B0921B04EEECF3E284917F01C7
:10B490009FEFE91AF90A882321F00E941896F70114
:10B4A000F5CFEBE3FBE184917F01AFEFEA1AFA0AF3
:10B4B000882321F00E941896F701F5CF80916C1037
:10B4C0006090010270900202C0904710D090481026
:10B4D000E0904910F0904A1080904B1090904C10E2
:10B4E000A0904D10B0904E10882309F47DC220909A
:10B4F0006D1030906E1040906F105090701020E0E2
:10B5000030E0A901C201B1010E9417DA882371F06D
:10B51000A201910160914F107091501080915110D3
:10B52000909152100E9417DA87FF5EC2B301770C28
:10B53000880B990B0E941DDA209142023091430240
:10B5400040914402509145020E947CDA2AE037ED96
:10B5500043E25CE30E947CDA6DA77EA78FA798ABDD
:10B5600020910C0430910D0440910E0450910F0471
:10B57000C701B6010E942DDE2B013C012091100471
:10B58000309111044091120450911304C501B4018B
:10B590000E942DDE25966CAF7DAF8EAF9FAF2597B5
:10B5A00020E030E0A901C301B2010E9417DA811145
:10B5B00041C020E030E0A90125966CAD7DAD8EAD97
:10B5C0009FAD25970E9417DA811134C070908A06CA
:10B5D00019AA1AAA1BAA1CAAC982DA82EB82FC82C7
:10B5E0008D829E82AF82B88680914F1090915010CC
:10B5F000A0915110B091521089879A87AB87BC8770
:10B60000AE01475F5F4FBE016B5F7F4FCE0101967A
:10B610000E94C684FE01F1966F01E72C8E01035D46
:10B620001F4F23E530E1AE01475F5F4FBE016B5F07
:10B630007F4F27C2209114043091150440911604C5
:10B640005091170460914F107091501080915110DB
:10B65000909152100E942DDE29966CAF7DAF8EAF77
:10B660009FAF2997209118043091190440911A0432
:10B6700050911B046091531070915410809155109B
:10B68000909156100E942DDE21966CAF7DAF8EAF4B
:10B690009FAF2197A3019201C301B2010E947CDAFE
:10B6A0006B017C0125962CAD3DAD4EAD5FAD259770
:10B6B000CA01B9010E947CDA9B01AC01C701B60145
:10B6C0000E942EDE6B017C0129962CAD3DAD4EAD66
:10B6D0005FAD2997CA01B9010E947CDA9B01AC01D8
:10B6E000C701B6010E942EDE0E9499E06B017C0129
:10B6F0002DEB37E346E855E30E9417DA87FF17C0C2
:10B7000020E030E0A90121966CAD7DAD8EAD9FADFE
:10B7100021970E9454E02196CCACDDACEEACFFAC9E
:10B72000219787FF04C0F7FAF094F7F8F0942DEB17
:10B7300037E346E855E3C701B6010E9417DA87FDF3
:10B74000A4C120E030E040EA50E4C701B6010E9405
:10B750000ADF0E9477DF1B01672B19F42224239450
:10B76000312CB10180E090E00E941BDA9B01AC011A
:10B7700060E070E080E89FE30E940ADF4B015C011B
:10B780009B01AC01C701B6010E947CDA2D966CAF1B
:10B790007DAF8EAF9FAF2D97A5019401C301B2017C
:10B7A0000E947CDA698B7A8B8B8B9C8BA501940130
:10B7B00025966CAD7DAD8EAD9FAD25970E947CDA50
:10B7C0006D8B7E8B8F8B988FA501940129966CAD24
:10B7D0007DAD8EAD9FAD29970E947CDA698F7A8FFF
:10B7E0008B8F9C8FA501940121966CAD7DAD8EADA4
:10B7F0009FAD21970E947CDA6D8F7E8F8F8F98A3EB
:10B8000080E1ECE0F4E0DE01119601900D928A9562
:10B81000E1F7992493945E01F1E1AF0EB11CB1E020
:10B820002B1A310809F495C08091D906811111C0F5
:10B8300029D6DC01CB0188539F4FAF4FBF4F809378
:10B84000D5069093D606A093D706B093D8069092CB
:10B85000D9060E94C16716D6C090D506D090D606EC
:10B86000E090D706F090D806DC01CB018C199D0939
:10B87000AE09BF09B7FD10C005D6DC01CB01885366
:10B880009F4FAF4FBF4F8093D5069093D606A0939E
:10B89000D706B093D8067DD96501CE0101967C010B
:10B8A000D6012D913D914D915D916D01F701608122
:10B8B0007181828193810E942EDED7016D937D93E9
:10B8C0008D939D937D01AA15BB0551F7E0908A06E3
:10B8D0002D968CAD9DADAEADBFAD2D978DAB9EAB16
:10B8E000AFABB8AF89819A81AB81BC8189A39AA3A0
:10B8F000ABA3BCA38D819E81AF81B8858DA39EA390
:10B90000AFA3B8A789859A85AB85BC8589A79AA777
:10B91000ABA7BCA7AE01475D5F4FBE016B5D7F4F1C
:10B92000CE0181960E94C684DE01D5966D018E01FE
:10B93000035D1F4F9E01235F3F4FAE01475D5F4F89
:10B94000BE016B5D7F4FCE0181960E942A748111EA
:10B9500066CFE0908A062D968CAD9DADAEADBFADA5
:10B960002D9789AF9AAFABAFBCAF80914710909144
:10B970004810A0914910B0914A1089A39AA3ABA393
:10B98000BCA380914B1090914C10A0914D10B091A0
:10B990004E108DA39EA3AFA3B8A780914F10909196
:10B9A0005010A0915110B091521089A79AA7ABA73F
:10B9B000BCA7AE01475D5F4FBE016B5D7F4FCE01FF
:10B9C00081960E94C684DE01D9966D018E01035DC9
:10B9D0001F4F23E530E1AE01475D5F4FBE016B5D58
:10B9E0007F4FCE0181964FC0B301770C880B990B26
:10B9F0000E941DDA2091420230914302409144029C
:10BA0000509145020E947CDA2AE037ED43E25CE384
:10BA10000E947CDA69AB7AAB8BAB9CAB70908A06E8
:10BA200080914F1090915010A0915110B0915210F0
:10BA3000C982DA82EB82FC82898A9A8AAB8ABC8AC2
:10BA400089A39AA3ABA3BCA31DA61EA61FA618AAD2
:10BA5000AE014F5D5F4FBE016F5E7F4FCE0101961D
:10BA60000E94C684FE01BD966F01E72C8E010F5C1B
:10BA70001F4F23E530E1AE014F5D5F4FBE016F5EAA
:10BA80007F4FCE0101960E942A7480E1E7E4F0E145
:10BA9000ACE0B4E001900D928A95E1F7C45BDF4F12
:10BAA0000FB6F894DEBF0FBECDBFDF91CF911F91CF
:10BAB0000F91FF90EF90DF90CF90BF90AF909F904D
:10BAC0008F907F906F905F904F903F902F90089550
:10BAD0000F931F93CF93DF9380E00E94C249CEE77C
:10BAE000D6E00E941DDA01EA10E1F80120813181DF
:10BAF000428153810E947CDA688379838A839B83A5
:10BB000081E00E94C2490E941DDAF801248135813A
:10BB1000468157810E947CDA6C837D838E839F836C
:10BB200082E00E94C2490E941DDAF8012085318519
:10BB3000428553850E947CDA688779878A879B874C
:10BB4000DF91CF911F910F9108954F925F926F9265
:10BB50007F928F929F92AF92BF92CF92DF92EF929D
:10BB6000FF920F931F93CF93DF93EC016091140822
:10BB700070911508072E000C880B990B0E941DDA96
:10BB80009B01AC01688179818A819B810E942DDEB5
:10BB90006B017C016091160870911708072E000C4C
:10BBA000880B990B0E941DDA9B01AC016C817D8191
:10BBB0008E819F810E942DDE4B015C01A7019601C1
:10BBC00060911E0270911F028091200290912102CB
:10BBD0000E9417DA882309F465C0C0921E02D09231
:10BBE0001F02E0922002F09221022091760630910D
:10BBF00077064091780650917906C701B6010E94F8
:10BC00007CDA2B013C010E94A3DF6B017C0120E068
:10BC100030E0A9010E9417DA87FD10C020E030E073
:10BC200040E050E4C701B6010E9454E018164CF4FD
:10BC3000C12CD12CE12C00E4F02E03C0C12CD12C5E
:10BC40007601A7019601C301B2010E942DDE2B01EE
:10BC50003C0120E030E0A9010E9417DA87FD09C00D
:10BC60004092D1065092D2066092D3067092D406CA
:10BC700008C01092D1061092D2061092D3061092EC
:10BC8000D406C701B6010E9472DF6093D006862FEA
:10BC9000660F990B01968230910514F082E090E0D6
:10BCA0008093CF06A501940160911A0270911B0246
:10BCB00080911C0290911D020E9417DAD091190206
:10BCC000C091D006811103C0DC1367C02DC18092E2
:10BCD0001A0290921B02A0921C02B0921D022091A7
:10BCE0007A0630917B0640917C0650917D06C50115
:10BCF000B4010E947CDA4B015C010E94A3DF6B015E
:10BD00007C0120E030E0A9010E9417DA87FD10C015
:10BD100020E030E040E050E4C701B6010E9454E06A
:10BD200018164CF4C12CD12CE12C10E4F12E03C0D8
:10BD3000C12CD12C7601A7019601C501B4010E9446
:10BD40002DDE4B015C0120E030E0A9010E9417DAF2
:10BD500087FD09C08092CB069092CC06A092CD06BA
:10BD6000B092CE0608C01092CB061092CC0610926C
:10BD7000CD061092CE06C701B6010E9472DF609315
:10BD8000CA06062E000C770B6F5F7F4F623071057D
:10BD900014F062E070E06093C9062091CA06DC13DB
:10BDA00005C080911802821709F474C0C09319026B
:10BDB000209318028C2FCC0F990BC22F220FDD0B72
:10BDC0009C01220F331F820F931FFC01EC0FFD1FFC
:10BDD000EE0FFF1FEE0FFF1FE85EFF4E2081318147
:10BDE000428153812093C5063093C6064093C7060F
:10BDF0005093C8060091C906002E000C110BFC01DF
:10BE0000E00FF11FEE0FFF1FEE0FFF1FE85EFF4E6A
:10BE100060817181828193810E942DDE6093C106D1
:10BE20007093C2068093C3069093C406E091CF0638
:10BE30000E2E000CFF0BCF01880F991FE80FF91F82
:10BE4000CE0FDF1FCC0FDD1FCC0FDD1FC85EDF4E16
:10BE5000288139814A815B812093BD063093BE06DB
:10BE60004093BF065093C006E00FF11FEE0FFF1F77
:10BE7000EE0FFF1FE85EFF4E60817181828193812A
:10BE80000E942DDE6093B9067093BA068093BB06BC
:10BE90009093BC068090CB069090CC06A090CD06E7
:10BEA000B090CE062091C1063091C2064091C306E3
:10BEB0005091C406C501B4010E947CDA2091C506E8
:10BEC0003091C6064091C7065091C8060E942EDEEA
:10BED0006B017C016093B5067093B6068093B7063C
:10BEE0009093B8062091B9063091BA064091BB06EE
:10BEF0005091BC06C501B4010E947CDA2091BD06B8
:10BF00003091BE064091BF065091C0060E942EDEC1
:10BF1000A70196010E942DDE6093B1067093B206D0
:10BF20008093B3069093B4062091B1063091B20687
:10BF30004091B3065091B4066091D1067091D2063B
:10BF40008091D3069091D4060E947CDA2091B506A8
:10BF50003091B6064091B7065091B8060E942EDE89
:10BF6000DF91CF911F910F91FF90EF90DF90CF90D5
:10BF7000BF90AF909F908F907F906F905F904F9009
:10BF80000895CF92DF92EF92FF920F931F93CF937A
:10BF9000DF936C017A018B01C0E0D0E0CE15DF05A4
:10BFA00089F0D8016D918D01D601ED91FC91019040
:10BFB000F081E02DC6011995892B11F47E0102C094
:10BFC0002196ECCFC701DF91CF911F910F91FF9088
:10BFD000EF90DF90CF90089590E0FC013197E2312F
:10BFE000F10508F04EC08827EC56FF4F8F4F0C9498
:10BFF00039E1809180008F7703C0809180008F7D30
:10C0000080938000089580918000877FF9CF84B568
:10C010008F7702C084B58F7D84BD08958091B00074
:10C020008F7703C08091B0008F7D8093B00008951A
:10C03000809190008F7707C0809190008F7D03C022
:10C0400080919000877F8093900008958091A00058
:10C050008F7707C08091A0008F7D03C08091A000E2
:10C06000877F8093A0000895809120018F7707C07B
:10C07000809120018F7D03C080912001877F809374
:10C08000200108953FB7F89480913B0790913C07B9
:10C09000A0913D07B0913E0726B5A89B05C02F3F54
:10C0A00019F00196A11DB11D3FBFBA2FA92F982FDE
:10C0B0008827820F911DA11DB11DBC01CD0142E059
:10C0C000660F771F881F991F4A95D1F70895CF9360
:10C0D000DF93282F30E0F901E758FF4D8491F901F3
:10C0E000ED5CFF4DD491F901E351F04EC491CC23A6
:10C0F00089F0811171DFEC2FF0E0EE0FFF1FED52A0
:10C10000F04EA591B491EC91ED2381E090E021F403
:10C1100080E002C080E090E0DF91CF9108951F930E
:10C12000CF93DF93282F30E0F901E758FF4D84913A
:10C13000F901ED5CFF4DD491F901E351F04EC4914A
:10C14000CC23C1F0162F811147DFEC2FF0E0EE0F6A
:10C15000FF1FE754F04EA591B4918FB7F8941111D9
:10C1600005C09C91ED2FE095E92302C0EC91ED2BE9
:10C17000EC938FBFDF91CF911F910895CF93DF9301
:10C1800090E0FC01ED5CFF4D2491FC01E351F04E89
:10C190008491882361F190E0880F991FFC01E1569A
:10C1A000F04EC591D491FC01E754F04EA591B491A5
:10C1B000611109C09FB7F8948881209582238883F4
:10C1C000EC912E230BC0623061F49FB7F894388154
:10C1D000822F809583238883EC912E2B2C939FBFF5
:10C1E00006C08FB7F894E8812E2B28838FBFDF918C
:10C1F000CF9108951F93CF93DF93182FEB0161E048
:10C20000BDDF209711F460E004C0CF3FD10531F4C9
:10C2100061E0812FDF91CF911F9181CFE12FF0E07D
:10C22000E758FF4DE4914E2F50E0FA013197E2318B
:10C23000F10508F09DC08827EA55FF4F8F4F0C94F9
:10C2400039E184B5806884BDC7BD97C084B580627C
:10C2500084BDC8BD92C080918000806880938000BA
:10C26000D0938900C093880088C08091800080624C
:10C2700080938000D0938B00C0938A007EC0809111
:10C280008000886080938000D0938D00C0938C00E4
:10C2900074C08091B00080688093B000C093B300F8
:10C2A0006CC08091B00080628093B000C093B400F5
:10C2B00064C080919000806880939000D093990032
:10C2C000C09398005AC08091900080628093900043
:10C2D000D0939B00C0939A0050C0809190008860DA
:10C2E00080939000D0939D00C0939C0046C08091A5
:10C2F000A00080688093A0008091A0008F7B809335
:10C30000A000D093A900C093A80037C08091A000DE
:10C3100080628093A000D093AB00C093AA002DC090
:10C320008091A00088608093A000D093AD00C0935E
:10C33000AC0023C080912001806880932001D093BD
:10C340002901C093280119C0809120018062809347
:10C350002001D0932B01C0932A010FC080912001AE
:10C36000886080932001D0932D01C0932C0105C0DB
:10C37000C038D1050CF04CCF46CFDF91CF911F9143
:10C3800008958F929F92AF92BF92CF92DF92EF92D9
:10C39000FF926B017C0176DE4B015C01C114D1047C
:10C3A000E104F104E9F06EDEDC01CB0188199909A2
:10C3B000AA09BB09883E9340A105B10578F321E0A5
:10C3C000C21AD108E108F10888EE880E83E0981EB1
:10C3D000A11CB11CC114D104E104F10421F7DECF8A
:10C3E000FF90EF90DF90CF90BF90AF909F908F9095
:10C3F0000895AF92BF92CF92DF92EF92FF920F9388
:10C40000CF93DF935C01EB0169017A0180E20E9426
:10C4100018960F3F11F084E501C082E40E9418963F
:10C420008AE30E941896F50160817181828193816F
:10C4300042E00E94A296488159816A817B8183E90A
:10C440009FE10E949AC820E030E040E85DE3C70128
:10C45000B6010E947CDAAB01BC0180E99FE10E9439
:10C460009AC889E20E94189662E070E080E090E04D
:10C47000DF91CF910F91FF90EF90DF90CF90BF9021
:10C48000AF907FCF2FB7F89460913707709138073E
:10C490008091390790913A072FBF08952F923F92CC
:10C4A0004F925F926F927F928F929F92AF92BF92C4
:10C4B000CF92DF92EF92FF920F931F93CF93DF9370
:10C4C00000D01F92CDB7DEB75C017A8369834A0141
:10C4D000170107FD05C0802F002E000C990B02C02C
:10C4E00081E090E0F90140805180628073809C017E
:10C4F000220F331F220F331F3C832B83265E384FBE
:10C500007901A3019201F701608171818281938198
:10C510000E9417DA882391F0F701408251826282EB
:10C52000738211E020E030E0A901C301B2010E9452
:10C5300054E018160CF010E0F5011083F50180812D
:10C540008230D1F0833009F45CC0813009F07BC0C7
:10C55000EB81FC81E65EF84F20813181428153817D
:10C56000F40160817181828193810E9417DA87FDD5
:10C570006AC082E0F50180832B813C81265E384FC2
:10C580007901B60180E090E00E941BDA9B01AC01CA
:10C59000F70160817181828193810E942DDE9B0170
:10C5A000AC01F40160817181828193810E9454E029
:10C5B00087FD15C067DF6B017C019101A8EEB3E038
:10C5C0000E941EDEDC01CB018C0D9D1DAE1DBF1D2A
:10C5D000E981FA8180839183A283B38334C052DFDF
:10C5E000E981FA81C080D180E280F380DC01CB0157
:10C5F0008C199D09AE09BF09B7FD25C083E0F5017F
:10C6000080830F3F19F047EE5EE102C04AEF5EE122
:10C610006EE07FE1802F0F900F900F900F90DF91D1
:10C62000CF911F910F91FF90EF90DF90CF90BF902F
:10C63000AF909F908F907F906F905F904F903F90C2
:10C640002F900C942A480F900F900F900F90DF912D
:10C65000CF911F910F91FF90EF90DF90CF90BF90FF
:10C66000AF909F908F907F906F905F904F903F9092
:10C670002F9008951F920F920FB60F9211242F93AF
:10C680003F938F939F93AF93BF9380913707909180
:10C690003807A0913907B0913A073091360723E067
:10C6A000230F2D3720F40196A11DB11D05C026E8EA
:10C6B000230F0296A11DB11D2093360780933707E3
:10C6C00090933807A0933907B0933A0780913B07BE
:10C6D00090913C07A0913D07B0913E070196A11DA6
:10C6E000B11D80933B0790933C07A0933D07B09307
:10C6F0003E07BF91AF919F918F913F912F910F90E6
:10C700000FBE0F901F9018954F925F926F927F927D
:10C710008F929F92AF92BF92CF92DF92EF92FF9251
:10C720000F931F93CF93DF933C01B0E2A0E06A2FF9
:10C7300070E0AB014B0F511D559547954A1711F00D
:10C740004B130BC0E2EAFDE165917491072E000CDA
:10C75000880B990B0E941DDA62C0CA010197880FED
:10C76000991F880F991FFC01EC5DF24E0591149101
:10C770009A01220F331F220F331FF901EC5DF24E95
:10C78000C591D4916016710614F4B42FD2CFA42FA2
:10C79000C615D7050CF4CBCF8A5D924EFC01E5900F
:10C7A000F490F901EA5DF24EC590D490B7010F2CD8
:10C7B000000C880B990B0E941DDA4B015C01B30140
:10C7C000601B710B072E000C880B990B0E941DDA61
:10C7D0002B013C01B6016E197F09072E000C880B56
:10C7E000990B0E941DDA9B01AC01C301B2010E94AA
:10C7F0007CDA6B017C01C01BD10BBE01DD0F880B05
:10C80000990B0E941DDA9B01AC01C701B6010E9481
:10C810000ADF9B01AC01C501B4010E942EDEDF914D
:10C82000CF911F910F91FF90EF90DF90CF90BF902D
:10C83000AF909F908F907F906F905F904F900895F2
:10C840000F931F93CF93DF93CDB7DEB72C970FB61F
:10C85000F894DEBF0FBECDBF6091340770913507ED
:10C86000072E000C880B990B0E941DDA9B01AC016E
:10C870008091240490912504BC01990F880B990B99
:10C8800029873A874B875C870E941DDA6D837E83F8
:10C890008F8398878091260490912704A091280483
:10C8A000B091290489839A83AB83BC830DEF2985DA
:10C8B0003A854B855C85BE016B5F7F4FCE0101964B
:10C8C00098DD6091320770913307072E000C880BBA
:10C8D000990B0E941DDA9B01AC0180911E0490917E
:10C8E0001F04BC01990F880B990B29873A874B8746
:10C8F0005C870E941DDA6D837E838F839887809189
:10C90000200490912104A0912204B09123048983F2
:10C910009A83AB83BC830FEF29853A854B855C8571
:10C92000BE016B5F7F4FCE01019663DDEBE9FFE156
:10C9300084918F010F5F1F4F882321F00E9418966A
:10C94000F801F6CFE091FF06F0E0E350F94F608187
:10C9500070E080E090E00E948896E6E9FFE1849133
:10C960008F010F5F1F4F882321F00E941896F80156
:10C97000F6CF6091FE0670E080E090E00E9488961D
:10C980002C960FB6F894DEBF0FBECDBFDF91CF91CE
:10C990001F910F910895EF92FF920F931F93CF93E2
:10C9A000DF93809136028F37A0F08F579091FD066C
:10C9B00090933107992311F02C9A01C02C98209163
:10C9C000FE062093300790910201222369F0909592
:10C9D0000BC090913107891708F02C98909130077F
:10C9E000891728F0909102019072909300018F5F57
:10C9F0008093360290912F0781E0892780932F073B
:10CA00008091350285301CF4C1E0C80F01C0C0E040
:10CA1000823009F4B1C054F4882301F1813009F067
:10CA2000E0C088E080937B0085E4BDC0843009F4D9
:10CA3000C2C00CF4B4C0853009F0D3C090912E0769
:10CA4000911102C080932E0780912E078150809310
:10CA50002E07882309F4C5C0C5E0C3C08091340205
:10CA60008F5F80311CF480933402BBC0109234027B
:10CA70008091FA06811113C08091240790912507B7
:10CA80009093350780933407809122079091230774
:10CA9000909333078093320781E08093FA068AE00F
:10CAA000E4E2F7E0DF011D928A95E9F7109223078F
:10CAB00010922207009134071091350711950195C6
:10CAC0001109D1E08091FD06811101C0D0E0809173
:10CAD00034049091350491958195910980179107BF
:10CAE0004CF4DD2339F04EE15FE16FE37FE180E05C
:10CAF0000E942A48809106029091070291958195A3
:10CB00009109081719074CF4DD2339F041E55FE17D
:10CB100062E77FE180E00E942A4811E080911E04D4
:10CB200090911F04181619060CF010E0E0903207DF
:10CB3000F090330780913204909133048E159F0555
:10CB40004CF0112339F04EE25FE16FE37FE18FEFAC
:10CB50000E942A488091040290910502E816F90685
:10CB60000CF43FC01123E9F141E65FE162E77FE1A8
:10CB70008FEF0E942A4835C080917A0086FD2EC032
:10CB800080917800909179002091240730912507B9
:10CB9000820F931F909325078093240722C088E07B
:10CBA00080937B0086E480937C0080917A0080648F
:10CBB00080937A0016C080917A0086FD11C0809122
:10CBC0007800909179002091220730912307820FFD
:10CBD000931F909323078093220703C0C2E001C0F4
:10CBE000C4E0C09335020E9400C78091FB0690917B
:10CBF000FC060097A9F001979093FC068093FB0632
:10CC0000892B71F484E89FE190931C0880931B08A2
:10CC1000DF91CF911F910F91FF90EF900C94C16F16
:10CC2000DF91CF911F910F91FF90EF9008950F9397
:10CC30000FB70F9300916E000B7F00936E007894F6
:10CC40000F930BB70F930CB70F921F922F933F9335
:10CC50004F935F936F937F938F939F93AF93BF9304
:10CC6000EF93FF93112497DEFF91EF91BF91AF9166
:10CC70009F918F917F916F915F914F913F912F91F4
:10CC80001F900F900CBF0F910BBF0F910460F89491
:10CC900000936E000F910FBF0F911895CF92DF9206
:10CCA000EF92FF92C0902004D0902104E0902204E3
:10CCB000F090230480911E0490911F040697BC01FC
:10CCC000990F880B990B0E941DDA9B01AC01C701DB
:10CCD000B6010E9417DA87FF1EC020E030E040E076
:10CCE00050E4C701B6010E942EDE0E9477DF7093E8
:10CCF000190760931807C6DBDC01CB01805A954108
:10CD0000AF4FBF4F8093140790931507A09316075A
:10CD1000B093170708C010921407109215071092CD
:10CD2000160710921707FF90EF90DF90CF900895AD
:10CD3000CF92DF92EF92FF92C0902604D09027040A
:10CD4000E0902804F0902904809124049091250417
:10CD50000697BC01990F880B990B0E941DDA9B0165
:10CD6000AC01C701B6010E9417DA87FF1EC020E0A0
:10CD700030E040E050E4C701B6010E942EDE0E9480
:10CD800077DF70931307609312077CDBDC01CB0124
:10CD9000805E914BAF4FBF4F80930E0790930F076C
:10CDA000A0931007B093110708C010920E071092BD
:10CDB0000F071092100710921107FF90EF90DF906D
:10CDC000CF9008951092F906109225041092240431
:10CDD00080E0AEDF10921F0410921E045FDF0E94FD
:10CDE0008449109225041092240480E0A1DF10925F
:10CDF000FD062C9810921F0410921E041092FE063D
:10CE00008091020180728093000108954F925F9299
:10CE10006F927F928F929F92AF92BF92CF92DF924A
:10CE2000EF92FF920F931F93CF93DF933C01B0E4F7
:10CE3000A0E06A2F70E0AB014B0F511D559547954F
:10CE40004A1711F04B130BC0E5EEFEE165917491AA
:10CE5000072E000C880B990B0E941DDA62C0CA01D4
:10CE60000197880F991F880F991FFC01E951F24E15
:10CE7000059114919A01220F331F220F331FF901DC
:10CE8000E951F24EC591D4916016710614F4B42F95
:10CE9000D2CFA42FC615D7050CF4CBCF8751924E15
:10CEA000FC01E590F490F901E751F24EC590D49061
:10CEB000B7010F2C000C880B990B0E941DDA4B0157
:10CEC0005C01B301601B710B072E000C880B990BE2
:10CED0000E941DDA2B013C01B6016E197F09072E55
:10CEE000000C880B990B0E941DDA9B01AC01C30159
:10CEF000B2010E947CDA6B017C01C01BD10BBE0128
:10CF0000DD0F880B990B0E941DDA9B01AC01C70154
:10CF1000B6010E940ADF9B01AC01C501B4010E9469
:10CF20002EDEDF91CF911F910F91FF90EF90DF9058
:10CF3000CF90BF90AF909F908F907F906F905F90B9
:10CF40004F90089560E08091340790913507DCDBC5
:10CF500060932604709327048093280490932904F7
:10CF6000809132079091330751DF609320047093D2
:10CF700021048093220490932304A8951092FA062A
:10CF800008958F929F92AF92BF92CF92DF92EF92CD
:10CF9000FF920F93CF93DF9300D01F92CDB7DEB7F0
:10CFA0008091FA06811110C00F900F900F900F9092
:10CFB000DF91CF910F91FF90EF90DF90CF90BF90D6
:10CFC000AF909F908F900895BDDF5CDA4B015C01BC
:10CFD0006091240470912504072E000C880B990B96
:10CFE0000E941DDA69837A838B839C8338E0C32E89
:10CFF000D12C4CE3E42EF12C00E09E012F5F3F4F3B
:10D0000046E254E06AE077E089E097E047DAC090D2
:10D010002604D0902704E0902804F0902904809101
:10D02000360490913704BC01990F880B990B0E942C
:10D030001DDA9B01AC01C701B6010E9454E018162D
:10D04000D4F46091080270910902072E000C880B3D
:10D05000990B0E941DDA9B01AC01C701B6010E9429
:10D0600017DA87FF08C080E00E94D4460E9472DF72
:10D070007595679501C060E06093FD0680910E078D
:10D0800090910F07A0911007B09111070097A1058B
:10D09000B10529F1A5019401281B390B4A0B5B0B43
:10D0A00057FD1DC0609112077091130780E090E05A
:10D0B0000E941BDA9B01AC01609126047091270449
:10D0C00080912804909129040E9417DA87FFD3C029
:10D0D00046EC5DE168ED7DE180E00E942A488091A8
:10D0E000F5069091F606A091F706B091F806A50115
:10D0F0009401281B390B4A0B5B0B57FD10C00E9493
:10D100009748D501C4018C53964FAF4FBF4F8093C2
:10D11000F5069093F606A093F706B093F806809173
:10D12000140790911507A0911607B0911707009763
:10D13000A105B10529F1A5019401281B390B4A0B62
:10D140005B0B57FD1DC0609118077091190780E0B7
:10D1500090E00E941BDA9B01AC0160912004709169
:10D16000210480912204909123040E9417DA87FF02
:10D170007EC044EA5DE167EB7DE18FEF0E942A48C3
:10D180008091050790910607A0910707B0910807C5
:10D19000A5019401281B390B4A0B5B0B57FD04CFEB
:10D1A00038E8830E33E1931EA11CB11C8092050761
:10D1B00090920607A0920707B092080760911E049C
:10D1C00070911F04072E000C880B990B0E941DDA2A
:10D1D00069837A838B839C8382E0C82ED12C94E16F
:10D1E000E92EF12C0FEF9E012F5F3F4F40E254E0FC
:10D1F00060E077E084E097E051D9C0902004D090BF
:10D200002104E0902204F090230420E030E040EA82
:10D2100050E4C701B6010E9454E087FD20C020E021
:10D2200030E04CED52E4C701B6010E9417DA18163F
:10D23000B4F060911E0470911F04072E000C880B3F
:10D24000990B0E941DDA9B01AC01C701B6010E9437
:10D2500017DA87FD0EC080E08093FE06A5CE1092FF
:10D26000FE06809102018072809300019DCE16DD42
:10D2700087CF8FE7F1CF80E05BDD31CFCF92DF92B8
:10D28000EF92FF926B017C0183E3C816D104E104A5
:10D29000F10460F082E3C81AD108E108F10862E302
:10D2A00070E080E090E06DD86CDEEECFC701B60193
:10D2B00068D8FF90EF90DF90CF9063CE909172107E
:10D2C000E92FF0E0EE5AFB4F80839F5F943018F413
:10D2D0009093721002C010927210809173108F5F41
:10D2E000809373100895CF92DF92EF920F931F9364
:10D2F000CF93DF93CDB7DEB760970FB6F894DEBF5C
:10D300000FBECDBFE0908A06ECE0F4E08085918509
:10D31000A285B38544815581668177810081118121
:10D320002281338109831A832B833C834D835E835F
:10D330006F83788789879A87AB87BC871D861E860F
:10D340001F86188AAE01475F5F4FBE016B5F7F4F3C
:10D35000CE0101960E94C684CE010D966C0102E4B6
:10D3600012E028E134E0AE01475F5F4FBE016B5F22
:10D370007F4F0C970E942A7460960FB6F894DEBF18
:10D380000FBECDBFDF91CF911F910F91EF90DF9036
:10D39000CF900895CF93FC0180818B33A1F08091D1
:10D3A0007310843080F4C62FBF018091721020E684
:10D3B000829FC0011124895A9B4F0E949CE18C2FAF
:10D3C0007DDF81E001C080E0CF9108952F923F92F0
:10D3D0004F925F926F927F928F929F92AF92BF9285
:10D3E000CF92DF92EF92FF920F931F93CF93DF9331
:10D3F00000D000D0CDB7DEB78C0144D8F801C6808C
:10D40000D780E084F184C114D104E104F10409F06F
:10D41000F6C22485222309F460C332852150248773
:10D4200021E0230F22874585241301C01286F801CD
:10D4300024E0329FE00DF11D1124C684D784E088DA
:10D44000F188F801C282D382E482F582DC01CB014B
:10D450008C0D9D1DA11DB11D86839783A087B1876B
:10D4600084819581892B09F438C3FFB7FD83F89433
:10D47000F8012280338004811581809103028F316D
:10D4800021F08F3F09F0B8C205C0E3E4F1E1249137
:10D490002E83EDC08FE180930302E3E4F1E1E49198
:10D4A000EF3F09F4A9C2E23009F474C054F5EE2349
:10D4B00009F453C0E13009F0D9C0109280001092F5
:10D4C000810080918100886080938100809181003B
:10D4D000816080938100ECE0F0E2E491F0E0EE0FF7
:10D4E000FF1FE754F04E8591949190934C078093E1
:10D4F0004B07E2E5F0E2E491E0934A0781E08E8396
:10D50000B9C0E43009F48EC00CF468C0E53009F00D
:10D51000ADC01092200110922101809121018860FC
:10D520008093210180912101816080932101ECE0B1
:10D53000F0E2E491F0E0EE0FFF1FE754F04E85912A
:10D5400094919093430780934207E2E5F0E2E491DF
:10D55000E093410725E02E838DC014BC15BC84B533
:10D56000826084BD85B5816085BDECE0F0E2E49128
:10D57000F0E0EE0FFF1FE754F04E859194919093E9
:10D580004F0780934E07E2E5F0E2E491E0934D0708
:10D590001E8270C01092B0001092B1008091B00055
:10D5A00082608093B0008091B10081608093B1006F
:10D5B000ECE0F0E2E491F0E0EE0FFF1FE754F04EF4
:10D5C0008591949190932B0480932A04E2E5F0E2F4
:10D5D000E491E0932C0492E09E834CC01092900062
:10D5E00010929100809191008860809391008091C9
:10D5F0009100816080939100ECE0F0E2E491F0E032
:10D60000EE0FFF1FE754F04E8591949190934907D8
:10D6100080934807E2E5F0E2E491E0934707E3E016
:10D62000EE8328C01092A0001092A1008091A1006A
:10D6300088608093A1008091A10081608093A10007
:10D64000ECE0F0E2E491F0E0EE0FFF1FE754F04E63
:10D65000859194919093460780934507E2E5F0E227
:10D66000E491E0934407F4E0FE8304C0EE838E81EE
:10D6700087FDC2C12101612C712C61E08FE10E9404
:10D68000BE604801A12CB12C8E818D7F09F0BDC0F8
:10D6900060E072E18AE790E0A50194010E941DE13B
:10D6A00029833A834B835C8369017A0191E0C91A2B
:10D6B000D108E108F108EFEFCE16D104E104F1043E
:10D6C00009F008F44DC060E472E48FE090E0A50139
:10D6D00094010E941DE169017A01F1E0CF1AD1089D
:10D6E000E108F1082E81223001F58FEFC816D10430
:10D6F000E104F10409F008F4EEC160E970ED83E0A3
:10D7000090E0A50194010E941DE169017A0191E078
:10D71000C91AD108E108F108EFEFCE16D104E104EF
:10D72000F10409F0E0F583E069C0FFEFCF16D10402
:10D73000E104F104B9F0B0F068E478EE81E090E043
:10D74000A50194010E941DE169017A0181E0C81AD6
:10D75000D108E108F1089E81992309F49AC190C18A
:10D7600081E001C082E09E819923A1F047C08981B8
:10D770009A81AB81BC812AE0B595A795979587954D
:10D780002A95D1F76C017D01E1E0CE1AD108E108BC
:10D79000F10885E095B5987F892B85BDA1C068E427
:10D7A00078EE81E090E0A50194010E941DE16901FD
:10D7B0007A01F1E0CF1AD108E108F1082FEFC21683
:10D7C000D104E104F10409F008F428C164E274EF23
:10D7D00080E090E0A50194010E941DE169017A01B9
:10D7E000E1E0CE1AD108E108F108FFEFCF16D1042D
:10D7F000E104F10411F008F013C185E09091B1004B
:10D80000987F892B8093B1006BC060E072E18AE75A
:10D8100090E0A50194010E941DE169017A01E1E017
:10D82000CE1AD108E108F108C114D104F1E0EF06E5
:10D83000F10488F068E478EE81E090E0A5019401BD
:10D840000E941DE169017A0181E0C81AD108E1084E
:10D85000F10883E001C081E09E81913071F49091E4
:10D860008100987F892B809381004528462847288E
:10D87000D9F52FEF3FEFA90168C0EE81E33071F4D5
:10D8800090919100987F892B80939100452846289C
:10D89000472851F52FEF3FEFA90179C0FE81F43001
:10D8A00071F49091A100987F892B8093A100452865
:10D8B00046284728C9F42FEF3FEFA9017AC02E81EF
:10D8C000253071F490912101987F892B809321015B
:10D8D00045284628472841F42FEF3FEFA9017BC098
:10D8E00045284628472869F09801220F331FD101A7
:10D8F0000E941EDE28EE33E040E050E00E94F2DDA0
:10D9000003C02FEF3FEFA9018E81823081F12CF40B
:10D91000882361F08130C9F06FC09E81943009F492
:10D9200048C0ACF1953009F456C066C0C7BC20931E
:10D9300060073093610740936207509363078091BB
:10D940006E00826080936E0057C0D0928900C092B2
:10D95000880020935C0730935D0740935E075093E7
:10D960005F0780916F00826080936F0045C0C09216
:10D97000B30020932D0430932E0440932F04509332
:10D9800030048091700082608093700035C0D09226
:10D990009900C092980020935807309359074093FC
:10D9A0005A0750935B0780917100826080937100E9
:10D9B00023C0D092A900C092A800209354073093AE
:10D9C0005507409356075093570780917200826025
:10D9D0008093720011C0D0922901C0922801209337
:10D9E000500730935107409352075093530780914B
:10D9F0007300826080937300ED81EFBF6EC0DC0125
:10DA0000CB018C199D09AE09BF09B7FD66C04698C8
:10DA1000F80116821782108611865FC084E0EECE70
:10DA200062E17AE780E090E0A50194010E941DE1A7
:10DA300069017A0181E0C81AD108E108F1089FEF75
:10DA4000C916D104E104F104C9F0C0F089819A81BA
:10DA5000AB81BC815AE0B595A795979587955A9566
:10DA6000D1F76C017D0121E0C21AD108E108F1086B
:10DA70008E81882309F48DCE87E0C0CE86E073CEF8
:10DA8000EFEFCE16D104E104F10409F048F684E08A
:10DA90006ACE8FEFC816D104E104F104D1F0C8F0CA
:10DAA00062E17AE780E090E0A50194010E941DE127
:10DAB00069017A01F1E0CF1AD108E108F1082FEFEE
:10DAC000C216D104E104F10411F008F050CE84E054
:10DAD00061CE83E05FCE82E091CE26960FB6F894B9
:10DAE000DEBF0FBECDBFDF91CF911F910F91FF9091
:10DAF000EF90DF90CF90BF90AF909F908F907F90EE
:10DB00006F905F904F903F902F9008958091CD0738
:10DB10009091CE07A091CF07B091D0078093420299
:10DB200090934302A0934402B09345028091CB07A7
:10DB30009091CC0790930202809301020895809106
:10DB4000420290914302A0914402B0914502809319
:10DB5000CD079093CE07A093CF07B093D0078091C5
:10DB60000102909102029093CC078093CB0784E648
:10DB700090E0909302028093010208954F925F9289
:10DB80006F927F928F929F92AF92BF92CF92DF92CD
:10DB9000EF92FF920F931F93CF93DF93CDB7DEB732
:10DBA0002C970FB6F894DEBF0FBECDBF6D837E837A
:10DBB0008F83988729873A874B875C87470158016D
:10DBC00036018091420290914302A0914402B091AB
:10DBD000450289839A83AB83BC83D601CD90DD90C7
:10DBE000ED90FC9020E030E0A901C701B6010E9451
:10DBF00017DA811106C0ECEDFCE1C590D590E590F7
:10DC0000F490A50194016091140470911504809121
:10DC10001604909117040E9417DA87FF11C0C09272
:10DC20004202D0924302E0924402F0924502809276
:10DC3000140490921504A0921604B092170453DBBA
:10DC4000F301408051806280738020E030E0A901C0
:10DC5000C301B2010E9417DA811108C040903E0250
:10DC600050903F0260904002709041024092420208
:10DC70005092430260924402709245028D819E81CF
:10DC8000AF81B88580930C0490930D04A0930E048B
:10DC9000B0930F0489859A85AB85BC858093100469
:10DCA00090931104A0931204B09313041CDBA501FC
:10DCB0009401609114047091150480911604909160
:10DCC00017040E9454E018168CF4C0924202D092BD
:10DCD0004302E0924402F092450280921404909232
:10DCE0001504A0921604B0921704FDDA0E94418434
:10DCF00089819A81AB81BC818093420290934302D7
:10DD0000A0934402B09345022C960FB6F894DEBF60
:10DD10000FBECDBFDF91CF911F910F91FF90EF907C
:10DD2000DF90CF90BF90AF909F908F907F906F903B
:10DD30005F904F900895CF92DF92EF92FF920F93F2
:10DD40001F936B01FC01E080F18002811381ECE004
:10DD5000F4E024813581468157816081718182811F
:10DD600093810CDF1F910F91FF90EF90DF90CF9088
:10DD70000895BF92CF92DF92EF92FF920F931F937D
:10DD8000CF93DF93CDB7DEB728970FB6F894DEBFF9
:10DD90000FBECDBF90914504981709F479C0B82EF5
:10DDA000882309F453C080E090E0A0E2B1E48D83C1
:10DDB0009E83AF83B887C0900704D0900804E0909A
:10DDC0000904F0900A0420E030E0A901C701B6017F
:10DDD0000E9417DA87FF0CC0A701960160E070E08F
:10DDE00080E291E40E942DDE6D837E838F8398878D
:10DDF00020E030E04DE453E46D817E818F81988591
:10DE00000E9454E0181644F480E090E0ADE4B3E4DE
:10DE10008D839E83AF83B8872091140430911504BD
:10DE200040911604509117046D817E818F819885F1
:10DE30000E9454E0181654F419821A821B821C8224
:10DE4000BE016F5F7F4FCE01059675DF60910C04B8
:10DE500070910D0480910E0490910F042091100494
:10DE600030911104409112045091130419821A82C6
:10DE70001B821C82E0901404F0901504009116049B
:10DE800010911704FE0131966F0178DEB0924504BF
:10DE900080E028960FB6F894DEBF0FBECDBFDF91AD
:10DEA000CF911F910F91FF90EF90DF90CF90BF9097
:10DEB00008950F931F93CF93DF9394E0899FE00120
:10DEC00011248E01095A1F4EFE01EA5BFB4FDE0151
:10DED000A756B94F2D913D914D915C916081718113
:10DEE000828193810E942EDEF80160837183828398
:10DEF0009383FE01EF5CFD4D85919591A591B491C1
:10DF0000FE01EB55F94F80839183A283B383FE0119
:10DF1000E35CFD4D85919591A591B491C85DDD4F70
:10DF200088839983AA83BB83DF91CF911F910F913F
:10DF30000895EF92FF921F93CF93DF937C0160E0EF
:10DF400029DA182F8823B1F0EEECF3E28491EF0187
:10DF50002196882321F00E941896FE01F7CFB70181
:10DF60008FEB90E20E94D0C882E20E9418968AE06D
:10DF70000E941896812FDF91CF911F91FF90EF9013
:10DF80000895DF92EF92FF920F931F93CF93DF9349
:10DF9000CDB7DEB76E970FB6F894DEBF0FBECDBF1C
:10DFA00060911B0870911C086115710541F14DE1EC
:10DFB00050E0CE0101967C010E94BFD91E8EF70170
:10DFC0008F010E191F09D190DD2019F09AE0D912A6
:10DFD000F7CFF701E00FF11F1082C701AADF8823F6
:10DFE00071F0DD20A9F00F5F1F4F80911B08909109
:10DFF0001C08080F191F10931C0800931B0881E0D0
:10E0000020911B0830911C08232B29F480E003C0C9
:10E0100000E010E0F0CF6E960FB6F894DEBF0FBEB2
:10E02000CDBFDF91CF911F910F91FF90EF90DF90C7
:10E0300008954F925F926F927F929F92AF92BF929C
:10E04000CF92DF92EF92FF920F931F93CF93DF93C4
:10E050001F92CDB7DEB795DF811165C28091731035
:10E06000843028F40E941397AC0197FF39C1809146
:10E07000810A882309F457C280917310811102C06C
:10E080001092CA07EE24E3944091FA0C5091FB0CD5
:10E090006091FC0C7091FD0C8091F60C9091F70C46
:10E0A000A091F80CB091F90C481759076A077B0743
:10E0B00008F4E12C00E010E0BB24B39480E6A82E25
:10E0C00097EFC92E91E2D92E2DE8922E80917310F0
:10E0D000843008F028C2E11026C28091CA0781115D
:10E0E00022C28091510C9091520CA091530CB0918E
:10E0F000540C8093FA0C9093FB0CA093FC0CB093FF
:10E10000FD0C41E050E0BE016F5F7F4F89E49CE071
:10E110000E945B9E019719F4898190E002C08FEF05
:10E120009FEFF82EEE24E3944090FA0C5090FB0CF5
:10E130006090FC0C7090FD0C4091F60C5091F70C27
:10E140006091F80C7091F90C441655066606770636
:10E15000C8F4E12C8F3FFFEF9F0709F46BC02AE062
:10E16000821709F48CC08DE0F81609F488C093E298
:10E17000F91619F0EAE3FE1299C08091C9078111DE
:10E1800095C072C00E94418489E49CE00E940E9C6C
:10E190008091640C882359F181508093640C989E7F
:10E1A000C001112441E061E08759934F0E94DBBC1C
:10E1B000E091640C24E0E29FF0011124EB59F34F4D
:10E1C00040815181628173814093FA0C5093FB0C22
:10E1D0006093FC0C7093FD0C89E49CE00E949CB958
:10E1E0008091820A8823A9F0B092810A12C010920D
:10E1F000810A0E9451840E9484490E9402496D3321
:10E2000071058105910528F0D0921C08C0921B0869
:10E21000B8DE8091810A81112BC0EAE0F2E284919C
:10E220003F019FEF691A790A8823F1F00E9418963E
:10E23000F301F5CFE9EBF3E284913F012FEF621A8E
:10E24000720A882321F00E941896F301F5CFEBEFB4
:10E25000F1E284913F019FEF691A790A882321F046
:10E260000E941896F301F5CFE3E2FE1208C005C044
:10E2700023E2F21255C100E010E0B092CA071092FA
:10E28000C9070115110519F40E94C1670CC08091DE
:10E290007210A89E000D111D1124F801E95AFB4FC0
:10E2A000108280E00BD800E010E010CF0F35110590
:10E2B00008F00CCFFBE3FF1202C0B092C9078091B7
:10E2C000C907811103CF80917210F801A89EE00D5B
:10E2D000F11D1124E95AFB4FF0820F5F1F4FF6CE5C
:10E2E000982F20913C1030913D108A3019F09D30CC
:10E2F00009F0E4C01092C8072115310519F40E94F5
:10E30000C167ACCEF901E859F84F108210923D1068
:10E3100010923C1028E637E08901F90180812F5FD7
:10E320003F4F8032C9F378018E3409F07CC001156B
:10E33000110509F478C062EF71E2C8010E94CED9DC
:10E34000DD24D394892B11F4D12C09C06EE470E044
:10E35000C80104960E9488E1009709F08C014AE008
:10E3600050E060E070E0C80101960E9443D76093DE
:10E370006407709365078093660790936707009121
:10E380003E1010913F1020914010309141100F5FCE
:10E390001F4F2F4F3F4F601771078207930729F0D8
:10E3A000D11003C08FEB91E22AC06AE270E0C7018E
:10E3B0000E94C0E19C01009701F1982F9E1910E086
:10E3C000992339F09150F701E90FF11D8081182749
:10E3D000F7CF4AE050E060E070E0C90101960E948A
:10E3E00043D7012F10E020E030E06017710782076B
:10E3F000930741F080EA91E202C086E791E20E9431
:10E4000078BE35CE8091640790916507A09166072C
:10E41000B091670780933E1090933F10A0934010F7
:10E42000B093411007C080917F0A882319F08CECCB
:10E4300090E2E5CF8091170281111DC067E470E082
:10E44000C7010E9488E10097B1F04AE050E060E027
:10E4500070E001960E9443D76430710560F4EFEFDD
:10E46000F0E284918F010F5F1F4F882321F00E94FB
:10E470001896F801F6CF6AE873E0C7010E9493E1AD
:10E48000892B11F4109200026FE873E0C7010E941B
:10E4900093E1892B21F486EF90E20E94775564E99D
:10E4A00073E0C7010E9493E1892B11F40E940DA330
:10E4B00061E088E697E00E94CA69D0CD2F3531052A
:10E4C0000CF0CCCD9C35C1F40E94139797FDC6CDBE
:10E4D0002091C8072111C2CD20913C1030913D10F0
:10E4E000A9014F5F5F4F50933D1040933C10F901DD
:10E4F000E859F84F8083B2CD9B3319F481E08093C3
:10E50000C8078091C8078111A9CDC90101969093D0
:10E510003D1080933C10F901E859F84F40839ECD9F
:10E520001092C907B1CE0F90DF91CF911F910F913B
:10E53000FF90EF90DF90CF90BF90AF909F907F9033
:10E540006F905F904F9008950F931F93CF93DF9339
:10E55000CDB7DEB72C970FB6F894DEBF0FBECDBF98
:10E56000ECE0F4E080859185A285B38544815581F6
:10E5700066817781008111812281338109831A8329
:10E580002B833C834D835E836F83788789879A874B
:10E59000AB87BC87AE01475F5F4FBE016B5F7F4FAC
:10E5A000CE0101960E94C68428E134E0AE01475FA7
:10E5B0005F4FBE016B5F7F4FCE0101960E9492C9F3
:10E5C0002C960FB6F894DEBF0FBECDBFDF91CF9172
:10E5D0001F910F9108951F93CF93DF93CDB7DEB7AF
:10E5E0002C970FB6F894DEBF0FBECDBF882331F055
:10E5F0002091101030911110232B91F190916C10FB
:10E60000891771F1182F8CE0E3E6F2E0DE01119634
:10E6100001900D928A95E1F7CE0101960E94A55DC9
:10E6200010936C10111117C00E94685D8EE796E080
:10E630000E948F848091860690918706A09188061B
:10E64000B09189068093140490931504A093160446
:10E65000B093170404C08CE094E00E948F8474DFB0
:10E660002C960FB6F894DEBF0FBECDBFDF91CF91D1
:10E670001F91089580E0AFDFE0E1F0E113821282A4
:10E6800011821082E4E1F8E013821282118210827A
:10E69000E8E1F0E180E090E0A0ECBFE780839183C7
:10E6A000A283B38384839583A683B783808791876E
:10E6B000A287B38784879587A687B787808B918B3E
:10E6C000A28BB38B848B958BA68BB78B808F918F0E
:10E6D000A28FB38F848F958FA68FB78F80A391A3BE
:10E6E000A2A3B3A308951F93CF93DF93CDB7DEB753
:10E6F00028970FB6F894DEBF0FBECDBF69837A832B
:10E700008B839C832D833E834F835887BE016B5F31
:10E710007F4FCE0101960FDB1091560410925604E4
:10E720000E94685D8EE796E00E948F848091860645
:10E7300090918706A0918806B09189068093140471
:10E7400090931504A0931604B0931704FDDE13FBF9
:10E75000112710F981E0812728960FB6F894DEBFC3
:10E760000FBECDBFDF91CF911F9108950E94C89732
:10E7700097FD0CC00E94C8976F3F710581059105F8
:10E7800009F034F40E94C897862F089580E0089518
:10E790008FEF0895EF92FF920F931F93CF93DF9324
:10E7A0007C0184E50E941F98D82F882341F1DEDF89
:10E7B000C82F181604F5EEECF3E284918F010F5F79
:10E7C0001F4F882321F00E941896F801F6CF8DE4A0
:10E7D0000E941896B70180E090E04AE00E942296DD
:10E7E0006C2FCC0F770B8EE192E20E94B7C88AE0C3
:10E7F0000E94189608C08093FF06D0E004C0809164
:10E800008A068093FF068D2FDF91CF911F910F9184
:10E81000FF90EF90089580913F0790914007892BDA
:10E8200031F0A4DF91E0811103C090E001C091E0DC
:10E83000892F089580913F0790914007009731F00C
:10E840004AE050E060E070E00C946BD860E070E06B
:10E85000CB0108952F923F924F925F926F927F92D9
:10E860008F929F92AF92BF92CF92DF92EF92FF92E0
:10E870000F931F93CF93DF93CDB7DEB7C957D1095D
:10E880000FB6F894DEBF0FBECDBFE091FB06F0914E
:10E89000FC06EF2B09F09FC72896DFAECEAE289777
:10E8A0002E2C79016A015B01FC01208131814281BA
:10E8B0005381A4962CAF3DAF4EAF5FAFA49720918C
:10E8C000B1103091B2104091B3105091B410A49691
:10E8D0006CAD7DAD8EAD9FADA4970E947CDA0E9499
:10E8E0005FE0E0966CAF7DAF8EAF9FAFE097D50154
:10E8F0008D919D910D90BC91A02DA8968CAF9DAF50
:10E90000AEAFBFAFA8972091B5103091B61040912F
:10E91000B7105091B810BC01CD010E947CDA0E9462
:10E920005FE0E4966CAF7DAF8EAF9FAFE497D6010A
:10E930002D913D914D915C91AC962CAF3DAF4EAF7A
:10E940005FAFAC972091B9103091BA104091BB10D5
:10E950005091BC10AC966CAD7DAD8EAD9FADAC97BB
:10E960000E947CDA0E945FE0E8966CAF7DAF8EAFCC
:10E970009FAFE897D7012D913D914D915C912296E3
:10E980002CAF3DAF4EAF5FAF22972091BD103091BD
:10E99000BE104091BF105091C01022966CAD7DAD5D
:10E9A0008EAD9FAD22970E947CDA0E945FE0609658
:10E9B0006CAF7DAF8EAF9FAF609780910E0883FFE5
:10E9C0001CC060962CAD3DAD4EAD5FAD6097209301
:10E9D0005D0A30935E0A40935F0A5093600A229664
:10E9E0008CAD9DADAEADBFAD229780934D0A909397
:10E9F0004E0AA0934F0AB093500AD801BC91BDA310
:10EA0000F801F181F9ABD8011296BC91BAABF801CB
:10EA1000F381FAAF80912B0A90912C0A891B8F7099
:10EA20008F3019F40E94C955F5CF00912B0AE99651
:10EA30000FAFE99780912B0A082F10E01CA30BA3BE
:10EA40008091510A9091520AA091530AB091540AB0
:10EA5000E0964CAC5DAC6EAC7FACE097481A590ABE
:10EA60006A0A7B0A8091550A9091560AA091570A2A
:10EA7000B091580AE4968CAC9DACAEACBFACE497B8
:10EA8000881A990AAA0ABB0A8091590A90915A0ACF
:10EA9000A0915B0AB0915C0AE8962CAD3DAD4EADFD
:10EAA0005FADE897281B390B4A0B5B0B2DA73EA7E0
:10EAB0004FA758AB80915D0A90915E0AA0915F0AC2
:10EAC000B091600A60960CAD1DAD2EAD3FAD609764
:10EAD000081B190B2A0B3B0B09A71AA72BA73CA74E
:10EAE000012B022B032B09F4BAC06091260470910C
:10EAF0002704809128049091290420910D08211168
:10EB000041C00E9472DF20913B0230913C026217AB
:10EB10007307C4F560962CAD3DAD4EAD5FAD60970B
:10EB200020935D0A30935E0A40935F0A5093600A17
:10EB300022968CAD9DADAEADBFAD229780934D0AB0
:10EB400090934E0AA0934F0AB093500AEEECF3E272
:10EB500084918F010F5F1F4F882321F00E94189628
:10EB6000F801F6CFE8E6F2E284918F010F5F1F4FC4
:10EB7000882321F00E941896F801F6CF19A61AA64C
:10EB80001BA61CA669A57AA58BA59CA50E941DDACB
:10EB9000A4E02A9EF0011124E95CFD4F208131811F
:10EBA000428153810E947CDA6B017C0120E030E0DD
:10EBB000A9010E9454E087FF04C0F7FAF094F7F827
:10EBC000F0946091BD107091BE108091BF10909133
:10EBD000C0100E9472DF9B01AC01A8ECB0E00E9463
:10EBE00014DE0E941DDA9B01AC01C701B6010E9430
:10EBF00054E01816C4F560960CAD1DAD2EAD3FADBA
:10EC0000609700935D0A10935E0A20935F0A309329
:10EC1000600A22962CAD3DAD4EAD5FAD229720939C
:10EC20004D0A30934E0A40934F0A5093500AEEEC2F
:10EC3000F3E284918F010F5F1F4F882321F00E9420
:10EC40001896F801F6CFE9E4F2E284918F010F5FA4
:10EC50001F4F882321F00E941896F801F6CF19A6BD
:10EC60001AA61BA61CA6D301C2018827B7FD83954F
:10EC70009927AA27BB27182FB7FC12608DA59EA540
:10EC8000AFA5B8A9B7FD146029A53AA54BA55CA509
:10EC900057FD186069A57AA58BA59CA50E941DDA71
:10ECA00034E0239EF0011124E95CFD4F2081318185
:10ECB000428153810E947CDA6B017C0120E030E0CC
:10ECC000A9010E9454E087FF04C0C701B601905813
:10ECD00002C0C701B60120E030E040E05FE30E94DF
:10ECE0002EDE0E9477DF6EAB7FAB88AF99AF88E5F1
:10ECF0004BA15CA1849FF001859FF00D1124EF537F
:10ED0000FF4E108216ABB301A20177FE07C0442765
:10ED10005527BA01441955096609770988E50BA1F9
:10ED20001CA1809FF001819FF00D1124EF53FF4E35
:10ED3000458B568B678B708F26968CAE9DAEAEAE94
:10ED4000BFAE2697B7FE0DC088279927DC0188192A
:10ED50009909AA09BB0926968CAF9DAFAEAFBFAF8C
:10ED6000269728E50BA11CA1209FF001219FF00D03
:10ED70001124EF53FF4E26968CAD9DADAEADBFADC9
:10ED80002697818F928FA38FB48F0DA51EA52FA5D7
:10ED900038A937FF07C030952095109501951F4F72
:10EDA0002F4F3F4FE8E53E2EABA1BCA13A9EF001AC
:10EDB0003B9EF00D1124EF53FF4E058F168F278FCA
:10EDC00030A38EA99FA9A8ADB9AD81A392A3A3A397
:10EDD000B4A326968CAD9DADAEADBFAD269784177E
:10EDE0009507A607B70710F4DB01CA018017910742
:10EDF000A207B30710F4D901C8010EA91FA928ADB5
:10EE000039AD80179107A207B30710F4D901C801E3
:10EE100028E50BA11CA1209FF001219FF00D1124DA
:10EE2000EF53FF4E85A396A3A7A3B0A70697A1050E
:10EE3000B10508F4C9C4DF01AE5ABF4F80911C046C
:10EE400090911D048D939C9321A6452B462B472B17
:10EE500009F05F9888E50BA11CA1809FF001819FBC
:10EE6000F00D1124EF53FF4E818D928DA38DB48D43
:10EE7000892B8A2B8B2B11F08A98479888E50BA158
:10EE80001CA1809FF001819FF00D1124EF53FF4ED4
:10EE9000858D968DA78DB0A1892B8A2B8B2B31F078
:10EEA0008091080181708093060147982EA93FA99F
:10EEB00048AD59AD232B242B252B09F48EC480910A
:10EEC0001308882319F0815080931308211004C07F
:10EED000129880E2809313082090090830900A0865
:10EEE00000910B0810910C089101A8016DA179A95E
:10EEF0008AA99AAD0E9417DA87FF04C02DA239AA09
:10EF00000AAB1AAFC301B2010E941DDA2091A11011
:10EF10003091A2104091A3105091A4100E947CDA6D
:10EF200026966CAF7DAF8EAF9FAF2697698B7A8B9D
:10EF30008B8B9C8BC501B4010E941DDA2091A5101A
:10EF40003091A6104091A7105091A8100E947CDA31
:10EF50002B013C016D8B7E8B8F8B988F6DA57EA5D1
:10EF60008FA598A90E941DDA2091A9103091AA10AE
:10EF70004091AB105091AC100E947CDA4B015C01C7
:10EF8000698F7A8F8B8F9C8F2091AD103091AE104E
:10EF90004091AF105091B010C701B6010E947CDAC9
:10EFA0006B017C016D8F7E8F8F8F98A388E50BA1FD
:10EFB0001CA1809FF001819FF00D1124EF53FF4EA3
:10EFC000258936894789508D2DA73EA74FA758AB75
:10EFD000263031054105510508F408C42896AEAD28
:10EFE000BFAD2897CD90DD90ED90FC9020E030E013
:10EFF000A901C701B6010E9417DA811116C426962D
:10F000002CAD3DAD4EAD5FAD2697CA01B9010E9452
:10F010007CDA6B017C01A3019201C301B2010E9461
:10F020007CDA9B01AC01C701B6010E942EDE6B01A8
:10F030007C01A5019401C501B4010E947CDA9B0109
:10F04000AC01C701B6010E942EDE0E9499E028E5BE
:10F050000BA11CA1209FF001219FF00D1124EF5363
:10F06000FF4E658776878787908B88E50BA11CA16B
:10F07000809FF001819FF00D1124EF53FF4E858496
:10F080009684A784B088A501940160E070E080E8D0
:10F090009FE30E940ADF66966CAF7DAF8EAF9FAF95
:10F0A00066979B01AC016DA179A98AA99AAD0E94CE
:10F0B0007CDA2B013C0180912B0A9091290A891B53
:10F0C0008F7027968FAF2797A301920160E074E2BB
:10F0D00084E799E40E940ADF0E945FE06B017C01F3
:10F0E00027968FAD27978250863008F4ADC3A301D1
:10F0F0009201C501B4010E947CDA9B01AC010E941F
:10F100007CDA6A966CAF7DAF8EAF9FAF6A9788E569
:10F11000ABA1BCA18A9F80018B9F100D11240F53BE
:10F120001F4E6A962CAD3DAD4EAD5FAD6A97D801CE
:10F1300011962D933D934D935C93149795962D9135
:10F140003D914D915C9198972AAB3BAB4CAB5DAB3D
:10F15000CA01B9010E941BDA6AAF7BAF8CAF9DAFC9
:10F16000A30192010E947CDA0E94F4DE0E9477DF04
:10F170004B015C01F801EE5BFF4F6083718382837A
:10F1800093838E010F5E1F4F2A961FAF0EAF2A97F3
:10F190000051110924961FAF0EAF249701EF17E01D
:10F1A000A0961FAF0EAFA0978E010F5D1F4F1AA341
:10F1B00009A324960EAD1FAD249762961FAF0EAF24
:10F1C0006297312C212C10E81DA30FE309AB2A967E
:10F1D000AEADBFAD2A976D917D918D919D912A968F
:10F1E000BFAFAEAF2A97A30192010E947CDA6B01F8
:10F1F0007C016296EEADFFAD62976193719381934E
:10F2000091936296FFAFEEAF629720E030E0A901E4
:10F210000E9454E087FF04C0F7FAF094F7F8F094E6
:10F22000A096AEADBFADA0970D911D912D913D91D2
:10F23000A096BFAFAEAFA0976E960CAF1DAF2EAF2E
:10F240003FAF6E97A9019801C701B6010E9454E033
:10F2500018160CF433C32A960EAD1FAD2A9729A1B8
:10F260003AA10217130709F0B2CF20E030E040E8DE
:10F270005FE3632D722D8DA199A90E9417DA87FF94
:10F2800056C07E0131E1E30EF11C24960EAD1FAD98
:10F290002497232D322D4DA159A9D8016D917D912F
:10F2A0008D919C910E947CDAF80161937193819316
:10F2B00091938F01EE15FF0561F728E50BA11CA1C5
:10F2C000209FC001219F900D11249C012F533F4E80
:10F2D000790189010E5B1F4FC501B4010E941BDA41
:10F2E000232D322D4DA159A90E947CDA0E9477DF8F
:10F2F000D8016D937D938D939C931397232D322D7D
:10F300004DA159A9632D722D8DA199A90E947CDA76
:10F310009B01AC016A966CAD7DAD8EAD9FAD6A97D9
:10F320000E947CDAF70161837283838394836696FB
:10F330002CAD3DAD4EAD5FAD66976AAD7BAD8CAD8E
:10F340009DAD0E947CDA6DA37EA38FA398A70DA527
:10F350001EA52FA538A9012B022B032B09F0CAC229
:10F3600088E52BA13CA1829F8001839F100D112471
:10F370000F531F4EF801818D928DA38DB48D892B73
:10F380008A2B8B2B09F0B6C2858D968DA78DB0A1E7
:10F39000892B8A2B8B2B09F0ADC22091ED07309180
:10F3A000EE074091EF075091F0076DA17EA18FA16C
:10F3B00098A50E947CDA0E94F4DE0E9477DF2B0180
:10F3C0003C01D801D7961C9288E52BA13CA1829FD5
:10F3D0008001839F100D11240F531F4EF801E25B33
:10F3E000FF4F4082518262827382C301B2010E9448
:10F3F0001BDA6B017C012DA13EA14FA158A50E94F3
:10F400000ADF6AAF7BAF8CAF9DAFD80151966D9389
:10F410007D938D939C9354972DEB37E346E051E415
:10F42000C701B6010E947CDA0E9477DFF80162AB67
:10F4300073AB84AB95AB87A9882371F1FE962081CD
:10F440003181428153816091E1077091E20780919F
:10F45000E3079091E4070E947CDA2AAD3BAD4CAD06
:10F460005DAD0E947CDA2091BD103091BE104091BC
:10F47000BF105091C0100E947CDA9B01AC0160E08B
:10F4800074E284EF99E40E940ADF0E9477DFD801DA
:10F49000D9967C936E93D89788E50BA11CA1809F89
:10F4A000F001819FF00D1124EF53FF4E2181328135
:10F4B000438154812C962CAF3DAF4EAF5FAF2C975C
:10F4C000CA01B9010E9499E0162F072F382E292E64
:10F4D00041ED57E062965FAF4EAF62973E0151E15A
:10F4E000650E711C81ED97E09BAB8AAB24964EAC08
:10F4F0005FAC249719A70DA73DA229AA1EAAD20185
:10F50000CD90DD90ED90FD902D0120E030E0A9013F
:10F51000C701B6010E9454E087FF04C0F7FAF094D7
:10F52000F7F8F094EAA9FBA981909190A190B1908D
:10F53000FBABEAABA5019401C701B6010E9454E000
:10F5400018160CF4F6C446145704C9F659A5679664
:10F550005FAF67978DA56B968FAF6B979DA16F96E9
:10F560009FAF6F97A9A9EA96AFAFEA972796BFAD6D
:10F570002797B1111EC567968FAD67976B969FADA4
:10F580006B976F96AFAD6F97EA96BFADEA97809392
:10F590000F0890931008A0931108B093120888E503
:10F5A0004BA15CA1849F8001859F100D11240F53F6
:10F5B0001F4E29A53DA54DA159A969A57DA58DA1E0
:10F5C00099A90E947CDAD80119966D937D938D9349
:10F5D0009C931C976AAD7BAD8CAD9DAD90589B0103
:10F5E000AC010E942EDEF8012585368547855089BD
:10F5F0000E947CDA9B01AC016BE077ED83E29BE338
:10F600000E942DDE9B01AC018BE097EDA3E2BBE3F2
:10F61000F80185839683A783B08710812C966CAD03
:10F620007DAD8EAD9FAD2C970E9417DA18160CF0A9
:10F63000FEC581E0182B88E52BA13CA1829FF0013B
:10F64000839FF00D1124EF53FF4E108380E1FE01E4
:10F650003196A1E3BAE001900D928A95E1F72C96DC
:10F660008CAD9DADAEADBFAD2C9780932D0A909320
:10F670002E0AA0932F0AB093300AE0960CAD1DAD70
:10F680002EAD3FADE0970093510A1093520A20939C
:10F69000530A3093540AE4962CAD3DAD4EAD5FADA8
:10F6A000E4972093550A3093560A4093570A509393
:10F6B000580AE8968CAD9DADAEADBFADE89780938E
:10F6C000590A90935A0AA0935B0AB0935C0A609619
:10F6D0000CAD1DAD2EAD3FAD609700935D0A10934C
:10F6E0005E0A20935F0A3093600AA4962CAD3DAD6C
:10F6F0004EAD5FADA4972093410A3093420A4093E8
:10F70000430A5093440AA8968CAD9DADAEADBFADF3
:10F71000A8978093450A9093460AA093470AB0930E
:10F72000480AAC960CAD1DAD2EAD3FADAC97009325
:10F73000490A10934A0A20934B0A30934C0A2296A6
:10F740002CAD3DAD4EAD5FAD229720934D0A309369
:10F750004E0A40934F0A5093500A90912B0A809181
:10F760002C0A981303C084E68093280AE9968FAD8B
:10F77000E9978F5F8F7080932B0A80912B0A90916D
:10F780002A0A81508F70891354C500912C0A0BA34B
:10F7900010912B0A19A798E509A51BA10113D2C541
:10F7A000812C912CA12CB12C1DA61DA219AA1EAE34
:10F7B000212C312C00E010E0FBA129A5F213CFC5CC
:10F7C0002114310409F080C680916F00826080931B
:10F7D0006F0081E0DEC780E0DCC720900508309034
:10F7E000060800910708109108087ECB818D928D44
:10F7F000A38DB48D0697A105B10508F0EFCB858DDB
:10F80000968DA78DB0A10697A105B10508F0E6CBAE
:10F8100020E030E0A901C701B6010E9454E087FF53
:10F8200004C0F7FAF094F7F8F09488E50BA11CA156
:10F83000809FF001819FF00D1124EF53FF4EC5868C
:10F84000D686E786F08A11CC809101089091020853
:10F85000A0910308B0910408C816D906EA06FB0671
:10F8600008F045CC8C199D09AE09BF09BC01CD013A
:10F87000660F771F881F991F27964FAD2797042F74
:10F8800010E020E030E0A90198010E94F2DDCA01F9
:10F89000B9010E941BDA0E945FE06C0D7D1D8E1D78
:10F8A0009F1D0E941BDA9B01AC0160E074E284E7BB
:10F8B00099E40E940ADF2B013C0119CCA7019601B3
:10F8C0006E966CAD7DAD8EAD9FAD6E970E940ADFDA
:10F8D0007B018C019B01AC01632D722D8DA199A937
:10F8E0000E9454E018160CF0B6CC3E2C2F2C0DA321
:10F8F00019ABB1CC0EA91FA928AD39AD012B022B34
:10F90000032B49F06091E9077091EA078091EB07BA
:10F910009091EC0708C06091E5077091E60780912F
:10F92000E7079091E8072DA13EA14FA158A50E949D
:10F930007CDA0E94F4DE0E9477DF2B013C012EA9C5
:10F940003FA948AD59AD232B242B252BC9F020E02E
:10F9500030E0A9016091E1077091E2078091E3072F
:10F960009091E4070E9417DA882351F081E009A5FD
:10F970001AA52BA53CA510161106120613060CF0AD
:10F9800080E098E52BA13CA1929F8001939F100DF0
:10F9900011240F531F4ED801D7968C93882309F456
:10F9A000B2C02091410A3091420A4091430A5091DD
:10F9B000440AA4966CAD7DAD8EAD9FADA4970E9418
:10F9C0002DDE69A77AA78BA79CA72091450A3091C5
:10F9D000460A4091470A5091480AA8966CAD7DAD01
:10F9E0008EAD9FADA8970E942DDE4B015C0120914A
:10F9F000490A30914A0A40914B0A50914C0AAC9600
:10FA00006CAD7DAD8EAD9FADAC970E942DDE6B01D0
:10FA10007C0129A53AA54BA55CA5CA01B9010E94A4
:10FA20007CDA69A77AA78BA79CA7A5019401C501D9
:10FA3000B4010E947CDA9B01AC0169A57AA58BA573
:10FA40009CA50E942EDE4B015C01A7019601C70117
:10FA5000B6010E947CDA9B01AC01C501B4010E9491
:10FA60002EDE0E9499E06B017C0120914D0A3091BD
:10FA70004E0A40914F0A5091500A22966CAD7DADCE
:10FA80008EAD9FAD22970E942DDEA70196010E94A8
:10FA90000ADF6B017C01F801FE966083718382832B
:10FAA000938320E030E040E450E40E9454E01816D4
:10FAB0001CF4F80117AA27C02091E1073091E20752
:10FAC0004091E3075091E407C701B6010E947CDA38
:10FAD0009B01AC016091DD077091DE078091DF072B
:10FAE0009091E0070E940ADF2DA13EA14FA158A5E9
:10FAF0000E947CDA0E9477DF6415750586059705FC
:10FB000010F42B013C0180917D1090917E10A0910A
:10FB10007F10B09180100AA91BA92CA93DA98017BC
:10FB20009107A207B30708F4E9C02DA53EA54FA58C
:10FB300058A9232B242B252B61F120918110309182
:10FB4000821040918310509184102415350546058C
:10FB50005705F8F46AA97BA98CA99DA90E94E3DD49
:10FB60006B017C01A30192016DA57EA58FA598A9CB
:10FB70000E94E3DDC616D706E806F90650F4C70171
:10FB8000B6012DA53EA54FA558A90E94F2DD290179
:10FB90003A0188E50BA11CA1809FF001819FF00D27
:10FBA0001124EF53FF4EC18CD28CE38CF48CC11422
:10FBB000D104E104F10441F12091851030918610C7
:10FBC000409187105091881024153505460557053A
:10FBD000D8F46AA97BA98CA99DA90E94E3DD4B01F9
:10FBE0005C01A3019201C701B6010E94E3DD861604
:10FBF0009706A806B90640F4C501B401A70196010D
:10FC00000E94F2DD29013A0188E50BA11CA1809F29
:10FC1000F001819FF00D1124EF53FF4EC58CD68C5F
:10FC2000E78CF0A0C114D104E104F10441F120916A
:10FC3000891030918A1040918B1050918C102415AE
:10FC4000350546055705D8F46AA97BA98CA99DA955
:10FC50000E94E3DD4B015C01A3019201C701B601E3
:10FC60000E94E3DD86169706A806B90640F4C50192
:10FC7000B401A70196010E94F2DD29013A0188E54D
:10FC80000BA11CA1809FF001819FF00D1124EF5367
:10FC9000FF4EC1A0D2A0E3A0F4A0C114D104E1049E
:10FCA000F10409F491CB20918D1030918E10409188
:10FCB0008F1050919010241535054605570508F012
:10FCC00083CB6AA97BA98CA99DA90E94E3DD4B0186
:10FCD0005C01A3019201C701B6010E94E3DD861613
:10FCE0009706A806B90608F06FCBC501B401A701B5
:10FCF00096010E94F2DD29013A0166CB2DA53EA5B1
:10FD00004FA558A9232B242B252BB9F160918110E5
:10FD10007091821080918310909184106415750504
:10FD20008605970550F50E941BDA2AAD3BAD4CAD18
:10FD30005DAD0E947CDA6B017C016DA57EA58FA56F
:10FD400098A90E941BDA4B015C01C301B2010E9419
:10FD50001BDAA50194010E947CDAA70196010E949A
:10FD600054E0181654F4A5019401C701B6010E948D
:10FD70000ADF0E9477DF2B013C0188E50BA11CA163
:10FD8000809FF001819FF00D1124EF53FF4E818C75
:10FD9000928CA38CB48C81149104A104B104A9F1B8
:10FDA00060918510709186108091871090918810D5
:10FDB000641575058605970540F50E941BDA2AAD86
:10FDC0003BAD4CAD5DAD0E947CDA6B017C01C501A1
:10FDD000B4010E941BDA4B015C01C301B2010E9415
:10FDE0001BDAA50194010E947CDAA70196010E940A
:10FDF00054E0181654F4A5019401C701B6010E94FD
:10FE00000ADF0E9477DF2B013C0188E50BA11CA1D2
:10FE1000809FF001819FF00D1124EF53FF4E858CE0
:10FE2000968CA78CB0A081149104A104B104A9F10F
:10FE30006091891070918A1080918B1090918C1034
:10FE4000641575058605970540F50E941BDA2AADF5
:10FE50003BAD4CAD5DAD0E947CDA6B017C01C50110
:10FE6000B4010E941BDA4B015C01C301B2010E9484
:10FE70001BDAA50194010E947CDAA70196010E9479
:10FE800054E0181654F4A5019401C701B6010E946C
:10FE90000ADF0E9477DF2B013C0188E50BA11CA142
:10FEA000809FF001819FF00D1124EF53FF4EC1A000
:10FEB000D2A0E3A0F4A0C114D104E104F10409F438
:10FEC00083CA60918D1070918E1080918F109091E7
:10FED0009010641575058605970508F075CA0E948F
:10FEE0001BDA2AAD3BAD4CAD5DAD0E947CDA4B0117
:10FEF0005C01C701B6010E941BDA6B017C01C301E2
:10FF0000B2010E941BDAA70196010E947CDAA501CA
:10FF100094010E9454E018160CF056CAA7019601ED
:10FF2000C501B4010E940ADF0E9477DF2B013C016A
:10FF30004BCAFEA9FF2329F1A5019401612F702F5F
:10FF4000832D922D0E947CDA4B015C0129A53DA5F1
:10FF50004DA159A9C701B6010E947CDAA5019401FF
:10FF60000E9454E0181614F5A7019601C501B401CA
:10FF70000E940ADF69A77DA78DA399AB21E02EAB74
:10FF8000E2CAA7019601C501B4010E940ADF9B01E4
:10FF9000AC0169A57DA58DA199A90E947CDA69A70C
:10FFA0007DA78DA399AB31E03EABCDCA41E04EAB0E
:10FFB000CACAC0902D0AD0902E0AE0902F0AF09065
:10FFC000300A2DEB37E346E855E3C701B6010E943E
:10FFD00017DA87FDD0CAC701B6010E9499E06B010C
:10FFE0007C019B01AC01612F702F832D922D0E940B
:10FFF00017DA87FD04C01C2D0D2D3E2C2F2C9601E9
:020000021000EC
:10000000A701612F702F832D922D0E940ADF669623
:100010006CAF7DAF8EAF9FAF6697E1E3FAE02896B5
:10002000FFAFEEAF289720E030E040E85FE32EAB73
:100030003FAB48AF59AF1AAA2896AEADBFAD2897CF
:100040006D917D918D919D912896BFAFAEAF289710
:1000500066962CAD3DAD4EAD5FAD66970E947CDAE5
:100060006B017C012496EEADFFAD249781909190B9
:10007000A190B1902496FFAFEEAF2497FAA9FF2389
:1000800091F02EA93FA948AD59AD0E947CDA6B01D1
:100090007C012EA93FA948AD59ADC501B4010E940C
:1000A0007CDA4B015C01A5019401C701B6010E94F5
:1000B00054E020E030E0A90118162CF5C501B40188
:1000C0000E9454E018164CF020E030E0A901C7016E
:1000D000B6010E9417DA87FF05C0A5019401C70188
:1000E000B60124C02401350177FA709477F8709432
:1000F000A3019201C701B6010E9454E018165CF5F5
:100100002601370128C0C501B4010E9417DA87FD16
:1001100009C020E030E0A901C701B6010E9454E007
:1001200018164CF4A7019601C501B4010E942DDEFA
:100130002B013C0110C02601370177FA709477F843
:100140007094A5019401C301B2010E9454E01816F5
:1001500014F0240135016296AEADBFAD6297CD902B
:10016000DD90ED90FD906296BFAFAEAF6297A701B4
:100170009601C301B2010E9454E01816ACF4A30129
:100180009201C701B6010E940ADF9B01AC016EA972
:100190007FA988AD99AD0E947CDA6EAB7FAB88AF4A
:1001A00099AFBAA9BF5FBAAB2896EEADFFAD28975D
:1001B000E154FA4009F040CF3AA9332371F02EA957
:1001C0003FA948AD59AD612F702F832D922D0E940C
:1001D0007CDA162F072F382E292E24EA30E74DE738
:1001E0005FE3612F702F832D922D0E947CDA6B01CB
:1001F0007C019B01AC0160910F0870911008809107
:100200001108909112080E9454E018165CF4A7019E
:10021000960169A57DA58DA199A90E9454E01816A3
:100220000CF4A9C919A70DA73DA229AAA4C983E066
:1002300001CAF0902B0A8FEF8F0D8F708BA3B090B7
:100240002A0A80912B0AB81206C000912A0A0BA331
:10025000C12CD12C69C0C12CD12C1BA11B15A9F319
:100260001BA1812E912C28E5289D8001299D100D30
:1002700011240F531F4ED8018C9183FD27C009AB69
:100280001EAF0115110521F11996BC91B9A7F8010E
:10029000F285FDA7D8011B96BC91BDA3F801A484EB
:1002A000458056806780708429A53DA54B2F5A2D27
:1002B000C301B2010E9417DA81117FC1C114D104B8
:1002C00039F0D6018C9180FD78C102C0C9AADEAE9A
:1002D0008BA181508F708BA380912A0AB81649F0A8
:1002E0000BA10B1509F4B1CF81E08B0D8F70B82EE7
:1002F000F3CFC9A8DEACB1CF0BA1802E912C28E59D
:10030000289D8001299D100D11240F531F4ED801E7
:100310008C9183FD15C05801C114D10459F48BA1EF
:100320008F5F8F708BA3650180912B0A1BA118131F
:10033000E3CF2BCAC6010E94E0498111F0CFB3C1BF
:100340005601EDCF89A581508F70989FF00111243F
:10035000EF53FF4E208123FF23CA89A71DCA28E53A
:100360003BA1239FC0011124AC014F535F4E1A01E2
:10037000DA018C9183FD19C015966D917D918D9157
:100380009C9118970E9499E0F62EE72ED82EC92E40
:100390000115110509F48AC0F801808180FD0AC0A9
:1003A000D1018C9180FD06C081C0FDA4EDA0D9A82B
:1003B000CEAC81C0F801808181608083C8010E9439
:1003C000E04981116FC0F80161817281838194815C
:1003D0000E9499E02B013C019B01AC0160E070E0C0
:1003E00080E89FE30E940ADF4B015C019B01AC01A6
:1003F0006F2D7E2D8D2D9C2D0E947CDA69837A8352
:100400008B839C83A50194016DA57DA189A99EADD7
:100410000E947CDA698B7A8B8B8B9C8BAE014F5F51
:100420005F4FBE016F5E7F4FC8010E9468C4D80154
:10043000D7968C918823B1F12091E1073091E207A2
:100440004091E3075091E407F801FE9660817181C5
:10045000828193810E947CDA2091BD103091BE1080
:100460004091BF105091C0100E947CDA4B015C019A
:100470009B01AC01C301B2010E947CDA0E9477DFCC
:10048000F80173AF62AFA50194016F2D7E2D8D2D04
:100490009C2D0E947CDA0E9477DFD801DD967C9348
:1004A0006E93DC97F80180818E7F80838F2C9E2C49
:1004B000AD2CBC2C81018BA18F5F8F708BA3FDA60F
:1004C000EDA2D9AACEAE78C9D1018C9181608C936E
:1004D000C8010E94E04981116BC0F1016181728104
:1004E000838194810E9499E06B017C019B01AC01A6
:1004F00060E070E080E89FE30E940ADF2B013C018E
:100500002DEC3CEC4CE45DE30E947CDA69837A8359
:100510008B839C83A3019201B401C5010E947CDA04
:10052000698B7A8B8B8B9C8BAE014F5F5F4FBE01CB
:100530006F5E7F4FC1010E9468C4D101D7968C9134
:100540008823B1F12091E1073091E2074091E30760
:100550005091E407F101FE9660817181828193815F
:100560000E947CDA2091BD103091BE104091BF10E6
:100570005091C0100E947CDA4B015C019B01AC01E0
:10058000C701B6010E947CDA0E9477DFF10173AFE8
:1005900062AF2DEC3CEC4CE45DE3C501B4010E947C
:1005A0007CDA0E9477DFD101DD967C936E93DC9735
:1005B000F10180818E7F808307C928E5289DF001A5
:1005C000299DF00D1124EF53FF4E808181FD3FC026
:1005D000C114D10431F0F601C580D680E780F084E3
:1005E00008C08BE0C82E87EDD82E83E2E82E8BE37F
:1005F000F82E28E5289DF001299DF00D1124EF53D8
:10060000FF4E81899289A389B489BC01CD0190589C
:100610009B01AC010E942EDED8011D962D913D91CB
:100620004D915C9150970E947CDA9B01AC01C7010F
:10063000B6010E942DDE1B016C019B01AC0169A576
:100640007DA58DA19A2D0E9417DA87FF04C029A4E9
:100650003DA4CDA0DA2C9101A601C301B2010E94F4
:1006600017DA882309F434CEB8E5B89DC001B99DE6
:10067000900D1124FC01EF53FF4E4F0180818160EA
:100680008083C8010E94E049882329F0D4018C911D
:100690008E7F8C931DCEC101D601F4018583968394
:1006A000A783B08715CED6018C9181FD50C0D601AD
:1006B00015962D913D914D915C91189729A73AA7D8
:1006C0004BA75CA71501B5E02B0E311CF801458046
:1006D000568067807084A301920169A57AA58BA5D5
:1006E0009CA50E9417DA87FF32C0F60181899289A2
:1006F000A389B489BC01CD0190589B01AC010E9433
:100700002EDED6011D962D913D914D915C91509715
:100710000E947CDA9B01AC0169A57AA58BA59CA5FA
:100720000E942DDE6B017C01A30192010E9417DA69
:1007300087FF0DC0D8018C9181608C93C5010E9408
:10074000E0498823E1F0F80180818E7F808318E5FD
:10075000189DF001199DF00D1124EF53FF4E2185D6
:1007600032854385548565817681878190850E9495
:1007700017DA8111D4CD0BA100932A0AD0CDD10173
:10078000CD92DD92ED92FC9213970BA100932A0A71
:10079000DECFC758DF4F0FB6F894DEBF0FBECDBF18
:1007A000DF91CF911F910F91FF90EF90DF90CF904D
:1007B000BF90AF909F908F907F906F905F904F9081
:1007C0003F902F90089580912B0A90912C0A891BBD
:1007D0008F708F3019F40E94C955F5CF80912B0A84
:1007E0008F5F8F70E0912B0A98E59E9FF001112496
:1007F000EF53FF4EDF011D929A95E9F798E0908341
:100800004091510A5091520A6091530A7091540AD2
:10081000458B568B678B708F4091550A5091560AC5
:100820006091570A7091580A418F528F638F748F6D
:100830004091590A50915A0A60915B0A70915C0A82
:10084000458F568F678F70A340915D0A50915E0A65
:1008500060915F0A7091600A41A352A363A374A3DD
:1008600020912B0A90912C0A291303C094E69093AF
:10087000280A80932B0A80916F00826080936F001A
:10088000089590912B0A80912C0A981719F00E94D4
:10089000C955F7CF8091FB069091FC06892BB9F7DB
:1008A000089590912B0A80912C0A981719F00E94B4
:1008B000C955F7CF8091FB069091FC06892BB9F7BB
:1008C0000C945C55CF93DF9390916F0091FB22279E
:1008D00020F991FF05C090916F009D7F90936F006C
:1008E00094E0899FE0011124FE01E052FA4F6081FB
:1008F000718182819381222329F020916F002260EF
:1009000020936F000E941DDACF55DF4E2881398178
:100910004A815B810E947CDADF91CF910895CF926A
:10092000DF92EF92FF92CF93DF9320916C102223FE
:1009300031F1EC0108960E943BC66B017C0120E07E
:1009400030E0A9010E9417DA882361F0CE010E94ED
:10095000A55D9B01AC01C701B6010E947CDA9B0139
:10096000AC0103C020E030E0A901688579858A8563
:100970009B850E942DDE688779878A879B87DF9118
:10098000CF91FF90EF90DF90CF9008954F925F92BC
:100990006F927F92AF92BF92CF92DF92EF92FF92CF
:1009A0000F931F93CF93DF93CDB7DEB72C970FB67E
:1009B000F894DEBF0FBECDBF20916C10222309F446
:1009C00046C08A017B016C01CA010E943BC62B0113
:1009D0003C01CE0101965C018CE0F50111928A95F3
:1009E000E9F7F60180819181A281B38189839A839D
:1009F000AB83BC83F70180819181A281B3818D8318
:100A00009E83AF83B88720E030E0A901C301B20123
:100A10000E9417DA882361F0C5010E94A55D9B0141
:100A2000AC01C301B2010E947CDA9B01AC0103C09E
:100A300020E030E0A901F801608171818281938119
:100A40000E942EDEF80160837183828393832C964B
:100A50000FB6F894DEBF0FBECDBFDF91CF911F91CF
:100A60000F91FF90EF90DF90CF90BF90AF907F906D
:100A70006F905F904F900895CF93DF938B399240A2
:100A8000B1F0E9EBF3E28491EF012196882321F0A4
:100A90000E941896FE01F7CFE3E8F2E28491EF019D
:100AA0002196882331F00E941896FE01F7CF80E04E
:100AB00001C081E0DF91CF9108952F923F924F9234
:100AC0005F926F927F928F929F92AF92BF92CF92DE
:100AD000DF92EF92FF920F931F93CF93DF93CDB7E7
:100AE000DEB7C157D1090FB6F894DEBF0FBECDBF38
:100AF0002DB63EB6A7961FAE1EAEA79784E690E031
:100B0000A5969FAF8EAFA59701E09E012B593F4F51
:100B100044E050E0BE01695A7F4FCE018D599F4F8E
:100B20000E9496B59E012B593F4F42E050E0BE0116
:100B30006F597F4FCE018D599F4F0E9496B543E06C
:100B400050E0BE01695A7F4F8BEE92E00E94A3E114
:100B5000892B09F43BC06B968FAD6B97882339F0D6
:100B60008FE368968FAF689769961FAE6997EEEC32
:100B7000F3E284918F010F5F1F4F882321F00E94C1
:100B80001896F801F6CFE6E4F3E284918F010F5F47
:100B90001F4F882321F00E941896F801F6CFBE015E
:100BA000695A7F4F8DE393E20E94D0C8EFE2F3E2EF
:100BB00084918F010F5F1F4F882321F00E941896A8
:100BC000F801F6CF81E080931808F8C42DB73EB73E
:100BD000E0963FAF2EAFE09767961CAE1DAE1EAEFF
:100BE0001FAE6797A7961FAE1EAEA79701E09E01A6
:100BF0002B593F4F41E050E0BE0164597F4FCE0179
:100C00008D599F4F0E9496B580E1EFE6F2E0DE013C
:100C1000919601900D928A95E1F780E1EFE7F2E07D
:100C2000DE01519601900D928A95E1F780E1EFE89F
:100C3000F2E09E012F5F3F4F7901D90101900D92A3
:100C40008A95E1F7AD964FADAD9750E04D5F5F4FA0
:100C5000440F551F440F551F8DB79EB7841B950B2E
:100C60000FB6F8949EBF0FBE8DBFEDB7FEB731969D
:100C70004F0100E02C593F4FBF01CE018D599F4FCE
:100C80000E9496B59E012B593F4F44E050E061E031
:100C900078E0CE018D599F4F0E9496B5AD966FAC0E
:100CA000AD97712CF3E06F0E711C660C771C660C0F
:100CB000771C2DB73EB7261937090FB6F8943EBFFB
:100CC0000FBE2DBF8DB79EB701965C01EDB7FEB785
:100CD000E619F7090FB6F894FEBF0FBEEDBF2DB7AA
:100CE0003EB72F5F3F4F69019E012B593F4FA30134
:100CF000BC01CE018D599F4F0E9496B59E012B5984
:100D00003F4FA301B601CE018D599F4F0E9496B56A
:100D100080910B10882309F4A2C000E09E012B599A
:100D20003F4F44E050E069EE77E0CE018D599F4F90
:100D30000E9496B59E012B593F4F44E050E06DEE66
:100D400077E0CE018D599F4F0E9496B59E012B5999
:100D50003F4F44E050E065EE77E0CE018D599F4F64
:100D60000E9496B59E012B593F4F44E050E069E048
:100D700078E0CE018D599F4F0E9496B59E012B5968
:100D80003F4F44E050E065E078E0CE018D599F4F41
:100D90000E9496B59E012B593F4F40E150E061ED16
:100DA00077E0CE018D599F4F0E9496B59E012B5939
:100DB0003F4F44E050E0BE016D5A7F4FCE018D5948
:100DC0009F4F0E9496B59E012B593F4F4CE050E03B
:100DD00066E474E0CE018D599F4F0E9496B59E0146
:100DE0002B593F4F44E050E06CE070E1CE018D594B
:100DF0009F4F0E9496B59E012B593F4F44E050E013
:100E0000BE016D5A7F4FCE018D599F4F0E9496B5FE
:100E100001E09E012B593F4F41E050E0BE01655972
:100E20007F4FCE018D599F4F0E9496B59E012B5941
:100E30003F4F41E050E0BE0166597F4FCE018D59D2
:100E40009F4F0E9496B5AC968FADAC97AB96EFAC2A
:100E5000AB978E9D70011124C12CD12C5FC0AD9633
:100E60002FADAD9730E02E5F3F4F81EF97E0E296D8
:100E70009FAF8EAFE29761EB70E1A1E9B0E180E056
:100E800090E040E050E02417350714F0840104C0DE
:100E900001E210E00C0F1D1F080F191FF801408020
:100EA0005180628073804D925D926D927D92241785
:100EB000350714F0850104C001E110E00C0F1D1F7F
:100EC000080F191FF8014080518062807380FB0178
:100ED0004192519261927192BF012417350714F02B
:100EE000860101C08701080F191FF8014080518059
:100EF00062807380E296EEADFFADE297419251922F
:100F000061927192E296FFAFEEAFE2974F5F5F4F53
:100F100004964430510509F0B6CFFFCE00E09E01A3
:100F20002B593F4F44E050E0CE14DF0461F0BE0186
:100F30006D5A7F4FCE018D599F4F0E9496B5FFEF9E
:100F4000CF1ADF0AEBCF67E074E0CE018D599F4FD7
:100F50000E9496B51AE0115079F000E09E012B59DD
:100F60003F4F44E050E0BE016D5A7F4FCE018D5996
:100F70009F4F0E9496B5EFCF01E09E012B593F4F46
:100F800041E050E0BE0167597F4FCE018D599F4F20
:100F90000E9496B59E012B593F4F41E050E0BE01A3
:100FA00068597F4FCE018D599F4F0E9496B5AA96E2
:100FB0008FADAA97833089F5A9968FADA997833015
:100FC00061F580910B10811102C00E94EB7200E06C
:100FD0009E012B593F4F44E050E060E170E1CE01AB
:100FE0008D599F4F0E9496B59E012B593F4F44E06B
:100FF00050E064E178E0CE018D599F4F0E9496B594
:101000009E012B593F4F44E250E068E170E1CE0170
:101010008D599F4F0E9496B53BC000E09E012B5911
:101020003F4F44E050E0BE01635C7F4FCE018D59DD
:101030009F4F0E9496B59E012B593F4F44E050E0D0
:10104000BE016F5C7F4FCE018D599F4F0E9496B5B8
:10105000AA968FADAA97A996EFACA9978E9D70011D
:101060001124C12CD12CCE14DF0491F000E09E019C
:101070002B593F4F44E050E0BE016D5A7F4FCE01E7
:101080008D599F4F0E9496B52FEFC21AD20AEBCF0F
:1010900000E09E012B593F4F41E050E0BE016359F3
:1010A0007F4FCE018D599F4F0E9496B59E012B59BF
:1010B0003F4F41E050E0BE0169597F4FCE018D594D
:1010C0009F4F0E9496B59E012B593F4F44E050E040
:1010D000BE016D5A7F4FCE018D599F4F0E9496B52C
:1010E0009E012B593F4F44E050E0BE016D5A7F4FA7
:1010F000CE018D599F4F0E9496B59E012B593F4FAF
:1011000044E050E064E170E1CE018D599F4F0E94B0
:1011100096B59E012B593F4F44E050E0BE01615B04
:101120007F4FCE018D599F4F0E9496B59E012B593E
:101130003F4F44E050E0BE01655B7F4FCE018D59CB
:101140009F4F0E9496B59E012B593F4F44E050E0BF
:10115000BE01695B7F4FCE018D599F4F0E9496B5AE
:1011600010E000E09E012B593F4F44E050E0BE01EB
:101170006D5A7F4FCE018D599F4F0E9496B5111128
:1011800043C06796CCACDDACEEACFFAC679720E01B
:1011900030E84BE355E4C701B6010E9417DA882313
:1011A00099F180910B10811108C0C0920006D09275
:1011B0000106E0920206F092030600E09E012B5920
:1011C0003F4F44E050E06CEF75E0CE018D599F4FEA
:1011D0000E9496B59E012B593F4F44E050E064E0D9
:1011E00076E0CE018D599F4F0E9496B59E012B59F6
:1011F0003F4F44E050E0BE016D5A7F4FCE018D5904
:101200009F4F0E9496B514C084E0F82EFA94FF20F8
:1012100079F000E09E012B593F4F44E050E0BE01C1
:101220006D5A7F4FCE018D599F4F0E9496B5EECFDC
:101230001F5F153009F095CF00E09E012B593F4FFD
:1012400042E050E0BE01615A7F4FCE018D599F4F61
:101250000E9496B514E0115000E09E012B593F4FBB
:10126000112359F044E050E0BE016D5A7F4FCE018A
:101270008D599F4F0E9496B5EECF42E050E0BE01DF
:10128000635A7F4FCE018D599F4F0E9496B59E01A4
:101290002B593F4F41E050E0BE0163597F4FCE01D3
:1012A0008D599F4F0E9496B519E0115000E09E01A4
:1012B0002B593F4F112359F044E050E0BE016D5AC5
:1012C0007F4FCE018D599F4F0E9496B5EECF41E0E2
:1012D00050E064E770E1CE018D599F4F0E9496B5B2
:1012E00000E09E012B593F4F44E050E0BE016D5A93
:1012F0007F4FCE018D599F4F0E9496B580910B1064
:10130000811110C011110EC067968CAD9DADAEADB0
:10131000BFAD67978093791090937A10A0937B105C
:10132000B0937C101F5F1530D9F61CE0115079F096
:1013300000E09E012B593F4F42E050E0BE01655A4C
:101340007F4FCE018D599F4F0E9496B5EFCF1CE085
:10135000115000E09E012B593F4F112359F044E0FA
:1013600050E0BE016D5B7F4FCE018D599F4F0E94B3
:1013700096B5EECF46E050E0BE01635C7F4FCE01F4
:101380008D599F4F0E9496B59E012B593F4F44E0C7
:1013900050E061EE77E0CE018D599F4F0E9496B5E7
:1013A0009E012B593F4F4CE050E0BE016F5C7F4FD8
:1013B000CE018D599F4F0E9496B51CE1115079F0D6
:1013C00000E09E012B593F4F44E050E0BE016D5AB2
:1013D0007F4FCE018D599F4F0E9496B5EFCF14E0FD
:1013E000115079F000E09E012B593F4F44E050E04E
:1013F000BE016D5A7F4FCE018D599F4F0E9496B509
:10140000EFCF1BE0115079F000E09E012B593F4FC8
:1014100044E050E0BE016D5A7F4FCE018D599F4F81
:101420000E9496B5EFCFA5968EAD9FADA597845639
:10143000910922DB80931808882301F1EEECF3E296
:1014400084918F010F5F1F4F882321F00E9418960F
:10145000F801F6CFA5966EAD7FADA59764567109DC
:1014600087E293E20E94B7C86BE972E08FE193E2F2
:101470000E94B7C88AE00E9418968DC0A7962EAD2C
:101480003FADA797A3968EAD9FADA39728173907B9
:1014900009F446C081E080931808E9EBF3E28491F7
:1014A0008F010F5F1F4F882321F00E941896F801CB
:1014B000F6CFEFEFF2E284918F010F5F1F4F882389
:1014C00021F00E941896F801F6CFA3966EAD7FAD7D
:1014D000A39780E090E04AE00E942296EAEFF2E2D1
:1014E00084918F010F5F1F4F882321F00E9418966F
:1014F000F801F6CFA7966EAD7FADA79780E090E09C
:101500004AE00E942296EAEEF2E284918F010F5F98
:101510001F4F882309F43FC00E941896F801F5CFA9
:1015200080910B10811137C0EEECF3E284918F01B2
:101530000F5F1F4F811103C00BEE12E004C00E9429
:101540001896F801F3CFF80181918F01882319F0E3
:101550000E941896F8CFA5966EAD7FADA5976456FC
:1015600071098DEC92E20E94B7C8A7964EAD5FADAF
:10157000A79760E070E080EC92E20E947DC8EDEBFE
:10158000F2E284918F010F5F1F4F882321F00E94A8
:101590001896F801F6CF80910B10811106C080914A
:1015A0001808811102C00E9458B6E0962EAD3FADDA
:1015B000E0970FB6F8943EBF0FBE2DBF80910B1081
:1015C000811102C00E94DDAF9091180881E0892747
:1015D0000FB6F8943EBE0FBE2DBECF58DF4F0FB6EC
:1015E000F894DEBF0FBECDBFDF91CF911F910F9159
:1015F000FF90EF90DF90CF90BF90AF909F908F9033
:101600007F906F905F904F903F902F9008958F92B2
:101610009F92AF92BF92CF92DF92EF92FF920F9381
:101620001F93CF93DF93CDB7DEB7CE59D1090FB655
:10163000F894DEBF0FBECDBFC757DF4F18821982A7
:101640001A821B82C958D04085E492E5A2E5B0E039
:10165000CB57DF4F88839983AA83BB83C558D0407B
:10166000CB56DF4F19821882C559D04084E690E0EE
:10167000CD56DF4F99838883C359D0401092180804
:101680009E012B563F4F44E050E0BE016B577F4F09
:10169000CE018D569F4F0E94E4B5CD56DF4F888115
:1016A0009981C359D0400296CD56DF4F99838883E4
:1016B000C359D040CB56DF4F19821882C559D0404C
:1016C00081E0C256DF4F8883CE59D0409E012B5611
:1016D0003F4F41E050E0BE0162567F4FCE018D5634
:1016E0009F4F0E94E4B59E012B563F4F40E150E0D2
:1016F00061E970E1CE018D569F4F0E94E4B59E01D5
:101700002B563F4F44E050E061E078E0CE018D562B
:101710009F4F0E94E4B59E012B563F4F40E150E0A1
:1017200061EB70E1CE018D569F4F0E94E4B59E01A2
:101730002B563F4F40E150E061EF77E0CE018D56F0
:101740009F4F0E94E4B59E012B563F4F44E050E06E
:1017500069EE77E0CE018D569F4F0E94E4B59E0161
:101760002B563F4F44E050E06DEE77E0CE018D56B2
:101770009F4F0E94E4B59E012B563F4F44E050E03E
:1017800065EE77E0CE018D569F4F0E94E4B59E0135
:101790002B563F4F44E050E069E078E0CE018D5693
:1017A0009F4F0E94E4B59E012B563F4F44E050E00E
:1017B00065E078E0CE018D569F4F0E94E4B59E0112
:1017C0002B563F4F40E150E061ED77E0CE018D5662
:1017D0009F4F0E94E4B58AE097EDA3EABCE3C757A8
:1017E000DF4F88839983AA83BB83C958D0409E0169
:1017F0002B563F4F44E050E0BE0167577F4FCE016C
:101800008D569F4F0E94E4B59E012B563F4F4CE0F2
:1018100050E066E474E0CE018D569F4F0E94E4B51F
:1018200080916D1090916E10A0916F10B09170101A
:10183000CF57DF4F88839983AA83BB83C158D04099
:101840009E012B563F4F44E050E0BE016F577F4F43
:10185000CE018D569F4F0E94E4B5C757DF4F1882C7
:1018600019821A821B82C958D04083E0C356DF4FC9
:101870008883CD59D040C456DF4F8883CC59D0409F
:101880009E012B563F4F44E050E0BE0167577F4F0B
:10189000CE018D569F4F0E94E4B59E012B563F4FBF
:1018A00041E050E0BE0163567F4FCE018D569F4F01
:1018B0000E94E4B59E012B563F4F41E050E0BE012F
:1018C00064567F4FCE018D569F4F0E94E4B51AE0BB
:1018D00011509E012B563F4F44E050E0112349F038
:1018E000BE0167577F4FCE018D569F4F0E94E4B5D2
:1018F000EFCF67E074E0CE018D569F4F0E94E4B5B4
:10190000C757DF4F188219821A821B82C958D040EC
:101910001AE0115071F09E012B563F4F44E050E009
:10192000BE0167577F4FCE018D569F4F0E94E4B591
:10193000F0CF83E0C556DF4F8883CB59D040C656E1
:10194000DF4F8883CA59D0409E012B563F4F41E05C
:1019500050E0BE0165567F4FCE018D569F4F0E94CD
:10196000E4B59E012B563F4F41E050E0BE01665664
:101970007F4FCE018D569F4F0E94E4B59E012B569E
:101980003F4F44E050E060E170E1CE018D569F4F43
:101990000E94E4B59E012B563F4F44E050E064E1C5
:1019A00078E0CE018D569F4F0E94E4B59E012B56E4
:1019B0003F4F44E250E068E170E1CE018D569F4F09
:1019C0000E94E4B5C756DF4F1882C959D0408FEF47
:1019D000C856DF4F8883C859D0409E012B563F4FD1
:1019E00041E050E0BE0167567F4FCE018D569F4FBC
:1019F0000E94E4B59E012B563F4F41E050E0BE01EE
:101A000068567F4FCE018D569F4F0E94E4B5C75751
:101A1000DF4F188219821A821B82C958D0409E015A
:101A20002B563F4F44E050E0BE0167577F4FCE0139
:101A30008D569F4F0E94E4B59E012B563F4F44E0C8
:101A400050E0BE0167577F4FCE018D569F4F0E94D9
:101A5000E4B59E012B563F4F44E050E064E170E155
:101A6000CE018D569F4F0E94E4B584EB90E0EF9637
:101A70009FAF8EAFEF9780EF90E0C158DF4F998313
:101A80008883CF57D04086E490E0EB969FAF8EAF2F
:101A9000EB978EE690E0ED969FAF8EAFED97E796D1
:101AA0001FAE1EAEE797E9961FAE1EAEE9979E01E8
:101AB0002B563F4F44E050E0BE0163587F4FCE01AC
:101AC0008D569F4F0E94E4B59E012B563F4F44E038
:101AD00050E0BE0167587F4FCE018D569F4F0E9448
:101AE000E4B59E012B563F4F44E050E0BE016B58D9
:101AF0007F4FCE018D569F4F0E94E4B5C12C80E8E8
:101B0000D82E8BE3E82E85E4F82E812C912C90E8DA
:101B1000A92E9FE3B92E11113AC09E012B563F4FBB
:101B200044E050E060E076E0CE018D569F4F0E9489
:101B3000E4B59E012B563F4F44E050E06CEF75E05A
:101B4000CE018D569F4F0E94E4B59E012B563F4F0C
:101B500044E050E064E076E0CE018D569F4F0E9455
:101B6000E4B5C757DF4F88829982AA82BB82C958E1
:101B7000D0409E012B563F4F44E050E0BE016757D6
:101B80007F4FCE018D569F4F0E94E4B52EC0C757A0
:101B9000DF4FC882D982EA82FB82C958D0409E01B9
:101BA0002B563F4F44E050E0BE0167577F4FCE01B8
:101BB0008D569F4F0E94E4B5C757DF4F1882198298
:101BC0001A821B82C958D04004E0015071F09E0176
:101BD0002B563F4F44E050E0BE0167577F4FCE0188
:101BE0008D569F4F0E94E4B5F0CF1F5F153009F06E
:101BF00092CF84E190E0CF56DF4F99838883C1591B
:101C0000D0409E012B563F4F42E050E0BE016F5640
